:020000040040BA
:1040000030540020E5E5400019504000B552400012
:10401000A5E64000A5E64000A5E64000000000003F
:10402000000000000000000000000000A1E94000C6
:10403000A5E640000000000001EA400065EA4000FB
:10404000A5E64000A5E64000A5E64000A5E6400044
:10405000A5E64000A5E64000A5E6400000000000FF
:10406000A5E64000F50B410000000000B1C1400092
:10407000C5C14000F5DD4000A5E64000A5E64000D2
:10408000A5E64000A5E6400005DE4000C5934000DF
:10409000090C4100A5E64000A5E640005954400047
:1040A000A5E64000A5E64000A5E64000A5E64000E4
:1040B000A5E64000A94A4000A5E640000000000037
:1040C00000000000000000000000000000000000F0
:1040D00000000000000000000000000000000000E0
:1040E00000000000000000000000000000000000D0
:1040F000000000000000000000000000A5E64000F5
:10410000C5D24000A5E6400000000000000000000D
:10411000000000000000000000000000000000009F
:10412000000000000000000000000000000000008F
:10413000000000000000000000000000000000007F
:10414000000000000000000000000000000000006F
:104400009C26010010B5054C237833B9044B13B139
:104410000448AFF300800123237010BDE80C002096
:1044200000000000BC5941000C4B43B10C480D4941
:1044300010B5AFF300800C48036823B910BD0A48DB
:10444000036833B97047094B002BF7D0BDE8104023
:104450001847064B002BF5D0184700BF000000009E
:10446000BC594100EC0C0020BC5941000000000088
:104470000120704770470120704700207047704747
:1044800001207047014B1878704700BF0C0D0020C9
:104490007047000058B908B5054B1B78012B00D0B8
:1044A00008BD044B1B68002BFAD09847F8E770470B
:1044B000100D0020040D002008B50C4B9847C37860
:1044C0000B4A1370012B0CD101220A4B1A700022E7
:1044D000094B1A80094B9847094B1B681BB1984739
:1044E00001E0084B9847012008BD00BFF9BD40001E
:1044F0000C0D0020100D00200E0D0020D50B4100EA
:10450000040D0020E10B410008B5054B1B78012B81
:1045100000D008BD0022034B1A70034B9847F8E700
:104520000C0D0020100D0020E10B410010B582B0F1
:10453000074B00930B46024600218420054CA04700
:1045400018B9054A13680133136002B010BD00BFEB
:1045500095444000FDD94000080D0020014B186033
:10456000704700BF040D00202DE9F0474FF40046CE
:10457000BF4B5E600B20BF4CA0470C20A047BE4B3A
:104580004FF0400CC3F810C0C3F8A0C0C3F834C04B
:104590004FF0807EC3F810E0C3F8A0E0C3F834E029
:1045A000B64A01271761C2F8A0705763022414614C
:1045B000C2F8A04054631C61C3F8A0405C631F664E
:1045C000C3F890705F655F62C3F88070196F3943FC
:1045D0001967596F21F0010159675F604FF480310D
:1045E0001966C3F8901059655962C3F88010186FA6
:1045F00008431867586F20F48030586759601C6171
:10460000C3F8A0405C6304205861C3F8A00058665A
:10461000C3F8900058655862C3F88000196F21F004
:1046200004011967596F21F00401596718211966AF
:10463000C3F8901059655962C3F880101D6F25F0BA
:1046400018051D675D6F25F018055D675960082521
:104650001D66C3F890505D655D62C3F88050196FA8
:1046600021F008011967596F21F0080159675D6051
:1046700010211966C3F8901059655962C3F880106B
:10468000D3F8708028F01008C3F87080D3F87480D5
:1046900028F01008C3F8748059604FF48028C3F8DC
:1046A0001480C3F8A0804FF02009C3F81490C3F819
:1046B000A090C3F810C0C3F8A0C0C3F834C0C3F8BA
:1046C00010E0C3F8A0E0C3F834E01761C2F8A070AE
:1046D00057631461C2F8A04054634FF4007CC3F8E0
:1046E00060C0C3F890C0C3F854C0C3F824C0C3F876
:1046F00080C01C6F44EA0C041C675C6F24F40074D7
:104700005C67C3F804C04FF480641C66C3F8904033
:104710005C655C62C3F880401F6F27431F675F6F53
:1047200027F480675F675C604FF4006EC3F810E0A9
:10473000C3F8A0E0C3F834E04FF400275F61C3F88A
:10474000A0701F66C3F890705F655F62C3F88070E9
:104750001F6F27F400271F675F6F27F400275F672D
:104760004FF480175F61C3F8A0701F66C3F89070A4
:104770005F655F62C3F880701F6F27F480171F6743
:104780005F6F27F480175F674FF480575F61C3F84E
:10479000A0705F66C3F890705F655F62C3F8807059
:1047A0001F6F27F480571F675F6F27F480575F677D
:1047B0004FF400575F61C3F8A0704FF480775761E2
:1047C000C2F8A0704FF48048C3F86080C3F89080AE
:1047D000C3F85080C3F82480C3F88080D3F870A059
:1047E0002AF4804AC3F870A0D3F874A02AF4804A4F
:1047F000C3F874A0C3F81080C3F8A080C3F8308059
:104800005E61C3F8A0604FF400365E61C3F8A0603B
:104810001066C2F8900050655062C2F88000166FB2
:1048200026F004061667566F26F004065667506099
:104830001566C2F8905055655562C2F88050106FE9
:1048400020F008001067506F20F008005067556096
:104850000B4DD5F8140140F03000C5F8140151613A
:10486000C2F8A0105166C2F890105165516209E07B
:1048700050140E402DE34000000E0E4000100E407C
:1048800000020E40C2F88010116F21F01001116774
:10489000516F21F010015167C2F81090C2F8A0903A
:1048A000C2F83490C2F810C0C2F8A0C0C2F830C03C
:1048B0004FF400015961C3F8A0105966C3F8901075
:1048C00059655962C3F88010196F21F40001196706
:1048D000596F21F400015967C2F860E0C2F890E016
:1048E000C2F854E0C2F824E0C2F880E0116F21F46D
:1048F00000611167516F21F400615167C2F804E053
:104900001466C2F8904054655462C2F88040116F3A
:1049100021F480611167516F21F480615167546007
:104920001F66C3F890701F655F62C3F880701A6FCE
:1049300022F480721A675A6F22F480725A671F61DC
:10494000C3F8A0701F63BDE8F08700BF08B5034B34
:1049500053F8203003B1984708BD00BF7010002005
:1049600010B582B0036B0193002400E00134172CD2
:1049700009D8064B53F82420019B1A42F6D0204652
:10498000034B9847F2E702B010BD00BFB04A4100A8
:104990004D49400000230360064A4260064A826097
:1049A0004FF48022C2600222027442748374C37482
:1049B000037570470000DC05808D5B00036C1943B4
:1049C0000164704710B58B7C23B34FF000434A68F5
:1049D0008C686400B2FBF4F2013A120292B2134303
:1049E0000A7C120602F0706213434A7C120702F03E
:1049F00040521343CA6813434360CB7C63B14FF00A
:104A000080730A7D52B90022134303640968054B81
:104A1000984710BD0023DAE70023F2E74FF4801235
:104A2000F2E700BFBD49400008B5036B13F0807F7B
:104A300001D0192008BD01230360064B98470023CD
:104A400004E00021044A42F823100133172BF8D95F
:104A5000002008BDC549400070100020B1F1FF3FA3
:104A600004D0044B53F82130436270474FF0FF33BA
:104A700043627047B04A410010B5084C44F8212009
:104A8000074A4FF00054C2F880411B01DBB282F8A4
:104A90001D331460034B984710BD00BF70100020F9
:104AA00000E100E05D4A400008B50248024B98472B
:104AB00008BD00BF008003406149400042F26663C8
:104AC00003FB00F008E000BF00BF00BF00BF00BF55
:104AD00000BF00BF00BF01380028F4D170470000BC
:104AE000124B1A68126802601A6853684360936830
:104AF0008360D368C3600E4B1B68D9680161196974
:104B00004161596981619969C161D9690162196A13
:104B10004162596A81629B6AC36213690363054BF0
:104B20001B68436353698363704700BFC41300204D
:104B30006C110020781100200D4B1A6892690260F8
:104B40001B68DB6943600B4B1B681A6882605A68FC
:104B5000C2609B680361002306E05A1D064951F8B4
:104B6000231040F822100133092BF6D9704700BFFB
:104B7000C41300206C110020E01000200A2308E07C
:104B800003F180420A3A044951F8231040F82210F8
:104B90000133182BF4D97047E0100020192308E0E6
:104BA00003F18042193A064951F8231040F82210C7
:104BB00001331F2BF4D9024BD3F88030C361704707
:104BC000E0100020FEE70000284B5B6A13F0010FA5
:104BD00005D0EFF30583042B01D004207047234B4D
:104BE0005B6A13F0020F05D0EFF30583052B01D0AC
:104BF000052070471D4B5B6A13F0080F05D0EFF3DB
:104C00000583062B01D006207047184B5B6A13F012
:104C1000800F05D0EFF305830B2B01D00B207047DD
:104C2000124B5B6A13F4807F05D0EFF305830C2BE6
:104C300001D00C2070470D4B5B6A13F4806F05D0D8
:104C4000EFF305830E2B01D00E207047074B5B6AF4
:104C500013F4006F05D0EFF305830F2B03D00F2063
:104C60007047002070470020704700BF00ED00E053
:104C700000230FE0114AD2F80412A3F12000012210
:104C80008240114205D0EFF3058203F110009042FB
:104C900013D10133312B0FD81F2BEBD8074AD2F891
:104CA000001201229A401142F3D0EFF3058203F182
:104CB00010009042EDD070470020704700E100E006
:104CC00010B5EFF308831C4613F0070F00D01C1F2C
:104CD000174B5B6813F0010F01D0B7EE000A154BBC
:104CE0005B6813F4006F15D0134A22F001026FF0D5
:104CF000060E002303F1807344F8043C44F8082CAA
:104D00000E4B44F80C3C203C84F3088884F309885B
:104D1000704710BD0A4B9847034628B1094A22F054
:104D200001026FF00E0EE5E7074B98470346F5E7E3
:104D300030EF00E000ED00E0E14D4000C54B4000E9
:104D4000C94B4000C14C4000714C4000064A93687A
:104D500023F07F4323F4706343F0254343F4E0637F
:104D60009360024B1360704700140E40080000A5CA
:104D7000024B1860024B1960704700BF641100209D
:104D8000C0130020014B1870704700BF110D0020A8
:104D9000C0F30800014B1880704700BFDC100020F2
:104DA00008B5024650B9084B0849196008495960CE
:104DB000002199601046074B984708BD024B0649F1
:104DC000196006495960F5E7FC01002098020020AF
:104DD0000802002015B74000E0000020F800002085
:104DE00070B564201B4B984700221B4B1A7062B6AB
:104DF00061B60120194B9847194B9847194B9847B2
:104E000007E01948194B98470028FAD0184B1B782F
:104E1000DBB9114B1B78002BFBD0154B1B7813B95A
:104E200000210D4A117010484D220270114A157868
:104E300045708370104E34682A46214604300F4B6B
:104E400098472C4434600020DEE7013B084A137089
:104E5000DFE700BFBD4A400070110020A14D4000B7
:104E600005BE4000ED0B41008013002021B740003B
:104E700068110020D4100020D8100020D12041005B
:104E8000F8B505464F4B4FF0FF32C3F88020C3F80A
:104E90008420C3F88021C3F8842103F540635A6855
:104EA00042F020625A605A6A22F400425A62464B2B
:104EB0009A6D5A6C22F040625A645A6C42F0006259
:104EC0005A64424C4FF4804363634FF4006363635E
:104ED0004FF48073636302203D4EB0474FF0807300
:104EE00063630420B0473B4F01237B630420B0473A
:104EF00002237B6340236363374A136823F0010373
:104F00001360364B5A6F42F480725A675A6F42F4FC
:104F100000725A67324AD2F8143143F44063C2F83F
:104F20001431002383F311882E4B1D60EA6A12F0BE
:104F3000040F26D069682C4B19602B4B1B6820335B
:104F40002A490B6012F0100F1FD148330B60284D17
:104F50002846284B9847244B1F6807F12004403D02
:104F600007F1600E2E4620686168A268E3680FC6EC
:104F7000103435467445F5D13A6E1F4BC3F8802086
:104F800006E02968184B1960D7E71B481B4B984768
:104F9000144B1B689B6813F4007F03D0134A1368FB
:104FA00004331360164B1B7813B90322154B1A8078
:104FB000154BD96A154A11609A6A154B1A60154B40
:104FC0009847F8BD00E100E000000140000E0E40EF
:104FD000BD4A400000100E4010E000E000400440D8
:104FE00000020E406C110020C41300207811002034
:104FF00020110020ED524000E0100020E15240005E
:10500000110D0020DC10002000ED00E0D010002089
:1050100074110020C14C40006FF0060E70477047BD
:1050200070B58AB00446402200217F487F4B9847E4
:1050300023782A3B2A2B37D8DFE813F02B003600E1
:1050400036003600360036003600360036003600B0
:1050500036003600360036003600360036003600A0
:10506000360036003600360036003600EE00EB0023
:10507000360036003600860036008C0036003600DA
:105080003600C20036003600360036003B004B00CA
:10509000770065490B462A2203F8012B644A106801
:1050A000C1F8010092889A805F48624B98470AB025
:1050B00070BD5D4B52221A705F4A12785A705F4A77
:1050C00012885A805E4A12685A605E4A12689A6074
:1050D000EAE7554B53221A7062785A706378032BB3
:1050E000E2D8DFE803F0020A121A574C2046574B69
:1050F00098473C2304F8013CD6E7534C2046544BD8
:1051000098473C2304F8013CCEE74F4C2046514BD6
:1051100098473C2304F8013CC6E74B4C20464E4BD5
:105120009847202304F8013CBEE73F4C54232370EA
:105130004A4D102128684A4B9847C2B262702968CC
:10514000A01C484B9847AFE7374B47221A70042200
:105150005A70A9E7344B49221A7062785A70637802
:105160004BB1012B10D0022B14D0032B1BD02E4B94
:105170005E609D6098E73C4E3C4D3D4B3D4A92E859
:10518000030018601971F2E73B4E3C4D3C4A384B26
:105190001A60ECE73B4E3C4D354B3C4A92E803002D
:1051A00018609980E3E73A4E68463A4B9847009D6D
:1051B00035442F4B384A92E8030018601971D6E73E
:1051C0002579637905EB0325A37905EB0345E3799D
:1051D00005EB0365314B1D6013484D230370637865
:1051E0004370A37883706278294604301D4B98473A
:1051F000A378002B3FF458AF627829490A70013B2D
:1052000028490B701544254B1D600122264B1A704E
:105210004AE7264B984747E7254BBB221A601A22DC
:105220005A60224B98473FE780130020CD2241006F
:10523000104B410021B74000110D0020DC10002070
:10524000D01000207411002084130020E14A400097
:10525000394B40007D4B40009D4B4000C013002067
:105260005D264100D120410010000020E80C002004
:105270008C130020184B4100E80C00203024002043
:10528000627373003024002030540020204B410012
:105290003054002081234100284B4100D8100020C9
:1052A000D410002068110020701100204D4D4000E6
:1052B00090140E4072B671B6EFF30383EFF30982D8
:1052C000EFF30881DFF814D02DE9FE4F6846FFF7B1
:1052D000D7FDBDE8FE4F8D467047000080130020CB
:1052E000F1EE101AA0EC200A01607047A0EC108AC1
:1052F000704700BF10B51720234CA0471820A047C7
:10530000224B4FF480321A66C3F890205A655A62D5
:10531000C3F88020196F11431967596F21F4803148
:1053200059675A6001225A66C3F890205A655A623A
:10533000C3F88020196F11431967596F21F00101DB
:1053400059675A60A3F5206340F21262DA644FF4A1
:1053500000621A600E4B0F4A5A6041225A620521C0
:1053600019600D4A5A644FF4F572DA6500229A65A5
:1053700019640A4B1A700A4B4FF400021A6070222B
:1053800083F8172310BD00BF2DE34000000E0E4030
:10539000000001400406090001C4000ACC130020EB
:1053A00000E100E010B54FF40002124BC3F880207A
:1053B000BFF34F8FBFF36F8F0F4B4FF480321A66DE
:1053C000C3F890205A655A62C3F88020196F21F4FF
:1053D00080311967596F21F4803159671A601A6159
:1053E000C3F8A0205A631720044CA0471820A047F8
:1053F00010BD00BF00E100E0000E0E4081E3400060
:10540000642800D964200F4AD36D03FB00F30E49D2
:10541000A1FB03135B09936548B10A4B5A6C22F058
:1054200040625A645A6C42F080625A647047134674
:10543000526C22F040625A645A6C42F000625A6424
:10544000704700BF000001401F85EB51014B1888D9
:10545000704700BFD01300200F4B1B6A13F0010FE1
:1054600006D000220D490A700D490A600D490A60F4
:1054700013F0400F0ED00122084B1A70064B9A69A8
:10548000094BB3FBF2F3064A1360C3EB03139A0014
:10549000044B1A60704700BF00000140CC1300208D
:1054A000C8130020D01300201F1A0500014B1870EC
:1054B000704700BF00010020064B1B7823B94FF452
:1054C0000062054B1A6370474FF40062024B5A6347
:1054D000704700BF00010020000E0E40064B1B78F5
:1054E00023B94FF40062054B5A6370474FF40062D2
:1054F000024B1A63704700BF00010020000E0E40EF
:105500002DE9F04186B00F4616469846B8B9344B9F
:10551000984704460025049598238DF8043001230C
:105520008DF805308DF8065002238DF8083005AB54
:1055300003938DF8075020462A4B98470EE02A4BDC
:1055400098470446E6E72046284B9847002044E069
:105550009DF8153008F805300135EDB2B54238D266
:105560008DF814708DF8155000238DF80630322216
:1055700001A920461E4B9847A379DBB2022B0BD022
:1055800020461C4B9847322201A92046184B9847C9
:10559000A379DBB2022BD6D101238DF8063032225B
:1055A00001A92046124B9847A379DBB2022BCFD03A
:1055B0002046104B9847322201A920460C4B9847B1
:1055C000A379DBB2022BC3D02046084B98470020BA
:1055D00003E02046054B9847012006B0BDE8F08166
:1055E000C50B4100D5764000CD0B4100E976400067
:1055F00001774000B17840002DE9F04186B00C46BB
:1056000017469846D8B9264B984705460026049673
:1056100098238DF8043001238DF8053002238DF88E
:10562000063003238DF8083005AB03938DF807404F
:105630008DF8156028461B4B9847344605E01A4BF9
:1056400098470546E2E70134E4B2BC4221D28DF826
:10565000144018F804308DF81630322201A928467B
:10566000124B98470646AB79DBB2022BEBD02846AB
:105670000F4B9847322201A928460C4B9847064603
:10568000AB79DBB2022BDED028460A4B98470026C6
:1056900002E02846074B9847304606B0BDE8F08147
:1056A000C50B4100D5764000CD0B4100017740008D
:1056B000B1784000E97640002DE9F04387B00C4610
:1056C00090461F46DDF83890D8B9274B98470546D5
:1056D0000026049698238DF8043001238DF80530B8
:1056E00002238DF8063003238DF8083005AB0393B1
:1056F0008DF807408DF8156028461C4B98473446B6
:1057000005E01B4B98470546E2E70134E4B2BC4292
:1057100023D204EB08038DF8143019F804308DF807
:105720001630322201A92846124B98470646AB791B
:10573000DBB2022BE9D028460F4B9847322201A951
:1057400028460C4B98470646AB79DBB2022BDCD0DF
:1057500028460A4B9847002602E02846074B984700
:10576000304607B0BDE8F083C50B4100D576400058
:10577000CD0B410001774000B1784000E976400050
:10578000F8B506460D461746344BAA221A70112268
:105790005A700222F021324CA047012801D000208B
:1057A000F8BD2C0AEDB22D4B1C705D709C70DD7045
:1057B0001C715D7100229A719022DA7167B18222A8
:1057C0001A72264B0922C2213046254FB8470128BC
:1057D00006D001280BD0F8BD0222204B1A72F0E748
:1057E0001E4B0922C22130461E4EB047F1E71B4B2B
:1057F0001B789C4201D00020F8BD184B9B789C423E
:1058000001D00020F8BD154B1B799C4201D000202F
:10581000F8BD124B5B789D4201D00020F8BD0F4BC4
:10582000DB789D4201D00020F8BD0C4B5B799D4296
:105830000BD10A4B9B7953B9084BDB79902B08D1DC
:10584000064B1B7A022B06D1F8BD0020F8BD0020C4
:10585000F8BD0020F8BD0020BDE700BFD413002034
:10586000F95540000155400010B50022054B1A7053
:1058700029B91121034B0122034CA04710BD10216F
:10588000F8E700BFD4130020F955400010B50022FE
:10589000054B1A7029B92821034B0122034CA0475C
:1058A00010BD2921F8E700BFD4130020F9554000AE
:1058B00070B506460A4CAA23237011236370234651
:1058C0000222F021074DA847FF232370012800D0B2
:1058D00070BD23460122C0213046A847F8E700BF2B
:1058E000D4130020F955400010B539B90022044BFB
:1058F0001A7001223621034CA04710BD0322F6E79F
:10590000D4130020F955400038B505460C4BAA22A7
:105910001A7012225A700222F0210A4CA047012864
:1059200001D0002038BD064B0322BF212846064C7B
:10593000A047012801D0002038BD014B987838BD20
:10594000D4130020F95540000155400038B50D46EC
:10595000094B0E228421094CA047012801D00020C8
:1059600038BD054B186859689A6828606960AA6054
:105970009B89AB810E2038BDD41300200155400017
:1059800010B50B462C227021014CA04710BD00BF62
:10599000F95540002DE9F04184B000238DF80F3017
:1059A0000139062945D8DFE801F00806040D0F117A
:1059B0001300214D02E0214D00E0214D80460120E1
:1059C000002411E01F4DF9E71F4DF7E71F4DF5E7E4
:1059D0001F4DF3E70DF10F03024640461D4EB04741
:1059E0003C44E4B20134E4B201280BD123462F5DDC
:1059F00047B1621CA95C012FECD902332B44781EFD
:105A0000C0B2E9E7012804D0012809D004B0BDE8FC
:105A1000F081114B0222FF2140460E4CA047F3E7D4
:105A20000E4B00930D230B22F92140460C4CA0474E
:105A3000ECE70020EAE700BF844B4100344D410011
:105A4000B44D4100344B4100084C4100B44C41007E
:105A5000584C4100F9554000304B4100384E410050
:105A6000B956400008B50721014B984708BD00BF53
:105A70009559400010B5274900238B72CB720B73E8
:105A800040F2DC528A806422CA800B8021F8083FF1
:105A90000620214B98470B20204B984780B90C20BB
:105AA0001E4B984788B900221A4B5A801C4B9847C6
:105AB00001211C4B984701280CD0164B987A10BD39
:105AC00019490B20144B9847E9E718490C20124B51
:105AD0009847E8E701220F4B9A72114B984705212E
:105AE000134B9847034650B10A4AD372002BE4D0B7
:105AF0000B4B98470F4B9847064B5880DDE7084CF7
:105B0000A0470021074B9847A0470321084B98471F
:105B10000346E9E734140020B5804000E9804000E6
:105B2000CD0B4100355C4000381400203A140020B1
:105B3000655E4000F55D4000014B987A704700BFFC
:105B40003414002008B5274B9B7A8BB9264A13786A
:105B500024490888254921F813000133DBB213706A
:105B60000F2B02D90022204B1A7000231A461FE087
:105B70001F4B98471F4B98471A4B18801E4B98474E
:105B800060B1184A13881289934203D80022154B3A
:105B90001A80DBE79B1A134A1380D7E70022114BC8
:105BA0009A72D3E7114931F813100A440133DBB27A
:105BB0000F2BF7D912090B4B1B7B4BB109498B8873
:105BC000C9885B1A9A420CD80022064B1A7308BD8A
:105BD00004498B88C9880B449A4202D30122014BA5
:105BE0001A7308BD34140020120D00201414002074
:105BF000CD0B4100855D4000355F4000014B187BB7
:105C0000704700BF34140020014B1888704700BF54
:105C10003414002008B5014B984708BD415F40008F
:105C200008B5024B9847024B984708BDCD0B410081
:105C3000495F400030B587B005460C4600238DF81B
:105C4000073072228DF808208DF80B3001228DF874
:105C500009208DF80C200DF10702049202228DF824
:105C60000A200593434B9847322202A92846424B0B
:105C70009847002C43D1012402238DF80A30802359
:105C80008DF80B3001238DF807309C4244D08F23D0
:105C90008DF80B3003238DF80A30012C43D09DF88A
:105CA000073003F0F00343F005038DF807300223BB
:105CB0008DF80A30012C3DD0AA238DF80B3001233A
:105CC0008DF807309C423CD007238DF80730F9232C
:105CD0008DF80B30012C3BD005238DF80730802345
:105CE0008DF80B30012C3AD02846244B9847012CD4
:105CF0003CD00022224B1A70204607B030BDA823AA
:105D00008DF80B3001238DF80730322202A9284686
:105D1000194B98470446AFE7322202A92846164B92
:105D200098470446B3E7322202A92846124B984707
:105D30000446B4E7322202A928460F4B984704468E
:105D4000BAE7322202A928460B4B98470446BBE724
:105D5000322202A92846084B98470446BCE7322263
:105D600002A92846044B98470446BDE70122044B8C
:105D70001A70C1E7D576400001774000E97640000F
:105D8000130D002030B587B004460023059301AB06
:105D9000049372238DF8083001238DF809309C2379
:105DA0008DF80B3002238DF80C3003238DF80A3068
:105DB0000C4B9847322202A920460B4B98470546C8
:105DC00020460A4B9847012D04D00020084B18703C
:105DD00007B030BD9DF804009DF8053000EB0320AE
:105DE00080B2F5E7D576400001774000E9764000C3
:105DF000130D002030B587B004460023059301AB96
:105E0000049372238DF8083001238DF80930C023E4
:105E10008DF80B3002238DF80C3003238DF80A30F7
:105E20000C4B9847322202A920460B4B9847054657
:105E300020460A4B9847012D04D00020084B1870CB
:105E400007B030BD9DF804009DF8053000EB03203D
:105E500080B2F5E7D576400001774000E976400052
:105E6000130D0020F0B587B00646002305930DF111
:105E70000703049372238DF8083001238DF809304D
:105E8000D9228DF80B208DF80C3002238DF80A30C2
:105E90004901C9B241F010018DF80710214B984714
:105EA000322202A93046204B98470546D7238DF869
:105EB0000B3021238DF8073001280BD030461B4BC7
:105EC0009847DC238DF80B3003238DF80A3000242B
:105ED000274608E0322202A93046134B9847054670
:105EE000ECE70134A4B2012D18D1BFB9092C15D8A3
:105EF00019200F4B984730460A4B9847322202A987
:105F00003046094B984705463046084B98479DF860
:105F1000073013F0010FE4D00127E2E7384607B05D
:105F2000F0BD00BFD576400001774000E976400023
:105F300075F84000014B1878704700BF130D002022
:105F40000048704744140020A84BDB78032B00F274
:105F50004081A64B1B793F2B00F23D81A34B5B791F
:105F6000072B00F23A81A14B9B79082B00F2378175
:105F70009E4B1B7A013BDBB2022B00F232819B4B22
:105F80005B7A032B00F22F81984B9B7A072B01D968
:105F90000020704710B586B0044600230593722395
:105FA0008DF8083001238DF809300DF107020492B5
:105FB0008DF80C308E4B984780238DF80B300323DF
:105FC0008DF80A30322202A920468A4B98470128D0
:105FD00017D1864B1B78D3B19DF8073043F01003DF
:105FE0008DF8073002238DF80A30322202A92046AC
:105FF000804B9847012811D020467F4B98470020BE
:1060000003E020467C4B9847002006B010BD9DF869
:10601000073023F010038DF80730E3E782238DF873
:106020000B30724B5B788DF80730322202A9204684
:10603000704B9847012817D18D238DF80B304023E2
:106040008DF80730694B9B7813B148238DF80730E2
:10605000322202A92046674B9847012809D02046E2
:10606000654B98470020D0E72046634B98470020B7
:10607000CBE78E238DF80B305C4AD3789B01DBB2E3
:10608000127902F03F0213438DF80730322202A941
:106090002046584B9847012804D02046564B984735
:1060A0000020B2E78F238DF80B30504A53795B0103
:1060B000DBB2927902F00F0213438DF807303222DF
:1060C00002A920464B4B9847012804D020464A4B52
:1060D0009847002099E7A9238DF80B30434BDB79D3
:1060E0008DF80730322202A92046424B98470128FA
:1060F0000CD1AA238DF80B303C4B1B7A022B18D005
:10610000032B1AD0012B06D000207EE720463A4B05
:106110009847002079E78DF80730322202A92046FF
:10612000344B984701280CD02046334B9847002029
:106130006BE702238DF80730EFE703238DF8073074
:10614000EBE7B3238DF80B30284B5B7A03F00303A6
:106150008DF80730322202A92046264B98470128A5
:1061600004D02046244B984700204EE7D9238DF8D1
:106170000B3003238DF80A30322202A920461D4B32
:106180009847012804D020461B4B984700203CE745
:106190009DF8073003F0F80343F01003134A927A96
:1061A00002F0070213438DF8073002238DF80A30FE
:1061B000322202A920460F4B9847012804D02046DE
:1061C0000D4B9847002020E720460B4B98470120B5
:1061D0001BE7002070470020704700207047002018
:1061E0007047002070470020704700BF4414002013
:1061F000D576400001774000E976400000FB01F0D1
:10620000C0F3C71070470000F0B587B004460E46D3
:10621000234B9847002304938A238DF804300123ED
:106220008DF805308DF808300DF1170303933427EE
:106230008DF8077002238DF8063033788DF817300B
:10624000322201A92046174DA8478DF807703378F0
:106250008DF81730322201A92046A8478DF8077023
:1062600033788DF81730322201A92046A84735230C
:106270008DF8073073788DF81730322201A9204647
:10628000A84736238DF80730B3788DF817303222BF
:1062900001A92046A8472046034B984707B0F0BD08
:1062A000D576400001774000E9764000F0B587B030
:1062B0000446002505958A238DF8083001268DF8BF
:1062C00009608DF80C600DF107030493254B984786
:1062D00055238DF807308DF80B5002238DF80A30C6
:1062E000322202A92046204DA84703238DF807300B
:1062F0008DF80B60322202A92046A8478DF807606E
:1063000004238DF80B30322202A92046A847072328
:106310008DF8073030238DF80B30322202A9204649
:10632000A8470F278DF8077031238DF80B303222E4
:1063300002A92046A8478DF8077032268DF80B6019
:10634000324602A92046A8478DF8077033238DF8FE
:106350000B30324602A92046A8472046034B9847F7
:1063600007B0F0BDD576400001774000E9764000E7
:10637000F0B583B007460C46802900D980240C4B29
:106380001C700C4E214630780B4DA8478DF8040048
:1063900021467078A8478DF805002146B078A847B7
:1063A0008DF8060001A93846044B984703B0F0BDAC
:1063B00001010020140D0020FD6140000962400031
:1063C00010B5054B0C888A781C809A70034B19789D
:1063D000034B984710BD00BF140D002001010020A1
:1063E00071634000F0B58FB006460F4614460EADFF
:1063F00005F8342D19460DF105000D4B984758232B
:106400008DF8283000230D938DF82B700C950134F6
:106410008DF82C4001238DF8293002238DF82A3085
:1064200032220AA93046034B98470FB0F0BD00BF97
:10643000D12041000177400010B586B001248DF8CD
:1064400004408DF8052058238DF80830002305936B
:106450008DF80B1001AB049302238DF80C308DF8EE
:1064600009408DF80A30322202A9024B984706B043
:1064700010BD00BF0177400030B585B00546202231
:10648000364B1A630120364B98472846354B9847C0
:10649000354B93E803000190ADF8081001AB0622DC
:1064A00000212846314CA0470446012815D0012C74
:1064B0001AD0012C1FD0012C24D0012C29D0012C62
:1064C0002ED0012C37D0012C3CD02846284B9847A1
:1064D000012C3ED0204605B030BD9622062128462C
:1064E000244B98470446E2E7082207212846214B1F
:1064F00098470446DDE77C22092128461D4B984732
:106500000446D8E780220A2128461A4B98470446B9
:10651000D3E780220B212846164B98470446CEE746
:1065200004AB002243F8042D04220C2128460F4C12
:10653000A0470446C5E70022F62128460D4B9847A0
:106540000446C0E70122FF2128460A4B984704462B
:10655000BBE70122084B1A70BCE700BF00100E40D9
:1065600075F84000D5764000484E4100E563400094
:10657000E976400039644000170D0020F0B587B07F
:106580000646174B9847174C202525630220164BCB
:10659000984758238DF808300023059301AB0493E6
:1065A00002238DF80C3001228DF80920FF218DF88F
:1065B0000B108DF80A308DF804208DF8053032224A
:1065C00002A93046094B984707463046084B984782
:1065D0006563012F14BF0020012007B0F0BD00BF8C
:1065E000D576400000100E4075F84000017740005D
:1065F000E976400010B586B004468DF808100023F7
:106600000593E7238DF80B300DF107030493012365
:106610008DF80C308DF8093003238DF80A303222C2
:1066200002A90A4B9847012801D006B010BD9DF879
:10663000073043F001038DF8073002238DF80A304C
:10664000322202A92046014B9847EEE7017740002D
:1066500010B586B004468DF80810002305930DF19F
:106660000703049301238DF80C308DF809300623BD
:106670008DF80B3003238DF80A30322202A9224B09
:1066800098479DF8073063F07F038DF807300223A9
:106690008DF80A30012818D000238DF807300C231C
:1066A0008DF80B30012816D00D238DF80B30012802
:1066B00017D00E238DF80B30012818D00F238DF83A
:1066C0000B30012819D006B010BD322202A9204695
:1066D0000D4B9847E0E7322202A920460A4B984723
:1066E000E2E7322202A92046074B9847E1E732222F
:1066F00002A92046044B9847E0E7322202A920462F
:10670000014B9847DFE700BF0177400010B586B026
:1067100004468DF8081000230593E7238DF80B300D
:106720000DF10703049301238DF80C308DF8093027
:1067300003238DF80A30322202A90A4B9847012818
:1067400001D006B010BD9DF8073023F001038DF88D
:10675000073002238DF80A30322202A92046014B6D
:106760009847EEE70177400070B504462022214BA0
:106770001A630A20204B98472046204B9847102147
:1067800020461F4EB047054612212046B047064618
:10679000012D0ED0012E12D0012D16D0012E1AD0AF
:1067A0002046184B9847012D1BD0012E1DD028469E
:1067B00070BD10212046144B98470546EAE7122188
:1067C0002046114B98470646E6E7102120460F4B1E
:1067D00098470546E2E7122120460C4B98470646AB
:1067E000DEE701220A4B1A70DFE70122094B1A701B
:1067F000DDE700BF00100E4075F84000D576400080
:10680000F5654000E9764000516640000D674000A4
:10681000180D0020190D002010B1034B1878704797
:10682000024B1878704700BF190D0020180D00208A
:1068300030B587B004460D4600220592A8238DF896
:10684000083001238DF809308DF80B200DF1070277
:1068500004928DF80C3002238DF80A30124B9847C1
:10686000012D0ED0022D15D000238DF807303222D5
:1068700002A920460D4B984720460D4B984707B07C
:1068800030BD03238DF80730322202A92046074B82
:106890009847F1E702238DF80730322202A92046FB
:1068A000024B9847E8E700BFD576400001774000EB
:1068B000E976400030B587B072238DF800300123AF
:1068C0008DF8013000238DF802308DF80330082256
:1068D0008DF8042004AA029203938DF81000C0F3EF
:1068E00007238DF81130C0F307438DF81230000EE6
:1068F0008DF813008DF81410C1F307238DF81530AF
:10690000C1F307438DF81630090E8DF81710084CA7
:10691000A047084B9847A04732226946064B984744
:106920000546A047054B9847284607B030BD00BF35
:10693000C50B4100D576400001774000E976400064
:1069400030B587B00D4672238DF8043001238DF8E1
:10695000053000238DF806308DF8073004228DF8BD
:10696000082005AA039204938DF81400C0F30723AE
:106970008DF81530C0F307438DF81630000E8DF8F2
:106980001700184CA047184B9847A047322201A97E
:10699000164B98470446012808D0124B9847144BD1
:1069A0009847012C0DD0204607B030BD01238DF84B
:1069B00006300C4B9847322201A90C4B98470446ED
:1069C000EBE79DF814309DF8152003EB02239DF8AA
:1069D000162003EB02439DF8172003EB02632B60A4
:1069E000E1E700BFC50B4100D576400001774000CC
:1069F000E97640002DE9F04E82B082468946934602
:106A00001BB11E46002501272FE00127012F40D092
:106A1000012F49D0012F4DD0012F51D04FF4000349
:106A200001932F4B98470446012F4FD1019B13F43C
:106A3000000F4BD00A9920462A4B984700284DD189
:106A400001A92948294B98470746EDE7EA18B25CA7
:106A50004FEAC30E02FA0EF211440133DBB2A34235
:106A6000F4D3012F0DD02544EDB228464D45CDD2AB
:106A7000A9EB0504042C28BF0424E4B20023194622
:106A8000EDE700F1201000F58070194B984707469C
:106A9000E9E74FEA0A4101F4FE0101F5000112485D
:106AA000134B98470746B3E749461248104B98479F
:106AB0000746AFE7594610480D4B98470746ABE7E6
:106AC000F2210E480A4B98470746A7E71FB9052051
:106AD00002B0BDE8F08E9DF80700F9E70620F7E761
:106AE000A57D4000BD7D40001001200041694000AF
:106AF000B56840001801200014012000FC002000AF
:106B000010B584B00A4B93E8030002908DF80C1086
:106B10003223009302AB002205210120054CA0473F
:106B2000034610B90121044A1170184604B010BD83
:106B3000504E4100F56940001A0D002070B5074D18
:106B40004FF480466E630A20054CA0472E6340F246
:106B50001310A047034B984770BD00BF000E0E40B6
:106B600075F84000016B400030B583B00D4632230C
:106B700000930023024604213120074CA04704461D
:106B800010B1204603B030BD29460448044B984755
:106B90000128F6D00524F4E7F56940002001200023
:106BA0004169400010B584B08DF80C100B0A8DF8C7
:106BB0000D300B0C8DF80E30090E8DF80F103223AE
:106BC000009303AB024604212120024CA04704B0ED
:106BD00010BD00BFF569400008B5044B1B780BB130
:106BE000002008BD024B984708BD00BF1A0D0020C9
:106BF000016B40002DE9F04383B059B1012904D065
:106C00000124204603B0BDE8F08340F65D0740F65E
:106C1000050503E040F2DD7740F2857580464FF0D0
:106C200000094C4601E0002CEBD1BD42E9D225F031
:106C30000306002CF7D101A93046164B98470446AD
:106C40000028F0D1019B8DF80030C3F307228DF8A6
:106C50000120C3F307428DF802201B0E8DF803308C
:106C6000E9B2F3B2C91AC9B2C1F10403BE1B9E4214
:106C700028BF1E46042E28BF0426F6B232466944B9
:106C800008EB0900044B984735444E445FFA86F9F7
:106C9000C9E700BF696B4000D120410028B101283D
:106CA00001D000207047094800E0094800B583B0D2
:106CB00001A9084B984728B9019B13F4006F02D033
:106CC000012000E0002003B05DF804FB4000350027
:106CD00040003100696B400010B52DED028B82B091
:106CE000044601A93548364B98470346F8B14BB3E3
:106CF000002B32D0002B3BD0DFED328A002B49D065
:106D00009FED308A73B9DDED017AB8EE677AC8EE8F
:106D1000077A9FED2D7A67EE877AFCEEE77A17EE19
:106D2000902A6281184602B0BDEC028B10BD02A908
:106D300051F8043D23801B0C63802448204B984766
:106D40000346D4E702A951F8043DA3801B0CE3805D
:106D50001F481B4B98470346CAE702A951F8043D58
:106D600003F01F0323721B48154B98470346C1E7E6
:106D700002A951F8043DC3F3094308EE903AF8EE36
:106D8000688A9FED158A68EE888A14480C4B9847EC
:106D90000346B3E702A951F8043DDBB208EE103A0E
:106DA000B8EE488A28EE888ADFED077A28EE278A2F
:106DB0000B48034B98470346A4E700BF3008220066
:106DC000696B4000000000000000C8423808220043
:106DD000540822000800200000401C46040822003D
:106DE0001408220030B583B005460C4601A94FF4C3
:106DF000C450064B9847024620B9019B2B70C3F341
:106E000005232370104603B030BD00BF696B4000FE
:106E100000B583B001A941F23070094B9847034691
:106E200018B1184603B05DF804FB019921F0060182
:106E3000019141F23070034B98470346F1E700BFE0
:106E4000696B4000A56B400000B583B001A90A48FA
:106E50000A4B9847034618B1184603B05DF804FB87
:106E6000019921F0FF0141F0010101910248044B19
:106E700098470346F0E700BF10180007696B400011
:106E8000A56B400030B583B015460C4AA2FB012328
:106E90001B090F330093002302461120084CA04722
:106EA000044610B1204603B030BD29460548064BC4
:106EB00098470128F6D00524F4E700BF1F85EB5161
:106EC000F5694000200120004169400010B582B002
:106ED00096230093134602462020024CA04702B09E
:106EE00010BD00BFF5694000072801D90120704797
:106EF00010B584B08DF80C0030238DF80D3041F2C0
:106F00008833009303AB002202211420014CA047D8
:106F100004B010BDF569400010F0800F11D110B51C
:106F200084B08DF80C0010238DF80D3041F28833B9
:106F3000009303AB002202211420034CA04704B0AD
:106F400010BD0120704700BFF5694000F0B583B067
:106F5000032832D8DFE800F00209050747F6F0768B
:106F600004E0184E02E0184E00E0184E00240127FD
:106F70003D4604E09CB10F2C11D00134E4B20F2C3B
:106F800013D801AA0121A019114B9847B8B9002DB7
:106F9000F0D09DF80430FF2BECD00025EAE79DF8F7
:106FA0000430002BE9D10027E7E717B11DB100201D
:106FB00006E0002004E0012002E0002000E00020C4
:106FC00003B0F0BDF0FF0100F0FF0300F07F02000E
:106FD000856E400070B582B006460020114B984780
:106FE00020B14FF4BE65002423460BE001200D4B79
:106FF000984718B90323184602B070BD0A4DF2E74E
:107000000134E4B20E2CF6D8002BF9D101AA0121EB
:107010002819064B984703460028F1D19DF8042013
:107020003255EDE74D6F4000F0050200856E4000DF
:1070300030B587B01D201C4B98471C4C236C23F4A3
:107040000013236468461A4B984769462046194B3B
:107050009847636823F47F436360636843F47F4326
:107060006360042323610823236101232361626891
:1070700022F08F026260104A032120460F4DA8477C
:10708000002120460E4B9847636813F0800F01D112
:10709000082222600B4B4FF000521A60702283F8D6
:1070A0001D2307B030BD00BF2DE34000008003402A
:1070B00095494000294A4000E9704000794A400063
:1070C000BD49400000E100E00222014B1A60704718
:1070D00000800340024B1880024B1980704700BFAC
:1070E000020100200401002010B5064C206D80B282
:1070F000054B9847A06DE16D89B280B2034B98476C
:1071000010BD00BF0080034049824000D5704000A0
:10711000014B1888704700BF02010020014B1888FE
:10712000704700BF040100200D4B1B8840F68962A8
:10713000934205D90B4A12883E2A01D80320704792
:10714000084A128840F689618A4203D93E2B01D849
:1071500004207047934201D80220704701207047F5
:10716000020100200401002008B50120034B9847CC
:10717000034B186000B1012008BD00BFEDEE4000D8
:107180005014002008B54FF0FF31024B1868024B35
:10719000984708BD50140020A9F0400010B5002306
:1071A0001A46194602480068024CA04710BD00BFAD
:1071B00050140020B5ED4000154B98421BD003F54C
:1071C000A033984219D003F58043984217D0A3F515
:1071D0004043984215D003F58043984213D0A3F55D
:1071E000A033984211D003F56033984201D0322089
:1071F00070471620704708207047092070470E20FE
:10720000704713207047142070471520704700BF47
:1072100000C000404900B0FBF1F00338002302E059
:1072200040080133DBB2FF28FAD8020202F47F42A1
:1072300052FA80F01B0403F4E02318447047000066
:107240002DE9F843D0F80090037ADBB2012B00F06F
:10725000E68009F5C0650B7913B91846BDE8F883D7
:1072600017460E460446012303720023C371E160F2
:107270006E4B98478046B378022B08D07378012B69
:1072800018D033781B0403F4FE036B6050E073786E
:10729000012B09D033781B0403F4FE0303F580733C
:1072A0006B60F378EB6043E033785B081B0403F515
:1072B0008073F5E733785B081B04E6E70323A371CB
:1072C00000232372237A002B00F0AB802B6A13F487
:1072D000807F53D113F4007F78D113F0400F7AD11F
:1072E00013F0800F7CD113F0040F4BD13946404688
:1072F0004F4B98470028E9D00723A371002323723E
:107300004C4BC9F800363DE00423A37100232372DF
:10731000D8E70523A37100232372D3E70623A371C3
:1073200000232372CEE739464046414B9847E8B9DF
:107330003379E2799B1A002BC4DD2B6A13F4807F2A
:10734000BCD113F4007FDFD113F0400FE1D113F073
:10735000800FE3D113F0040FE5D0B168E379DBB21D
:107360005A1CD2B2E271CB5C6B63DCE70723A371DA
:10737000002323722F4BC9F80036A3E70323A37120
:1073800000232372237A002B4DD00223C9F8003644
:107390002B6A13F0010F28D113F4807F2BD113F443
:1073A000007F2DD113F0400F2FD113F0800F31D17A
:1073B000394640461E4B98470028E9D00723A37161
:1073C000002323721B4AC9F8002646E70423A37151
:1073D00000232372D6E70523A37100232372D1E78C
:1073E0000623A37100232372CCE700232372022318
:1073F000A371012331E70323A371002323722CE738
:107400000423A3710023237227E70523A37100231C
:10741000237222E70623A371002323721DE70023B2
:107420001BE7002319E7002317E700BFA57D4000F5
:10743000BD7D4000028000052DE9F84FD0F800B076
:10744000037ADBB2012B00F0CE800BF5C0670B791D
:1074500013B91846BDE8F88F90460E46054601233D
:1074600003720023C371E960614B98478146B3788A
:10747000032B14D07378012B24D033781B0403F42E
:10748000FE0303F580537B6096F804A0BAF1010F68
:107490001ED00123CBF800364FF0000A64E0737869
:1074A000012B09D033781B0403F4FE0303F5885342
:1074B0007B60F378FB60E7E733785B081B0403F538
:1074C0008853F5E733785B081B0403F58053DAE74C
:1074D0000323CBF8003647E00323AB7100232B7264
:1074E0002B7A002B00F081803B6A13F0010F60D1F2
:1074F00013F4807F63D113F4007F65D113F0400F44
:1075000067D113F0800F69D141464846394B9847FF
:107510000028E9D00723AB7100232B72364ACBF841
:10752000002696E70423AB7100232B72D8E70523CE
:10753000AB7100232B72D3E70623AB7100232B72B0
:10754000CEE70723AB7100232B722B4BCBF8003611
:10755000C6E714F0020F07D0B168EB79DBB25A1C12
:10756000D2B2EA713A6BCA54EB79DBB23279934208
:10757000B6D23C6A14F4807FAED114F4007FD1D12E
:1075800014F0400FD3D114F0800FD5D141464846B6
:10759000184B98470028D4D1BAF1000FD9D13379CC
:1075A000EA799B1A012BD4D102233B604FF0010AE8
:1075B000CFE700232B720223AB71012349E703239A
:1075C000AB7100232B7244E70423AB7100232B72B1
:1075D0003FE70523AB7100232B723AE70623AB711B
:1075E00000232B7235E7002333E7002331E700BF88
:1075F000A57D4000BD7D4000028000052DE9F041E1
:1076000006468846046820461B4B9847312801D916
:10761000BDE8F0810546194B9847032323602423D6
:10762000C4F8003641461648164B9847C4F8100671
:10763000002333720123B3716BB2002B07DB5A09AD
:1076400005F01F00012181400F4840F82210002B57
:107650000BDB03F1604303F56143202283F8002331
:1076600001200A4B98473061D2E705F00F05084B1F
:1076700020225A55F4E700BFB97140002DE34000C5
:107680000000DC051572400000E100E0EDEE400076
:1076900014ED00E008B500680B4B9847312811D86D
:1076A00043B2002B0CDB5B0900F01F0101228A4072
:1076B0002033064941F82320BFF34F8FBFF36F8F6C
:1076C000034B984708BD00BFB971400000E100E0DE
:1076D00081E3400008B54FF0FF310069014B984746
:1076E000C0B208BDA9F0400010B500231A461946E3
:1076F0000069024CA047C0B210BD00BFB5ED40000C
:1077000008B5837963B18B78032B0BD8DFE803F0DE
:1077100002050205044B984708BD044B984708BD75
:10772000002008BD002008BD4172400039744000AF
:1077300080797047F8B50646036803F5C064256A8A
:10774000C76815F0040F0BD0E26A12F0040F07D0DF
:10775000BA78002A4DD0022A4BD0BA78032A5ED0DC
:1077600015F0020F08D0E26A12F0020F04D0BA78C6
:10777000012A73D0032A71D015F4807F0DD0E36AFB
:1077800013F4807F09D040F20733A36200233372E1
:107790000323B371FB6803B1984715F4007F0DD044
:1077A000E36A13F4007F09D040F20733A362002399
:1077B00033720423B371FB6803B1984715F0010FCE
:1077C00016D0E36A13F0010F12D0BB780BB1022B75
:1077D00009D140F20533A362002333720223B3714F
:1077E000FB6803B19847BB78012B54D0032B52D0D0
:1077F000F8BDF279D2B239798A4208D2B868F27902
:10780000D2B2511CC9B2F171825C6263A5E7022257
:10781000C3F80026012262620422A2629DE77A7800
:10782000012A11D03A78120402F4FE0202F58052C5
:1078300062603A79012A0DD00122C3F800260422A1
:10784000A262022262628BE73A785208120402F5C1
:107850008052EDE70322C3F80026F0E7B868F2791A
:10786000D2B2511CC9B2F171216B8154F179C9B204
:107870003A79013A91420AD0F379DBB23A799342EC
:107880007FF47AAF012363620223A36274E70222CA
:10789000C3F80026F0E740F20333A36200233372FB
:1078A0000223B371FB68002BA2D09847A0E7000029
:1078B00070B4056805F5C0660379202B0BD9A3F1D8
:1078C0002001CBB21A4C0121994021602165216130
:1078D0002163002211E0174CF5E701339BB2B3F5A9
:1078E0002F7FFAD36163002301E001339BB2B3F52C
:1078F0002F7FFAD321630132D2B2092A01D80023A3
:10790000EDE76161616032698023C5F800360023CC
:1079100001E001339BB2B3F52F7FFAD33261242308
:10792000C5F80036002303720123837170BC7047D1
:1079300000100E40000E0E4030B591B000238DF8BF
:1079400035308DF836308DF837308DF839308DF888
:107950003A30ADF83E300F238DF834300223ADF8C5
:107960003C3001248DF838400DAA0B4907A80B4D77
:10797000A8470DAA0A4901A8A8471023079A13602F
:10798000019A1360074B1C70074B1C7045F6FF7281
:10799000064B1A8011B030BD00C0024015DE400019
:1079A000000003401C0D002034160020FE160020AD
:1079B00042B110B420B119B1034B586099605A809C
:1079C0005DF8044B704700BF1C0D0020154B1B7861
:1079D0003BB3144B5B8823B3124A52680AB3114974
:1079E0008968F1B1F0B583B0009201930E4D6A46FB
:1079F000694628460D4FB8474FF480362E62094B32
:107A00009B6800930A4C6A4669462046B84726623E
:107A100001212846074DA84701212046A84703B069
:107A2000F0BD70471C0D002000C1024051DD400038
:107A30000001034069DD40000223034A136202F59E
:107A400080421362704700BF00C1024010B58CB085
:107A50000A4B9847069A136823F010031360009AA4
:107A6000136823F0100313600D20054CA04712206B
:107A7000A0470022034B1A700CB010BD397A4000A9
:107A800081E340001C0D0020064B1B783BB1054BE9
:107A90005888054BD3F80431C01A80B270470020D3
:107AA000704700BF1C0D002000C00240094AD36D82
:107AB00023F4FF4323F07F03C0F30E000343D36599
:107AC00002F58042D36D23F4FF4323F07F03184374
:107AD000D065704700C00240014B1880704700BF5E
:107AE000FE160020014B1870704700BF34160020AE
:107AF00000487047001700200048704754140020C9
:107B0000704770472DE9F8434F4B984705464F4B58
:107B1000984704467FE0A0EB070E1FFA8EFE0EF199
:107B2000F00E1FFA8EFE85E03121002308E02F21A0
:107B3000FBE747480078C0B2012831D001339BB23F
:107B4000994259D9DA1992B2EF2A01D9F03A92B290
:107B50003F4800780028ECD13E48B0F9000035F9E4
:107B6000126006FB00F6F6134FEA8308DFF8ECC05C
:107B70000CF8236008F10109C6F307260CF8096028
:107B800034F9122000FB02F2D21308F102000CF8C3
:107B9000002008F10308C2F307220CF80820CDE703
:107BA00035F9120034F91220024402EBD27252105D
:107BB00012F5004F05DBB2F5004F03DB47F6FF720D
:107BC00000E0254A2348B0F9000012B202FB00F29F
:107BD000D21398005FFA82FC204E06F823C000F111
:107BE0000108C2F3072206F8082000F1020806F88F
:107BF00008C003303254A1E7194BA3F800E00F444A
:107C0000BFB2184B1F80EF2F01D9F03F1F808900B2
:107C10001248154B98474FF0FF310120134B9847FE
:107C2000134B98470F4B1F88B842FFF474AFC01B2B
:107C30001FFA80FEBEF1300F3FF676AFBEF12F0F78
:107C40007FF675AF302170E7F17A4000F97A400095
:107C500034160020FE1600200080FFFF381600209A
:107C6000FC160020280D00202D45400081FD40001D
:107C7000897A4000F8B5084C4FF4804666630A20C4
:107C8000064DA847402767630A20A84727630A20B4
:107C9000A8472663F8BD00BF000E0E4075F84000EF
:107CA00038B5D0B14FF48072144B5A63144B9847D7
:107CB00001280ED00220134CA0470122124B1A6358
:107CC0000420A0474FF080720C4B1A630220A0479B
:107CD00038BD02220C4B1A63ECE7084D4FF4807359
:107CE0006B630220074CA0474FF080736B63042046
:107CF000A0470122044B5A6338BD00BF000E0E405E
:107D0000510C410075F8400000100E4038B50D4D83
:107D10004FF480736B6302200B4CA0474FF08073CD
:107D20006B630420A0470122084B5A630220A0473E
:107D3000074B9847012800D038BD0222034B5A63F5
:107D4000FAE700BF000E0E4075F8400000100E402C
:107D5000510C410008B54FF480420A4B5A63002091
:107D6000094B98470220094B9847094B984701282F
:107D700003D04022034B5A6308BD0222054B5A63CD
:107D8000F7E700BF000E0E40A17C400075F84000F0
:107D9000510C410000100E400322014B1A60704745
:107DA00030140E40044B986801E0034B9868024B76
:107DB0009B689842F9D1704730140E4010B584B0DA
:107DC00001900C46064B98470390039B019A9B1A1F
:107DD000A34202D2002004B010BD0120FBE700BF87
:107DE000A57D400030B585B01E4B1B68002B31D0FF
:107DF0001D4B98474FF0FF311A4B18681B4B9847A3
:107E0000EFF31083B3FA83F35B09039372B6BFF306
:107E10005F8F0022164B1A70039D80230093154B31
:107E2000152214211448154CA04704462DB10122F7
:107E30000F4B1A70BFF35F8F62B600231A461946C4
:107E4000084800680E4DA8470E4B984744B10020E3
:107E500005B030BD01200C4B9847024B1860C7E7B6
:107E60000120F5E72C0D002085714000A9F04000AD
:107E70002F030020E0180020000A0E40110000200F
:107E8000B5ED40009D714000EDEE400010B5074B90
:107E90009847002213210648064B98470446064B94
:107EA0009847B4FA84F0400910BD00BF85714000C6
:107EB000000A0E408DE040009D71400038B5114B26
:107EC0009847EFF3108404B972B6002308E09A00D3
:107ED00002F580020C4951F82310116001339BB266
:107EE0007F2BF4D9002212210848094B9847C5B2CC
:107EF00004B962B6074B98470DB1002038BD012088
:107F000038BD00BF85714000E0180020000A0E4017
:107F10008DE040009D71400010B400240EE0400050
:107F200080F00700C0B20133DBB2072B05D810F098
:107F3000800FF4D14000C0B2F5E70134944204D27E
:107F400011F8013B58400023EFE75DF8044B704700
:107F500070B50646002501E02C44A5B2B5F5007FBA
:107F600015D20E4BE918EA5CFF2A14D06B1C0B48A3
:107F70001B5C0333DCB2B242EED1621EFF20084B21
:107F800098472B19074A9B5C9842E5D101E04FF6D0
:107F9000FF75284670BD4FF6FF75FAE7E018002020
:107FA000197F4000DF18002008B5094B1B781BB172
:107FB000022B01D0074808BD074B9847012804D180
:107FC0000122034B1A70034808BD002008BD00BF02
:107FD000300D0020E0180020E57D400008B5094B79
:107FE0001B781BB1022B01D0074808BD074B9847EF
:107FF000012804D10122034B1A70034808BD002058
:1080000008BD00BF300D0020E0180020E57D4000D5
:10801000A8B108B50346B1F5007F12D28818B0F5B3
:10802000007F01D9002008BD08461946064B1844B8
:10803000064B98470222064B1A70012008BD00200B
:108040007047002008BD00BFE0180020D12041008B
:10805000300D002008B5064B1B78022B01D0002004
:1080600008BD044B98470128FAD1034B984708BD37
:10807000300D00208D7E4000BD7E400090B110B5D7
:1080800004460268094B9A4201D0002010BD9A2292
:108090000146FF20064B984794F89A30984203D047
:1080A000002010BD00207047012010BD5FE1AD5AD7
:1080B000197F400010B50C46084B9847B0F5007F7B
:1080C00001D3002010BD811C054B5A1C125C1944C1
:1080D0002046044B9847012010BD00BF517F40004F
:1080E000E0180020D120410008B5044B9847B0F5B6
:1080F000007F01D2012008BD002008BD517F400053
:1081000008B5054B9847B0F5007F02D2034BC05C21
:1081100008BD002008BD00BF517F4000E1180020CD
:10812000FF292FD02DE9F843D61CF6B28419B4F5F7
:10813000007F03D94FF6FF70BDE8F88317460C4661
:1081400005460221114A1170DFF84C8000EB080946
:1081500000F80840421C02F8087008443A461946E4
:1081600040440B4B98477C190234721E4946FF204D
:10817000084B984708F80400E81980B2033080B231
:10818000BDE8F8834FF6FF70704700BF300D002048
:10819000D1204100197F4000E018002010B5A8B0A0
:1081A000224B98470446224B984708B928B010BD87
:1081B0009B22214601A81F4B98474FF40072FF21D4
:1081C0001D481E4B984702AB1022012100201C4C79
:1081D000A0474FF6FF73984203D026AB032202213B
:1081E000A0474FF6FF73984205D00DF19B03012283
:1081F0000321134CA0474FF6FF73984204D027ABDE
:10820000012204210E4CA0474FF6FF73984205D07F
:108210000DF19D0301220521094CA0474FF6FF7384
:108220009842C3D0074B9847C0E700BFA97F4000E2
:108230007D804000D1204100E0180020CD22410087
:108240002181400055804000044B1880044A137877
:10825000591C1170034A22F813007047E41C0020D7
:10826000310D0020E41A002008B5194B1B8807EED9
:10827000903AF8EE677A9FED177A67EE877A164B99
:10828000C3ED007AF7EE006A76EEE76A87EEA67A2B
:10829000DFED126A67EE267A114BC3ED007A86EEA7
:1082A000A77A17EE100A0F4B9847DFED0F7A07EE0B
:1082B000100A27EE277ADFED0D7A77EEC77ADFED29
:1082C0000C6A86EEA77A0B4B83ED007A08BD00BFDF
:1082D000E41C002001088039E01A002000401C4600
:1082E000EC1C0020690C41003313954300F0574506
:1082F000C47D7B49E81C0020BFF35F8F024B1868E8
:10830000BFF35F8F704700BFE81C002068B90F4AB9
:108310001368B3F1FF3F0AD00320B3F1333F0ED00F
:1083200013B9536803B902207047094AF0E751684E
:10833000B1F1FF3F01D00320EFE70020EDE75168E6
:10834000B1F1333FECD10120EAE700BF00C04700A4
:1083500000E0470018B101280FD0022070470B48F9
:1083600041F6F87383B130B4C518C4588C4206D0B6
:10837000083B002BF8D1012004E00548F0E76B68CA
:108380001360002030BC70470120704700C04700D8
:1083900000E0470070B505460020124CA047064695
:1083A0000120A0471DB1012D12D0022070BD02286E
:1083B00003D0022E07D0022070BD012E01D0012073
:1083C00070BD002070BD012801D0002070BD70BDBF
:1083D000022E05D0022801D0022070BD012070BD00
:1083E000002070BD0D834000F8B504460F461646C8
:1083F000450A094B984704F4FE7000F580031F609E
:108400005E602A4601210548054B98470446054B06
:1084100098472046F8BD00BF85714000000A0E4015
:108420008DE040009D714000012909D002290CD146
:10843000002108B538B906480A46064B984708BDDA
:108440004FF03331F5E70448F6E70120704700BFED
:1084500000C04700E983400000E0470038B518B18C
:1084600001280DD0022038BD0A4C0823B3F5005F67
:108470000ED2E018E558B5F1FF3F03D00833F5E719
:10848000054CF2E7054B984708B1022038BD38BDCE
:10849000012038BD00C0470000E04700E9834000EC
:1084A00010B568B140F2F234074B984722460721D5
:1084B0000648074B98470446064B9847204610BD90
:1084C00040F2E234F0E700BF85714000000A0E4040
:1084D0008DE040009D71400070B582B00023019393
:1084E000044668B90125184E18490023B3F5006FFA
:1084F00028D251F82320B2F1FF3F05D10133F5E72F
:108500000025134E1349F0E72046134B98470446C5
:1085100010B1204602B070BD01AA314628460F4B6B
:10852000984748B9019A0132314628460C4B984782
:108530000028EED00124ECE7012231462846084B02
:108540009847F5E70024E4E70120FFFF00C047005B
:108550000220FFFF00E04700A18440005583400057
:108560005D84400070B582B005460E460846294B32
:108570009847012806D001213046274B98470446EA
:10858000002844D1002400E00134244B1B689C42A5
:1085900015D201AA224B53F824102846214B9847A4
:1085A000022833D00028EFD1019A1D4B53F8241034
:1085B00030461D4B98470028E6D0012427E0284686
:1085C0001A4B9847044610BB02213046124B98477D
:1085D0000446E0B995B9164D02AA002342F8083DB9
:1085E000294630460F4B984750B9009A0132294628
:1085F00030460D4B984750B1012408E00D4DEBE794
:10860000012229463046084B9847F4E701242046CA
:1086100002B070BD0D83400029844000200100207D
:1086200008010020558340005D844000A184400083
:108630000120FFFF0220FFFF10B50020104B9847DC
:10864000044608B1204610BD01200D4B9847044652
:108650000028F7D102210B4B984704460028F1D19E
:1086600001220949094B984708B10124EAE7012290
:108670000749064B98470028E4D00124E2E700BFF1
:10868000A1844000298440000120FFFF5D84400058
:108690000220FFFF38B50120384B9847384B18604F
:1086A000002869D00020374DA84704460120A8477C
:1086B000012C2BD05CB1022C46D0334B984703469B
:1086C00018B90122314B1A700023184638BD012811
:1086D00008D0022814D100202D4B984703460028CB
:1086E000EFD0F2E700202A4B984703460028ECD150
:1086F00002210120274B984703460028E1D0E4E7F8
:10870000214B984703460028DBD0DEE748B102281A
:1087100014D100210120204B984703460028D0D0D7
:10872000D3E701201A4B984703460028CDD10221F8
:10873000184B984703460028C3D0C6E7124B98470A
:1087400003460028BDD0C0E738B102280CD10E4B3B
:10875000984703460028B4D0B7E701200C4B984750
:1087600003460028ADD0B0E7012100200A4B98470E
:1087700003460028A5D0A8E70123A6E7EDEE4000B8
:10878000F01C00200D83400039864000320D00208F
:10879000D9844000298440006585400070B50E4BA7
:1087A0001B7813B90324204670BD0D4604460B4EBA
:1087B0004FF0FF3130680A4B98470120094B98472A
:1087C0002A462146084B9847044600231A46194674
:1087D0003068064DA847E6E7320D0020F01C002067
:1087E000A9F040009583400055834000B5ED40005E
:1087F000F8B5194B1B7813B903242046F8BD0E4673
:1088000005464FF0FF31154B1868154B984700206F
:10881000144B9847074632462946134B984704465F
:10882000012807D000231A4619460C4800680F4D4E
:10883000A847E2E7B7FA87F46409214638460C4BAB
:10884000984708B10224EDE7324629462046064BF8
:1088500098470446E6E700BF320D0020F01C0020D8
:10886000A9F04000958340005D844000B5ED4000D4
:108870006585400008B50020094B984708B10120E4
:1088800008BD2022074B5A630A20074B9847074B25
:108890009847074B9847012801D0002008BD08BD24
:1088A0001968400000100E4075F84000CD0B4100E3
:1088B0006967400030B587B0174B984704468A2354
:1088C0008DF808300025059501238DF809308DF8C5
:1088D0000C300DF107030493104B98478DF80B50A3
:1088E00003238DF80A30322202A920460C4B984708
:1088F00020460C4B9847022806D0002520460A4BFC
:108900009847284607B030BD9DF80730092B01D0A5
:108910000025F3E70125F1E7CD0B4100D5764000B6
:108920000177400031774000E976400030B587B0EC
:108930001A4B9847044600220592A8238DF8083068
:1089400001238DF809308DF80B2001AA0492022230
:108950008DF80C208DF80A30114B9847322202A96D
:108960002046104B984720460F4B9847022806D0C8
:10897000002520460D4B9847284607B030BD9DF88E
:10898000043033B99DF8053013F0F80F03D00025FB
:10899000EFE70025EDE70125EBE700BFC50B410040
:1089A000D57640000177400031774000E9764000FD
:1089B00008B5034B984708B1002008BD012008BD49
:1089C000D96B400030B587B0184B98470446002358
:1089D000059372238DF8083001238DF80930922217
:1089E0008DF80B200DF1070204928DF80C30032353
:1089F0008DF80A300E4B9847322202A920460D4BC3
:108A0000984720460C4B9847022806D00025204660
:108A10000A4B9847284607B030BD9DF80730442BD5
:108A200001D00025F3E70125F1E700BFCD0B4100A0
:108A3000D57640000177400031774000E97640006C
:108A400070B586B0002832D11C4B984704460025EB
:108A5000059598238DF8083001268DF809608DF86A
:108A60000A5002238DF80C3001AB04938DF80B50A3
:108A70002046134B984736238DF804308DF8055067
:108A8000322202A920460F4DA8478DF80A603222F3
:108A900002A92046A84720460B4B984702280AD037
:108AA00000252046094B9847284606B070BD084B64
:108AB00098470446CBE73546F3E700BFC50B4100B6
:108AC000D57640000177400031774000E9764000DC
:108AD000CD0B410038B50020064CA04705460120CB
:108AE000A047012D01D0002038BD0128FCD0002076
:108AF00038BD00BF418A40002DE9F0473D4BD3F817
:108B0000588019203C4B98474FF496703B4B984740
:108B1000002409E03A4B98473A4B23F8140003200D
:108B2000364B98470134E4B21F2CF3D9364B9847A3
:108B3000824600263746354634463FE0314931F813
:108B400013100A440133DBB21F2BF7D94FEA521935
:108B5000B9F10A0F17D92A4B9847631CDBB2294A8F
:108B600022F814001F2B1DD81C46A9F1FA039842C5
:108B70001AD309F1FA02904225D80135EDB2202D21
:108B800013D9012611E0B8F1000F05D0194BC3F835
:108B900058800020BDE8F0870020174B9847002040
:108BA000BDE8F0870024E0E700250320134B984739
:108BB0004FF47A615046154B984707462FB926B9AE
:108BC00000231A46C0E70025EFE7B8F1000F07D0F1
:108BD000084BC3F8588057B936B10120BDE8F0877B
:108BE0000020054B9847F6E70020BDE8F0870020FD
:108BF000BDE8F087000001400154400075F84000D6
:108C00004D544000F41C0020A57D4000BD7D400077
:108C100000487047584E4100062070472DE9F84340
:108C200005460E4617460A469C211E4B98470446A9
:108C3000451B40B1731B052B05D94378552B07D035
:108C400010237B7001E000237B702046BDE8F88391
:108C500090F80280C37888EA0303FF2B02D0112327
:108C60007B70F2E790F80490437909EB03291FFA2F
:108C700089F9B9F13A0F06D84D440635AE4205D20E
:108C800000237B70E1E712237B70DEE74A46811DFB
:108C9000381D054B9847A7F8029087F800800123FC
:108CA0007B70D2E7D11F4100D120410010B553881D
:108CB0009C1D8C4219D83A2B01D9002010BD1146B9
:108CC0009C23037055234370137883701378DB4320
:108CD000C3709378037153881B0A4371528804311F
:108CE0000630034B9847012010BD002010BD00BF87
:108CF000D120410070B582B004460378253B332B68
:108D000000F21982DFE813F045001702170217027C
:108D10001702340017021702170217021702170270
:108D2000170217021702170217021702170217027B
:108D3000170217021702170217021702170217026B
:108D40003E0117021702FA00170217021702170254
:108D50001702BA0113015C0017021702170217026B
:108D600017021702170265017900CB00A600E30085
:108D70009C4C2A2323709C4DA84760809B4B9847AE
:108D80000646A84702463146201D994B984702B037
:108D900070BD0120974B984780B2924B588010B914
:108DA00045221A70F3E794490120944B984718B173
:108DB00025228C4B1A70EAE745228A4B1A70E6E7A7
:108DC0004388032B05D0874B00225A8045221A7016
:108DD000DDE703798DF8043043798DF80530837928
:108DE0008DF80630864B984701A9864B98477D4BF6
:108DF00000225A8024221A70C9E74388012B05D02B
:108E0000784B00225A8045221A70C0E703790F2B55
:108E100005D9744B00225A8045221A70B7E77A4B65
:108E20009847704A5523137020235380237900EB11
:108E30004310066845688468C16856609560D460D0
:108E40001161066945698469C16956619561D4619A
:108E500011629CE74388212B05D0624B00225A8087
:108E600045221A7093E701790F2905D95D4B00223D
:108E70005A8045221A708AE7202249010530634B47
:108E80009847012805D0574B00225A8045221A7076
:108E90007DE7544B00225A8024221A7077E74388DA
:108EA0002BB1504B00225A8045221A706FE7584B65
:108EB0009847012805D04B4B00225A8045221A7052
:108EC00065E7484B00225A8024221A705FE74388E6
:108ED0002BB1444B00225A8045221A7057E74D4B64
:108EE000984728B93F4B00225A8024221A704EE737
:108EF0003C4B00225A8045221A7048E74388012BD8
:108F000005D0384B00225A8045221A703FE700797D
:108F1000414B984728B9334B00225A8024221A70BB
:108F200035E7304B00225A8045221A702FE74388DC
:108F3000082B05D02B4B00225A8045221A7026E7B9
:108F40000379427903EB0223827903EB0243C07970
:108F5000217A627A01EB0221A27A01EB0241E47AE2
:108F600001AA01EB046103EB00602C4B9847002839
:108F70007FF40DAF1B4B019A5A604B221A700422EA
:108F80005A8004E74388063B9BB21F2B05D9154B3B
:108F900000225A8045221A70F9E64379807903EB62
:108FA0000023E07903EB0043207A04F109022179E0
:108FB00003EB00601A4B984728B90A4B00225A80ED
:108FC00024221A70E3E6074B00225A8045221A70C9
:108FD000DDE6438833B3034B00225A8045221A70E2
:108FE000D5E600BF341D0020198C4000118C4000D4
:108FF000D120410001814000381D0020B580400093
:10900000CD0B4100C1634000DD7F40001180400076
:1090100055804000D96B4000E96E4000856E4000ED
:10902000CD6E40000020474B1871474B984720B148
:10903000444A137943F0010313710120424B9847CE
:1090400020B1404A137943F00203137102203E4BD2
:10905000984720B13B4A137943F00403137103206E
:10906000394B984720B1374A137943F008031371FD
:10907000344B01225A8054221A7088E64388012B0F
:1090800005D0304B00225A8045221A707FE60379C2
:10909000463B102B49D8DFE803F03F4809484848D1
:1090A000124848362D48481B48482400274B98470B
:1090B000244B18714A221A7001225A8067E6244B09
:1090C0009847204B18714A221A7001225A805EE696
:1090D000204B98471B4B18714A221A7001225A8064
:1090E00055E61D4B9847174B18714A221A700122FA
:1090F0005A804CE6194B9847124B18714A221A7045
:1091000001225A8043E6164B98470E4B18714A22AB
:109110001A7001225A803AE6124B9847094B18718F
:109120004A221A7001225A8031E6064B45221A70F3
:1091300000225A802BE6034B00225A8045221A70E7
:1091400025E600BF341D00204D6F400075884000AB
:10915000B58840002D894000B1894000C589400094
:10916000D58A4000F98A400000487047341D00202D
:10917000F0B583B0EFF31083B3FA83F35B09019387
:1091800072B6BFF35F8F0022364B1A70019E364BCA
:109190001B68364A15682B447F2B2AD8324B1C6833
:1091A0002246334933482844334B98472C442F4BAD
:1091B0001C6000222C4B1A602EB10122294B1A7020
:1091C000BFF35F8F62B62D4A284B196829482C4B94
:1091D00098470146D0B1274BC31A284842881A4401
:1091E000951D4478012C15D044BB802B1CD900243C
:1091F0002AE01D4A136814682C441B1B03F18004E9
:10920000204A137843F001031370C9E70024174B79
:109210001C6019E01748154F3E68761B324641190D
:10922000194B98473E600FE0104D2C68E41A224617
:109230001048154B98472C60002405E00133802B23
:1092400005D90024094B1C60204603B0F0BD094835
:10925000064D2C68E41A2246C1180B4B98472C6027
:109260000024F1E72F0300207C2000208C20002028
:10927000D42000207C1F0020D1204100902000201D
:109280001D8C4000882000200522410010B50DE013
:10929000144B195D1448154B98470134E4B2144B34
:1092A0001B689C42F4D30022114B1A600120114B21
:1092B0009847114B98470128F8D11048104B984710
:1092C000104B98470246802106480F4B98470128CB
:1092D000ECD10C4B984743880633054A13600024B1
:1092E000DDE700BFFC1F00200082014017E54000C1
:1092F0008420002075F840007191400090200020EB
:10930000F58C400069914000AD8C400030B583B0D1
:109310008024224600211C481C4DA84722460021DB
:109320001B48A84700231B4A13601B4A13601B4AB3
:1093300013701B4A10215166C2F89010516551629A
:10934000C2F88010116F21F010011167516F21F0E8
:1093500010015167134A4FF400211160202182F857
:1093600013130121104A9160104A01920093224682
:109370000F491048104CA047012802D00F48104B4D
:10938000984703B030BD00BFD4200020CD2241005B
:10939000FC1F00207C20002084200020882000204A
:1093A000000E0E4000E100E000820140802000201D
:1093B000604E41008D924000A1F54000684E410092
:1093C000291A4100104B1B6913F0010F12D00E4BEC
:1093D0005B6913F0010F0DD00C4B1B687F2B0AD972
:1093E0000B4A137843F001031370074B9A69094B3A
:1093F00083F87F207047054A1368591C1160024AA0
:109400009169044AD1547047008201407C200020B9
:1094100088200020D4200020064A936823F07F4350
:1094200023F4706343F0254343F4E0639360024BFD
:109430001360704700140E40080000A570B5064682
:109440000D46094B98470446002040B9294620465E
:10945000064B984728B93046054B9847F5E7012059
:1094600070BD002070BD00BFA57D4000BD7D4000E7
:1094700021B7400010B54FF47A72314B1A8004E0E6
:10948000402200212F48304B98472D4B188880B23E
:109490002E4B98472B4C23232370182363702C4B9F
:1094A0009847C0F30F23A370E0702A4B9847C0F38E
:1094B0000F2323716071284B9847C0F30F23A371CA
:1094C000E071264B9847C0F30F2323726072244B40
:1094D0009847C4F80A00234B1B7807EE103AB8EE01
:1094E000477A9FED216A27EE067ADFED206A37EE94
:1094F000667A17EE103AC4F80E301D4B1B7807EE53
:10950000903AF8EE677A67EE867A77EEE67A17EEAB
:10951000903AC4F81230174B9847C0F30F23A37545
:10952000E075154B9847C0F30F2323766076134BF5
:1095300098470028A4D032212046114B98479FE736
:10954000C821002078210020CD22410075F840007C
:109550004D544000095C4000117140001D714000F5
:10956000F9824000F8010020B4C8363F6FDB4A4260
:10957000F9010020ADAD4000B9AD4000EF0B410056
:109580003D944000F0B583B0402200219C489D4BA3
:1095900098470AE29C4B98479C4B984710E29A4B9D
:1095A00098479B4BBB221A601A225A60974B9847E8
:1095B00009E293490B462A2203F8012B954A1068C9
:1095C000C1F8010092889A8000E20120924B9847EE
:1095D00028B98B4B45221A7002225A70F9E188494A
:1095E000252301F8013B01208C4B9847F1E108202D
:1095F000894B984728B9824B45221A7002225A702B
:10960000EAE17F49262301F8013B0820834B984774
:10961000E2E10920804B984728B9794B45221A701E
:1096200002225A70DBE176497E2301F8013B0920D2
:109630007A4B9847D3E1C4F30723032B09D8DFE81B
:1096400003F0020B0406764807E0764805E076480A
:1096500003E04FF0FF3000E07448B0F1FF3F10D05E
:1096600001A9734B984730B9654B5A221A70019A79
:10967000C3F80120B7E1624B45221A7002225A70EA
:10968000B1E15F4B45221A7001225A70ABE1C4F37D
:109690000723032B09D8DFE803F0020B0406604818
:1096A00007E0604805E0604803E04FF0FF3000E06D
:1096B0005E48B0F1FF3F0ED05E4B19685E4B984795
:1096C00018B924224E4B1A7090E14D4B45221A7066
:1096D00003225A708AE14A4B45221A7001225A70BD
:1096E00084E12422464B1A7083E1454B45221A70CF
:1096F000524A12785A707FE1514B1B780F2B05D9D3
:109700003F4B45221A7001225A7078E14D4B984721
:109710003B4A5523137020235370494B1B7800EBB1
:109720004310D0F800E047688668C168C2F802E0DC
:10973000C2F80670C2F80A60C2F80E10D0F810E045
:1097400047698669C169C2F812E0C2F81670C2F8AA
:109750001A60C2F81E1052E1294B4B221A700422E3
:109760005A706A44384B1968384B1868384B984718
:1097700020B9234B019AC3F8022043E10022354B64
:109780001A603FE11E4B54221A7000205870324B71
:10979000984720B11A4A537843F0010353700120CF
:1097A0002D4B984720B1164A537843F0020353706B
:1097B0000220294B984720B1114A537843F0040303
:1097C00053700320244B9847002800F01E810C4A58
:1097D000537843F00803537017E1204B187807289B
:1097E00007D9802843D0064B45221A7001225A70AF
:1097F0000EE11B4B9847A8BB2422014B1A7007E1CE
:10980000D0210020CD224100490B41001994400095
:1098100090140E40104B410001814000B580400083
:109820000110FFFF0310FFFF0410FFFF0210FFFFF6
:109830009D874000C4210020F1874000CA210020FC
:10984000C0210020DD7F4000CC210020BC21002071
:10985000856E4000D22100204D6F40005421002031
:10986000E96E4000784A452111705070D0E0774B86
:10987000187810F0800FB6D1754B984718B924228C
:10988000714B1A70C4E0704B452119705870BFE0DD
:10989000704A714B1968714B1868714B984718B929
:1098A0002422694B1A70B6E0674B45211970587035
:1098B000B1E065484E2300F8013B6A4B9847002809
:1098C00000F0AC80684B4FF020321A605A609A600A
:1098D000C3F80B20A2E014F47F4F5B4E31464FF0EB
:1098E0005E0301F8023B14BF012000205F4B984744
:1098F0007070002840F095804522327091E04A2235
:10990000514B1A70C4F30723463B102B2DD8DFE8C8
:1099100003F0272C092C2C2C0E2C2C221D2C2C1364
:109920002C2C1800524B9847474B58707CE0514BF9
:109930009847454B587077E04F4B9847424B5870CB
:1099400072E04E4B9847404B58706DE04C4B984737
:109950003D4B587068E04B4B98473B4B587063E069
:10996000494B9847384B58705EE0374B45221A7088
:1099700001225A7058E0454B98472422324B1A7006
:1099800054E09A000232424951F823002E495050C7
:109990000133DBB20B2BF4D93E4B984700284ED154
:1099A0004022002128483C4B98474FF0FF310120CE
:1099B0003A4B984704460028F7D043283FF4EAADD5
:1099C000422C3FF4ECAD2A2C3FF4F3AD252C3FF4B0
:1099D000FCAD262C3FF40BAE7E2C3FF41AAEE5B264
:1099E0005A2D3FF428AE7A2D3FF451AE242C3FF48B
:1099F00078AE452C3FF479AE552C3FF47DAE4B2C20
:109A00003FF4AAAE542C3FF4BDAE442C3FF4E5AE77
:109A1000412C3FF43DAF4E2C3FF44BAF5E2D3FF455
:109A20005AAF4A2D3FF46BAF3D2CA4D0732CB3D169
:109A3000054B73221A7030225A700023AAE7322194
:109A40000148174B9847ABE7D0210020B8210020F0
:109A5000196F400058210020CC210020BC2100209B
:109A6000CD6E4000D56F4000D12100204D594000FF
:109A700075884000B58840002D894000B1894000BC
:109A8000C5894000D58A4000F98A400091AD400068
:109A9000C8230020EF0B4100CD22410081FD400092
:109AA0003D94400010B5002303220146024800689F
:109AB000024CA04710BD00BF340D0020A9FE40009D
:109AC00010B584B0002304AA42F8043D09490C688B
:109AD0000092032201462046074CA047039B3BB15E
:109AE0004FF08052054B1A60BFF34F8FBFF36F8F5B
:109AF00004B010BD340D002055FF400004ED00E01F
:109B000010B582B00F4B01930123009300238022F4
:109B10000D490E480E4CA047012802D00D480E4BAF
:109B20009847002301930122009280220B490C48A0
:109B3000074CA047012802D00A48074B984702B0BB
:109B400010BD00BF340D0020884E410085954000B7
:109B5000A1F54000984E4100291A4100C84E41002D
:109B600075944000D44E410070B584B0044603782B
:109B70002A2B00F0A1802378252B00F0A1802378E8
:109B8000262B00F0A18023787E2B00F0A180237883
:109B90005A2B00F0A18023787A2B00F0A480237840
:109BA000532B00F0B3802378472B00F0BC80237840
:109BB000672B00F0C9802378462B00F0D0802378F3
:109BC000662B00F0D3802378522B00F0D6802378C8
:109BD000502B00F0E68023785E2B00F00A8123787A
:109BE000492B00F017812378432B00F0268123783E
:109BF000422B00F026812378552B00F02681237814
:109C0000572B00F029812378562B00F038812378D8
:109C10004C2B00F0418123784D2B00F051812378AB
:109C20004B2B00F099812378542B00F0B1812378DD
:109C3000442B00F0B1812378412B00F0C4812378BC
:109C4000592B00F0E28123784E2B00F0F781237826
:109C50004A2B00F0F7812378402B00F0F98123781C
:109C60006F2B00F00E822378642B00F01C82237887
:109C7000702B00F03A8223785B2B00F04F82237820
:109C80003D2B00F051822378732B00F05182257810
:109C90002C2D00F051822E2D00F0578223783E2B80
:109CA00000F0658223782D2B00F0AA8223782B2BDD
:109CB00000F0BC8204B070BD2A20954B98475AE74B
:109CC0002520934B98475AE72620914B98475AE70F
:109CD0007E208F4B98475AE76078000240F05A0088
:109CE0008B4B984757E7A378E27803EB022322795E
:109CF00003EB0243627903EB0263864A13606078E8
:109D0000000240F07A00824B984748E7637833B905
:109D10000120814B984724207D4B984743E7002042
:109D20007D4B9847F7E76378A07800EB032080B27B
:109D300010F4004F05D1794B98472420744B984775
:109D400035E747F6FF70F6E76378A07800EB03206D
:109D500000B2734B984724206D4B98472BE76078EF
:109D6000704B984724206A4B984728E760786E4BE1
:109D700098472420664B984725E76278A37803EB41
:109D800002239BB2092B05D9684A13802420604B1B
:109D900098471CE70122664B1A7045205C4B984798
:109DA00015E763785BB1012B16D00022614B1A7066
:109DB00001225F4B1A704520554B98470BE7022054
:109DC0005D4B984730B90422594B1A704520504BCF
:109DD000984700E72420FAE70120574B984720B91D
:109DE0000422534B1A70452000E02420484B98472A
:109DF000F1E663782BB1012B07D04520444B9847FF
:109E0000EDE65E20424B9847E9E64FF4AF70404BD9
:109E10009847E4E66278A37803EB0223474A13806D
:109E20000520454B984720B90422414B1A70452024
:109E300000E02420364B9847D5E64320344B984722
:109E4000D5E64220324B9847D5E662783C4B1A70F3
:109E500055202F4B9847D2E661780F2908D8202249
:109E60004901A01C374B98472420294B9847CAE644
:109E700001222F4B1A704520254B9847C3E6082036
:109E80002D4B984720B90422294B1A70452000E039
:109E900024201F4B9847BAE62B4B62781A70A278A1
:109EA0005A70E2789A700720234B984720B9042211
:109EB0001F4B1A70452000E02420154B9847AAE656
:109EC000224B98476378003318BF01230370A378AF
:109ED0004370E378003318BF012383702379C37084
:109EE00063790371A3794371E3798371237AC37131
:109EF000637A0372A37A4372E37A837209200E4B6A
:109F0000984728BB04220A4B1A70452021E000BF65
:109F1000C19A4000C4210020E57A4000AD7A40009B
:109F2000D97A40000154400085AE4000C82100208D
:109F3000CA2100208F220020D1B54000AA22002093
:109F4000C0210020118040008C220020155C4000C0
:109F50002420964B984762E66378A27803EB0223AD
:109F6000E27803EB0243227903EB0263904A136029
:109F70006379A27903EB0223E27903EB0243227AAD
:109F800003EB02638B4A13604B20884B98474AE6E9
:109F90005420864B98474AE609228749E01C874BA4
:109FA000984748B96278864B1A70A278854B1A7028
:109FB00044207E4B98473EE60122834B1A70452091
:109FC0007A4B984737E66278531EDBB21F2B06D9CF
:109FD00001227D4B1A704520744B98472FE6754B34
:109FE0001A60A378E17803EB0123217903EB0143A5
:109FF000617903EB01636E490B60A11D7348744BDB
:10A0000098474120694B984719E6002604AD45F86A
:10A01000046D704B984700953346012204216E4D24
:10A02000A847039B002B3FF40EAE4FF080526B4BC2
:10A030001A60BFF34F8FBFF36F8F04E64E205B4B68
:10A04000984704E6607800024A30584B984702E689
:10A050006078634B98475F4B984703AB00930023AE
:10A06000012204215C4DA847039B002B3FF4F7AD70
:10A070004FF08052594B1A60BFF34F8FBFF36F8F71
:10A08000EDE5E21C6178A078564B98470620564BC8
:10A09000984720B904224C4B1A70452000E0242038
:10A0A000424B9847DFE56078504B9847012803D032
:10A0B00045203E4B9847DAE524203C4B9847454BDA
:10A0C000984703AB0093002301220421424DA84787
:10A0D000039B002B3FF4CBAD4FF080523F4B1A60F7
:10A0E000BFF34F8FBFF36F8FC1E5414B9847394B9B
:10A0F000984703AB0093002301220821364DA8475F
:10A10000039B3BB14FF08052344B1A60BFF34F8F2B
:10A11000BFF36F8F2420254B9847ACE5354B98470C
:10A120002420224B9847AAE53D20204B9847AAE5DA
:10A1300073201E4B9847AAE508222F49601C1F4B2D
:10A14000984700287FF4A7ADFFDE08222A49601C4B
:10A150001A4B984700287FF4A1AD284B4FF40042DA
:10A160001A60402183F80F13C3F8002196E50822F6
:10A170002149601C114B984700287FF493AD154B83
:10A18000984703AB0093002301224FF48011124D36
:10A19000A847039B002B3FF485AD4FF080520F4B37
:10A1A0001A60BFF34F8FBFF36F8F7BE5C19A4000FA
:10A1B000BC210020CC210020004F41007120410033
:10A1C00054210020B8210020CA210020582100205D
:10A1D000D12041007DA4400055FF400004ED00E087
:10A1E000E1A44000C9B44000D1B540002DA5400015
:10A1F00069AE400079AE40000C4F410000E100E044
:10A20000154B984703AB0093002301222021134DE7
:10A21000A847039B002B3FF449AD4FF08052104BF1
:10A220001A60BFF34F8FBFF36F8F3FE50A4B98471C
:10A2300003AB0093002301224021084CA047039B5D
:10A24000002B3FF437AD4FF08052054B1A60BFF33F
:10A250004F8FBFF36F8F2DE57DA4400055FF400069
:10A2600004ED00E08388B3F59F5F0DD0B3F5706F08
:10A2700025D0B3F5206F2FD0B3F5A05F38D0B3F55C
:10A28000706F41D000207047C288B2F51F6FEDD1CA
:10A290004189A1F5E752093A92B2C62A45D9A1F5FA
:10A2A000DD521D3A92B2C62A01D802207047A1F5AC
:10A2B000B8510D3989B2C629D8D806207047C2884E
:10A2C000B2F5F06FD5D14289A2F50B52053A92B2A0
:10A2D000C62ACED803207047C288B2F5206FCBD1F2
:10A2E0004289A2F6553292B2C62AC5D805207047D7
:10A2F000C288B2F5206FC2D14289A2F6553292B21D
:10A30000C62ABCD805207047C388B3F5F06F01D0CA
:10A31000002070474389A3F5B8530D3B9BB2C62B71
:10A3200001D80420704700207047012070470000CA
:10A3300000B9704710B504460120034B9847601ED2
:10A34000FFF7F6FF10BD00BF75F8400038B50125D6
:10A35000044B1D7000210846034CA04700212846ED
:10A36000A04738BD3C0D00208D58400010B500249A
:10A37000022C09D80B4B1A78002108460A4B984743
:10A38000012801D00134F3E70024022C09D8054B41
:10A390001A7800210120044B9847012801D001348C
:10A3A000F3E710BD3D0D00208157400038B51A4B32
:10A3B0001B786BB90024022C1FD8184B1A78184B45
:10A3C00019880020174B9847012816D00134F2E76E
:10A3D00001210020144CA04701210846A047142069
:10A3E000124CA0470020124DA8470120A847142076
:10A3F000A0470022084B1A70DCE70024022C0AD880
:10A40000064B1A78064B19880120064B98470128FD
:10A4100001D00134F2E738BD3C0D00203D0D002095
:10A420002C010020815740008D58400075F84000F5
:10A43000B1584000F8B505460E460024204601E01C
:10A440000134A4B22746B4EB960F14D215F82410A9
:10A4500005EB84035A7801EB02219A7801EB024163
:10A46000DB7801EB03610028EAD107F5406080004A
:10A47000014B9847E4E7F8BDA56B4000014B186815
:10A48000704700BF440D0020014B1878704700BF93
:10A49000400D002010B582B0084B019300230093BB
:10A4A0004FF4807206490748074CA047012802D0A4
:10A4B0000648074B984702B010BD00BF440D00206E
:10A4C0001856410079A54000A1F5400024564100EE
:10A4D000291A4100014B1878704700BF380D002041
:10A4E00001280CD038B102280DD0FF280FD00A4A1D
:10A4F0000A4B1A6070470A4A084B1A607047094AAB
:10A50000064B1A607047084A044B1A607047024AAB
:10A51000024B1A60704700BF185541002801002007
:10A5200018514100184F410018504100032817D816
:10A53000DFE800F002070C110A4A0B4B1A600120F9
:10A5400070470A4A084B1A6001207047084A064BB8
:10A550001A6001207047074A034B1A6001207047B8
:10A560000020704718554100280100201854410070
:10A5700018534100185241002DE9F04184B00123E5
:10A580008DF80B30914B00241C605C609C60DC609B
:10A590008F4B0093234622468E498F488F4DA84704
:10A5A0008F4B186004A9502301F8063D03208D4D00
:10A5B000A84704A901F8074D0D20A84710B90023AA
:10A5C00003930BE09DF80900874B9847F7E74FF09E
:10A5D000FF3303AA00210846844CA047039B13F0D5
:10A5E000010FF4D040F21310814B9847814B9847EC
:10A5F0007648814B98474FF48071804B1868804BA8
:10A60000984706E04FF0FF3303AA00210846774C35
:10A61000A047039B13F0020FF4D01920744B984706
:10A62000784B4FF480721A63DB6B13F4004F1BD02E
:10A63000754B98470F20754B984701467148744BEE
:10A6400098470023734A1370734A13700DF10B017E
:10A650000420644B984728B19DF80B3083F0010328
:10A660008DF80B30002403E06C4B9847E2E70024A0
:10A6700014205F4B9847002303AAFC2118465B4D2A
:10A68000A847039B13F0080F00D0012413F0100F0C
:10A6900040F0E480039B13F0040F35D05D4B1B7832
:10A6A000002B40F031810F20584B98470146554808
:10A6B0005B4B9847594B98475A4B98474D4B984797
:10A6C00042484D4B98474D4D4FF4807128684C4B94
:10A6D00098472B68544A934200F02281534A934290
:10A6E00000F01E81474BDB6B13F4004F00F01B8121
:10A6F000454B98470F20454B984701464148444BEE
:10A70000984724204A4B9847039B13F0200F40F0B2
:10A710000D81039B13F0400F40F01681039B13F053
:10A72000800F08D0434B1B788DF80A30394B1B78CB
:10A73000002B40F03081039B13F4801F40F03681E2
:10A74000344B1B78002B40F035813B4B9847002859
:10A7500040F0568100232F4A13702F4A13709DF842
:10A760000B3093B1354B1B787BB1354B1B78002BED
:10A7700000F08682334B984738B90022304B1A706C
:10A78000314B9847002840F06982002C3FF470AFAD
:10A790002B4B1D78002D7FF46AAF1E4B1C78002CCC
:10A7A0003FF466AF0122294B1A70294B98470C4B96
:10A7B00018680A23009300231A460321254CA0475A
:10A7C0000022254B1A702C4652E700BF10220020B1
:10A7D0004DA34000E09304004C5641003D0241006F
:10A7E00020220020B58040002DA5400005FE40003D
:10A7F00075F84000016B4000D56F40002801002033
:10A8000035A44000000E0E40DD5440000BDF400038
:10A81000E7DE4000400D00203B0D0020B954400011
:10A82000EBDE40003D6B400018514100184F4100E5
:10A83000A59A4000882200201D0C41002401002020
:10A840002E010020FD5B400089A44000380D00204F
:10A85000ADA34000790241003C0D00200F208E4B3B
:10A8600098478E4E014630468D4B98478D4B984702
:10A870004FF4804777630A208B4DA8478B4B98474E
:10A880004FF4FA70A8478A4B984777630120894BA9
:10A8900098471920A8474FF4807333630020864EF1
:10A8A000B0470120B04700210846844EB047002140
:10A8B0000120B04701210020814EB0470121084608
:10A8C000B0471420A84700207E4EB0470120B04773
:10A8D0004FF001087C4B83F8008000267B4B1E70F4
:10A8E0007B4B98479DF80A103346032241F4807150
:10A8F000784FB847784B9847334642460221B847CD
:10A900004FF0FF30A847C5E600226F4B1A70634D29
:10A910004FF480766E631920634B98472E63C2E62E
:10A920006E4B9847DEE65F4B9847E3E66C4B9847E3
:10A93000012803D045206B4B9847EAE66A4B9847BD
:10A940002420684B9847E4E6654B9847012803D0DC
:10A950004520644B9847E1E64FF480724F4B5A63B1
:10A96000594B1B78A3B9C8204F4DA8470120514B24
:10A970009847C820A8474FF48072484B1A630023B9
:10A98000514A1370514A13702420564B9847C5E61C
:10A99000564B9847E7E74E4B98479DF80A1000231F
:10A9A000032241F480714B4DA847C4E64020504B30
:10A9B0009847C5E64F4B984720B14F4B9847002822
:10A9C0007FF4C3AE0025404B1D70404B1D704B4BB8
:10A9D0001D703F4B98472B4603224FF480713D4E2C
:10A9E000B0473D4B98472B4601220421B0472B4DE1
:10A9F0004FF480766E6319202B4B98472E63A4E6A4
:10AA00003D4B984700283FF4A5AE2F4B1B78002BF9
:10AA10007FF4A5AE00203A4EB0473A4D2870012091
:10AA2000B047394B18702B78002B3FF498AE0028B4
:10AA30003FF495AE0122244B1A70344D2846344B16
:10AA4000984734493448354B98472846344B984703
:10AA50000746431FDBB2012B19D90022314B1A7074
:10AA60004FF4FA70104B98470020254EB047254D03
:10AA700028700120B047244B18702B780BB10028A8
:10AA800052D10023104A1370104A137067E6012256
:10AA9000244B1A70E4E700BF0BDF4000000E0E40AD
:10AAA000EBDE4000B954400075F84000557D400091
:10AAB000757C4000A17C4000655A40006958400008
:10AAC0008D584000B1584000400D00203B0D002043
:10AAD00029B64000A9FE400035B64000116E400086
:10AAE000510C4100A59A40000D7D4000496E400088
:10AAF00031A340001D0C4100290C4100380D0020FD
:10AB00009D6C40003E0D00203F0D00207C22002067
:10AB1000D96C4000390D00203A0D0020E56D400051
:10AB200065A240003D0D0020654B98479DF80A1036
:10AB30000023032241F48071624DA847624B98477D
:10AB4000002301220221A847394600205F4DA84773
:10AB500039460120A8470A205D4B9847F0B95D4D62
:10AB6000002128465C4B98472B78112B1BD00022E4
:10AB70005A4B1A7000210846594DA8470021012060
:10AB8000A8470025022D23D8564B1A7800210846E5
:10AB9000554B984701281BD00135F3E753490A204C
:10ABA000534B9847DBE76B78002BE0D1AB78002B59
:10ABB000DDD1EB78892BDAD12E46294600204D4D88
:10ABC000A84731460120A8470122444B1A70D1E71B
:10ABD0000025022D09D8434B1A7800210120424B51
:10ABE0009847012801D00135F3E701210020424DAB
:10ABF000A84701210846A8471420404B9847002049
:10AC00003F4DA8470120A8479DF80B3003B33D4BAB
:10AC10009847E8B13C4B1B78D3B13C4B1B782BB128
:10AC200001223B4B1A703B4B984798E50025384B67
:10AC30001D70394B9847394B1E68394B98470A238A
:10AC400000932B46024601213046364DA84786E543
:10AC500001222F4B1A702F4B984780E500252C4B73
:10AC60001D702D4B98472D4B1E682D4B98470A237E
:10AC700000932B460246012130462A4DA84784E521
:10AC8000294B984700283FF480AD01221F4B1A70D2
:10AC9000264B984700283FF478AD01221C4B1A70D0
:10ACA0001C4B98471D4B18680A23009300231A4633
:10ACB00003211C4DA84700221D4B1A7065E500BFFB
:10ACC00029B64000A9FE400035B640009559400025
:10ACD0000181400024220020F56B40003B0D002044
:10ACE000695840003D0D0020815740002C01002094
:10ACF000B5804000815940008D58400075F84000F3
:10AD0000B1584000395B4000240100202E01002092
:10AD1000380D0020ADA340006DA34000202200208C
:10AD20009DF6400079024100FD5B400089A440008F
:10AD30003C0D0020124A1080124A12787AB138B5C0
:10AD400004460025022D0CD80F4B1A78214600200E
:10AD50000E4B98470346012803D00135F2E7012046
:10AD6000704718460025022D09D8074B1A7821464E
:10AD70000120064B9847012801D00135F3E738BD83
:10AD80002C010020380D00203D0D0020815740008F
:10AD900010B5044B9847002303221021024CA04712
:10ADA000012010BD7DA44000A9FE4000014B188881
:10ADB000704700BF2C01002010B5224B1B78002BE0
:10ADC0002CD10024204B1B780BB144F002041F4B04
:10ADD0001B780BB144F004041D4B1B780BB144F0FD
:10ADE00008041C4B1B785BB31B481C4B984744EA78
:10ADF0000014A4B21A4B1B78063B182B16D8DFE8B8
:10AE000003F00F151515171515151515151515152D
:10AE10001115151515151515151513000124D1E774
:10AE2000012006E0032004E0042002E0002000E00E
:10AE3000022044EA00240B4B1878000380B204433C
:10AE4000204610BD380D00202E0100203C0D0020B2
:10AE50003B0D0020400D00207C22002065A2400018
:10AE60003A0D0020390D00200022024B1A700120FB
:10AE7000704700BF240100200120014B187070476B
:10AE80002401002010B584B000230393642800D966
:10AE900064200B4B18700B4B984703AB00930023B7
:10AEA00001228021084CA047039B3BB14FF0805208
:10AEB000064B1A60BFF34F8FBFF36F8F04B010BD06
:10AEC000882200207DA4400055FF400004ED00E0F2
:10AED00038B50024204609E000F47F43B3F5007F35
:10AEE0000CD000F47F43B3F5807F0CD00028F3D161
:10AEF0004FF0FF310120134B9847EDE70020124B34
:10AF000098470020EDE7C5B2002008E00134A4B264
:10AF100020460D4B98470A2101200A4B984758B903
:10AF2000AC42F3D308E0013CA4B22046064B98475C
:10AF30000A210120034B98470028D7D1AC42F2D810
:10AF4000D4E700BF81FD400001544000F0B583B05C
:10AF50000224002010F0010F0AD14FF0FF31012030
:10AF6000314B984700F00E03042BF3D10424F1E792
:10AF70002E4B1B68ADF804301B0C8DF8063001A970
:10AF800002202B4B9847042C07D02A4B984701A945
:10AF9000294B984700252E4607E0264B984700216D
:10AFA000264B9847F1E72E460225322101201E4B01
:10AFB000984700F00E00042812D0022814D0042C68
:10AFC000F3D1C5B1022D22D0032DEED10136F6B258
:10AFD000182EEAD900252E46E7E703250026E4E7E8
:10AFE00000252E460424E8E7124B98478021134B96
:10AFF00098470224E3E70F4B9847771CFFB2104BAA
:10B00000995D0E4B9847632FCDD83E46CDE7094B4F
:10B010009847771CFFB20B4B995D084B9847632FFD
:10B02000DBD83E46C1E700BF81FD400060564100CD
:10B03000B5804000CD0B4100C1634000716340000A
:10B04000940100203001002008B5044B984764208B
:10B05000034B9847034B9847F7E700BFC970400080
:10B0600075F840006982400070B582B0944B9847F3
:10B07000944B98470120944B984702A9002301F86C
:10B08000013D0520914B984728B19DF8073013B139
:10B0900000208D4B98478E4B98478E4B98478E4A91
:10B0A0008E4B1A6001208E4B98470446D0B98A4DCA
:10B0B0008C4C0FCC28606960AA60EB608A4B984783
:10B0C0008A4B98478A4B984701281AD0884B984753
:10B0D00002281BD00222874B1A63874B98470546EC
:10B0E000002420E07D4B19680120784B984705E04B
:10B0F0007A4B1B6800221A550134E4B20F2CF7D9A1
:10B10000DCE77E4B98477E4B9847E3E77B4B9847BD
:10B110007C4B9847DEE705207B4B9847764B98475A
:10B1200005460134E4B20DB9132CF4D9774B984796
:10B130002946774B9847774B9847774DA847002388
:10B1400001221146754CA0470120754B9847A8472E
:10B15000002301220221A047724B9847674B984772
:10B16000714B984700230122052170480068A047D1
:10B1700000252C4682E01146002341F8043B6C4830
:10B180006C4B984738B96C4B596801315960684825
:10B190006A4B98477DE001216548684B984778E005
:10B1A0001146002341F8043B6548624B984798B923
:10B1B000644B5968013159606148604B9847624956
:10B1C00062485C4B984760B95E4B596801315960E1
:10B1D0005E485A4B98476AE001215948574B9847B7
:10B1E000EDE701215948554B984760E0134600228E
:10B1F0001A605A6801325A60694655484D4B984763
:10B2000050B9544B5968009B994201D8002515E06C
:10B210004F484A4B9847F9E74E4B59684C48474BC3
:10B220009847F3E74C4A136801331360052B40F24B
:10B230009D80484B00251D605D601560474BA3FB5A
:10B240000423DB0803EB83035A00944200F0908050
:10B25000434B9847002840F09E80424BA3FB0423B9
:10B260005B09642202FB1343002B00F097800A2045
:10B27000254B98470134632C00D900240135B5F5DE
:10B280007A7FDBD32C4A1368013313603B2B3FF6E4
:10B2900072AF354B98470028C4D000222E4B1A605D
:10B2A000284A1368013313603B2B3FF679AF294AD4
:10B2B0001368013313603B2B98D80025BEE700BF0D
:10B2C000958640009D814000AD544000B58040000F
:10B2D000B9544000F5524000B022002090220020D6
:10B2E0000181400018574100350C41005D0C4100C0
:10B2F000510C4100000E0E4029714000CD0B410061
:10B30000696740007964400075F84000C50B410052
:10B3100031684000757C40007DA44000A9FE4000DB
:10B32000A17C4000755A4000AD6240006C0D0020C9
:10B330000110FFFF9D8740005C0D0020F187400059
:10B340000210FFFF4C0D0020500D00200410FFFFE5
:10B350000310FFFF540D0020480D0020CDCCCCCCB5
:10B36000395B40001F85EB51D5A44000002565E7FF
:10B370000C4B984728B947230B4A13700B4A13709C
:10B3800066E700200A4EB047074B18700120B0470F
:10B39000064B18705CE7074B984768E7064B9847E1
:10B3A00065E700BF89A44000F8010020F9010020F2
:10B3B00009594000455B4000755A400008B509E056
:10B3C00000210846314CA04700210120A04700225F
:10B3D0002F4B1A704FF0FF3101202E4B98472C4B0A
:10B3E0001B78013B082BF2D801A252F823F000BFD2
:10B3F00015B44000C1B340002FB440003FB440003A
:10B4000025B4400077B440005FB440006BB4400006
:10B4100071B44000012100201C4CA04701210846C6
:10B42000A047D4E71C4B18881C4B9847CFE7002156
:10B4300008461B4CA04700210120A047C7E7012177
:10B440000020174CA04701210846A0471420154BA7
:10B4500098470020144CA0470120A047B7E7134BA2
:10B4600098471349134B9847B1E7134B9847AEE7FA
:10B47000124B9847ABE7124AD01E134612F8032C22
:10B48000817840780F4CA047A1E700BFE958400001
:10B490008F22002081FD4000AA22002035AD40000F
:10B4A0008D58400075F84000B1584000CD0B410068
:10B4B0008C220020C163400055804000215C400088
:10B4C000C3220020F955400010B51446044B1870F3
:10B4D000597002462146981C024B984710BD00BF88
:10B4E000C0220020D120410010B582B0234B01932F
:10B4F000032300930023802221492248224CA047A5
:10B50000012802D02148224B9847224B0193002367
:10B5100000938022204921481B4CA047012802D0DB
:10B520001F481B4B984700230193009380221D491D
:10B530001D48154CA047012802D01C48144B9847C1
:10B540001B4B01930023009380221A491A480E4C8A
:10B55000A047012802D019480D4B9847184B01937A
:10B5600000230093802217491748074CA047012861
:10B5700002D01648064B984702B010BD680D002057
:10B5800064564100BDB34000A1F54000685641003B
:10B59000291A4100700D00208456410069B0400016
:10B5A00090564100B856410049B04000BC56410099
:10B5B0006C0D0020D85641004DAF4000DC564100D4
:10B5C000640D0020F8564100D1AE4000FC56410009
:10B5D00010B584B0104B18700022039204AB43F8EE
:10B5E000082D0E4A106803AA0092042201210C4C77
:10B5F000A047029B5BB9039B63B14FF08052094B9C
:10B600001A60BFF34F8FBFF36F8F012000E000205F
:10B6100004B010BD0120FBE78F220020680D002040
:10B6200055FF400004ED00E0014B1868704700BF73
:10B63000640D0020014B1868704700BF6C0D00209E
:10B640000023044A1370044A13700120034B18703E
:10B65000704700BF7C0D0020780D0020750D002084
:10B6600070470020704700000D4B5B881A0A032AC0
:10B6700001D00020704713F0FF0F0ED1084BDB887C
:10B68000402B01D000207047054B064A9A60064ABD
:10B690001A6140229A81012070470020704700BF44
:10B6A00024230020800D0020DDB640000122014B44
:10B6B0001A707047750D002010B5034B034A0449FA
:10B6C0000448054CA04710BD69B64000CC020020DC
:10B6D000780D00207C0D002021B8400008B5084BF3
:10B6E0009B89402B00D008BD064B1B781BB9064830
:10B6F000064B9847F7E70448054B984708BD00BF3D
:10B7000024230020740D0020800D0020699B400040
:10B7100021504000014B1870704700BF740D00208D
:10B72000224B1B780BB9184670472DE9F04184B0C5
:10B730000746EFF31083B3FA83F35B09039372B602
:10B74000BFF35F8F00211A4B1970DDF80C80194D83
:10B7500040222846184B98473C4640372E462068E2
:10B760006168A268E3680FC610343546BC42F5D163
:10B77000124B009340230F4A00218120104CA04718
:10B7800080F00100094B1870B8F1000F05D00122BC
:10B79000074B1A70BFF35F8F62B6044B1B7883F0C0
:10B7A0000103184604B0BDE8F08100BF750D00200C
:10B7B0002F030020C00D0020CD224100ADB6400077
:10B7C000FDD9400010B50446134B9847837A212BCE
:10B7D00001D0002010BD00F10902104B5B881B0A4C
:10B7E000212B04D0C27B93420BD0002010BD0B4B09
:10B7F0009A60427AD9888A4228BF0A469A810120F3
:10B8000010BD064B9C60028AD9888A4228BF0A462E
:10B810009A81012010BD00BFF9BD40002423002003
:10B82000F8B5264C247865B2002D07DB002D40DBEF
:10B8300004F06004202C22D00020F8BD14F0600633
:10B8400003D11E4F7F78062F0BD0202EEED11B4A3E
:10B850005278022A09D0032A0CD0012AE6D198474F
:10B86000F8BD1046164B9847F8BD144B9860012060
:10B870009881F8BD114B996001209881F8BD0F4A5D
:10B8800052780A2A07D00B2A0BD0092A01D00020AF
:10B89000F8BD9847F8BD094B5B881B0A037001206F
:10B8A000F8BD064BDB8833B9044B5B880B70012075
:10B8B000F8BD0020F8BD0020F8BD00BF2423002003
:10B8C000C5B74000014B1868704700BF90220020A8
:10B8D000024B1B681B685888184470470C0E0020E8
:10B8E00038B504460D46094B984702462078204457
:10B8F000904207D24378042B06D0AB4205D00378A0
:10B900001844F5E7002038BD002038BDD1B840000C
:10B9100038B5144B1B780BB3134B1B681B681A7993
:10B9200082421DD90D460446104A1360104B9847B9
:10B9300003E01A7813440D4A13600C4B1B689842BD
:10B940000AD95A78042AF4D19A789442F1D1DA7853
:10B95000AA42EED1012038BD002038BD002038BDFC
:10B96000002038BD080E00200C0E0020100E002014
:10B97000D1B84000084BDB8863B9074B5B88012BCB
:10B9800001D000207047054A138823F0020313807A
:10B99000012070470020704724230020000E002063
:10B9A00000207047044BDB8823B9044A024B1A611C
:10B9B000012070470020704724230020E9BC40008C
:10B9C00038B5134B1B7803B3124B1C79124B1B6811
:10B9D0001B681B799C4201D3002317E000212046FD
:10B9E0000E4B9847034688B10B4B1B685B6853F8B6
:10B9F0002450EB68984701462046084B9847034679
:10BA000020B1AB689847034600E00023184638BDD4
:10BA1000080E0020242300200C0E002011B9400045
:10BA200038B5104B1B78D3B100240F4B1B681A6834
:10BA30001279944211D25B6853F82450EB6898470E
:10BA400001462046094B9847034648B1AB689847E2
:10BA5000034628B90134E4B2E7E7002300E00023FD
:10BA6000184638BD080E00200C0E002011B9400009
:10BA700070B504460021114B9847054608B9284681
:10BA800070BD0F4B1B685B6853F82460F3689847E0
:10BA900001462046094B984705460028EFD0094B40
:10BAA0001C6805212046084B9847044618B1807849
:10BAB000064B9847F5E773689847E0E711B94000EF
:10BAC0000C0E0020100E0020E1B840007DD7400091
:10BAD00008B5064BDB88022B01D0002008BD0221EF
:10BAE0000348044B9847012008BD00BF24230020D1
:10BAF000000E002061D6400010B5184B9B78032B38
:10BB00002AD8DFE803F00502100B0920144C0CE0E2
:10BB100004211448144B9847002006E0134B984723
:10BB20000446102001E00620114C08B1002308E073
:10BB3000012010BDE15C0F4A02EB4302518001334A
:10BB4000DBB28342F6D3411C4900C9B209480170F7
:10BB5000054B9847012010BD002010BD2423002074
:10BB60001C0300201803002061D64000C5B8400027
:10BB700028030020F402002008B5234B5B88DAB2CA
:10BB80001B0A013B0E2B38D8DFE803F008173137CA
:10BB9000373737373737373737372A001B4B18686F
:10BBA00001781B4B9847184BDA889B899A4228D218
:10BBB000154B9A810123184608BD144B1B685B7C0A
:10BBC0009A4201D30023F6E7104B5B6853F832002A
:10BBD00041880F4B98470C4B9B6802225A70E2E752
:10BBE0000A4B986858B14188094B9847DBE7094BE5
:10BBF000984703460028D6D1DDE70023DBE7002382
:10BC0000D9E70123D7E700BF24230020FC0100204F
:10BC100061D64000F9BA400008B5064BDB88012B1D
:10BC200001D0002008BD01210348044B98470120A2
:10BC300008BD00BF24230020080E002061D640006C
:10BC400038B5154BDB88012B02D00024204638BDC7
:10BC5000124B1B78F3B1104B1D79114B1B681B68FD
:10BC60001B799D4201D30024F0E7002128460D4BAB
:10BC7000984704460028E9D0094B1B685B6853F8D5
:10BC80002530DB689847084B187001211846074B90
:10BC90009847DBE70024D9E724230020080E002082
:10BCA0000C0E002011B94000040E002061D64000A7
:10BCB00008B5094BDB88022B01D0002008BD064BDC
:10BCC0001879064B9847064B188002211846054BF9
:10BCD0009847012008BD00BF24230020CDD7400095
:10BCE000020E002061D6400008B5034B588800F0D2
:10BCF0007F00024B984708BD2423002009D640004E
:10BD000038B505460F4B98470346C0B10E4B1C682B
:10BD1000052120460D4B9847044640B18288C178E2
:10BD200080780B4B984703460028F1D107E0094B78
:10BD30001B685B6853F825301B6898470346184614
:10BD400038BD00BF11B94000100E0020E1B840001E
:10BD50006DD640000C0E002038B50C4BDB8893B933
:10BD60000B4B1B780BB900230EE0084B1C799D7818
:10BD70002046084B9847034630B129462046064BDB
:10BD80009847034600E00023184638BD24230020CE
:10BD9000080E002071BA400001BD400008B5074BF5
:10BDA000DB884BB9054B5B880BB1002008BD034B0A
:10BDB0001879034B984708BD002008BD24230020B4
:10BDC00009D94000094BDB886BB9084B5B880BB184
:10BDD0000020704710B5054C2079054B9847207915
:10BDE000044B984710BD0020704700BF242300205B
:10BDF00079DB400011D84000014B1868704700BF44
:10BE0000100E002008B5014B984708BDA9D440008A
:10BE100010B50B4B1B7863B1002404E02046094B9E
:10BE200098470134E4B2084B1B681B681B799C429D
:10BE3000F4D30022024B1A700122044B1A8010BD69
:10BE4000080E002071BA40000C0E0020000E0020E9
:10BE500008B5024B9847024B984708BD91D5400062
:10BE600011BE40001C4BDB8813B1002318467047FD
:10BE700010B51A4B984750B3174B9A78184B1B685C
:10BE80005B7C9A4201DD002322E0164B9847124B5F
:10BE90009B78154A1370EBB1114A526803F10053B5
:10BEA000013B02EBC303114A136000240F4B1B68D4
:10BEB0001B681B799C4208D2002120460C4B9847F6
:10BEC000034628B10134E4B2F0E7012300E0002387
:10BED000184610BD0123FBE72423002045D640006F
:10BEE000FC01002011BE4000080E00200C0E0020B6
:10BEF00001BD400008B5344B1B7813F0800F0ED104
:10BF000013F01F0343D1304A5278013A082A3ED831
:10BF1000DFE802F0343D373D313D3D3D3A002A4AED
:10BF2000D288002A4ED013F01F0306D1264A527839
:10BF3000062A0BD0082A0CD02AB1012B0CD0022BD8
:10BF400011D0002008BD214B984708BD204B9847D1
:10BF500008BD204B984708BD1B4A52780A2AEED1EB
:10BF60001D4B984708BD184B5B780BB1002008BDEE
:10BF70001A4B984708BD1A4B984708BD194B98476C
:10BF800008BD194B984708BD184B984708BD012BB1
:10BF900003D0022B08D0002008BD0B4A52780B2A90
:10BFA000F7D1134B984708BD074B5B78012B03D0A3
:10BFB000032B04D0002008BD0E4B984708BD0E4B44
:10BFC000984708BD002008BD24230020D1BA4000B6
:10BFD00079BB400019BC400041BC4000B1BC4000EE
:10BFE000A5B9400075B94000A1B9400065BE400048
:10BFF00059BD40009DBD4000C5BD40000B4B1B78A6
:10C0000013B110B5002402E070470134E4B2084BCC
:10C010001B681A681279944207D25B6853F824307F
:10C020001B69002BF1D09847EFE710BD080E0020E8
:10C030000C0E002008B5184B00229A811A615A6133
:10C040001B7813F0800F11D113F0600F14D0124B36
:10C050001B7803F01F03012B14D00F4B1B7803F048
:10C060001F03022B14D00023184608BD0A4AD288A9
:10C07000002AE9D10023F7E7084B98470346002838
:10C08000E5D0F1E7064B984703460028E5D0EBE7FB
:10C09000044B98470346E7E724230020F5BE400001
:10C0A000C1B9400021BA4000F8B504460E46114B14
:10C0B000984705462046104B9847054001D000247C
:10C0C00003E0F8BD0134062C11D88DB123010B4AD1
:10C0D000D058B042F6D102EB041359680D42F1D0AA
:10C0E0001F46DB6898477B6825EA0305EAE7F8BD49
:10C0F000F8BD00BFEFDE4000F3DE4000140E00206C
:10C10000F8B5164C2768062F26D8002401E0013424
:10C11000E4B2A446A7420AD3114E250106EB050E50
:10C1200075598D42F3D1DEF804509542EFD1CEF827
:10C130000010CEF80420CEF808300699CEF80C1086
:10C140000137BC4505D011461A46064B98470020DA
:10C15000F8BD02490F60F6E70120F8BD840E00200B
:10C16000140E0020B5DE40002DE9F04182B00446F7
:10C170000F4690460A4B984705462046094B98477C
:10C1800006462046084B9847CDF800803B460246BD
:10C1900031462846054CA04702B0BDE8F08100BFFB
:10C1A000F7DE400005DF40000BDF400001C140002A
:10C1B00008B50B210148024B984708BD000E0E4000
:10C1C000A9C0400008B50C210148024B984708BDA2
:10C1D00000100E40A9C04000F8B506460C461546B2
:10C1E000224B984707464FF0FF313046204B984787
:10C1F0003046204B9847002C0CDB630904F01F01EC
:10C2000001228A4020331C4941F82320BFF34F8F7D
:10C21000BFF36F8F002C08DB630904F01F010122BC
:10C220008A406033144941F82320002C17DB2D018C
:10C23000EDB204F1604303F5614383F80053002C31
:10C2400008DB620904F01F04012303FA04F40A4B1B
:10C2500043F8224039463046084B9847F8BD04F071
:10C260000F022D01EDB2064B9D54E8E7F3DE4000CE
:10C27000EBDE4000EFDE400000E100E0E7DE4000E2
:10C2800014ED00E082B0024610B9244B1B783BB994
:10C2900012B1224B1B780BB3204B1A7002B07047BF
:10C2A0001F4B1B7803B9FEE7EFF31083B3FA83F358
:10C2B0005B09009372B6BFF35F8F0021194B1970B1
:10C2C000009817490B78013B0B700028E0D0012142
:10C2D000144B1970BFF35F8F62B6D9E7104B1B7810
:10C2E000FF2B19D0EFF31083B3FA83F35B090193AB
:10C2F00072B6BFF35F8F00210A4B1970019808498D
:10C300000B7801330B700028C6D00121054B197042
:10C31000BFF35F8F62B6BFE7FEE700BF890E002064
:10C320003C2300202F03002084B02A4B9A6842F45B
:10C3300080729A609A6822F07F029A601A6B01926A
:10C34000019A42F04F020192019A22F4074222F030
:10C3500080020192019A42F400420192019A1A630A
:10C360001C4B1B6B13F4004FFAD01A4A136B029349
:10C37000029B43F04F030293029B43F4004302935A
:10C38000029B136300238DF8033006E000BF9DF885
:10C3900003300133DBB28DF803309DF80330DBB29C
:10C3A000132BF3D9EFF31083B3FA83F35B090393F1
:10C3B00072B6BFF35F8F0022074B1A70039B0121F7
:10C3C000044A116123B1044B1970BFF35F8F62B649
:10C3D00004B07047004004402F030020034A0023AC
:10C3E000136153619381024A137070472423002024
:10C3F0008E0E002082B00522104B1A70104A136B6B
:10C400000193019B43F04F030193019B43F02003F1
:10C410000193019B136300238DF8033006E000BFF6
:10C420009DF803300133DBB28DF803309DF8033003
:10C43000DBB2132BF3D902B0704700BF8E0E002081
:10C440000040044082B00322104B1A70104A136B54
:10C450000193019B43F04F030193019B43F01003B1
:10C460000193019B136300238DF8033006E000BFA6
:10C470009DF803300133DBB28DF803309DF80330B3
:10C48000DBB2132BF3D902B0704700BF8E0E002031
:10C49000004004400422014B1A7070478E0E0020A9
:10C4A00008B5024B1B6903B1984708BD242300203F
:10C4B00030B589B06A4B1B78032B29D0694B9C8916
:10C4C000694B1B88E41AA4B2002C43D1674A118837
:10C4D0000B449BB21380634AD288934203D0644BCF
:10C4E0001B78002B2CD0634B9847634A136B039344
:10C4F000039B43F04F030393039B23F00103039338
:10C50000039B13635C4B1B6B13F0010FFAD115E017
:10C51000594A136B0293029B43F04F030293029B11
:10C5200023F001030293029B1363534B1B6B13F025
:10C53000010FFAD1514B9847514B984709B030BD84
:10C54000484B5B6933B1984720B10022464B1A80B3
:10C55000444B9C893F2C37D90022454B1A7040240C
:10C56000404B9A68404B1B881A44EFF31083B3FA90
:10C5700083F35B09079372B6BFF35F8F0021414BD2
:10C58000197007983C4B1B6B13F0020F3ED028B17B
:10C5900001223C4B1A70BFF35F8F62B60422304B0E
:10C5A0001A70354A136B0493049B43F04F030493B2
:10C5B000049B23F001030493049B13632E4B1B6B1A
:10C5C00013F0010FFAD1B9E70122294B1A70C7E71E
:10C5D000157829490D650133DBB2013299B28C42DD
:10C5E000F6D8214B1A8814441C80234A136B0593F8
:10C5F000059B43F04F030593059B43F01003059300
:10C60000059B136300238DF8073008E00023E5E75E
:10C6100000BF9DF807300133DBB28DF807309DF87D
:10C620000730DBB2132BF3D9134A136B0693069B27
:10C6300043F04F030693069B23F001030693069BEA
:10C6400013630D4B1B6B13F0010FFAD100283FF45D
:10C6500075AF01220B4B1A70BFF35F8F62B66DE7A7
:10C660008E0E0020242300208A0E00208C0E002035
:10C67000880E002095C4400000400440A1C4400042
:10C68000DDC340002F03002010B586B0654B1B783A
:10C69000012B1ED0022B04D0042B02D0624B9847F2
:10C6A00001E0624B9847624A136B0093009B43F092
:10C6B0004F030093009B23F002030093009B13633E
:10C6C0005B4B1B6B13F0020FFAD15A4B984706B025
:10C6D00010BD574B186BC0F30A40574B9B89574A04
:10C6E00014882218934201DA181B80B2524B9A68C0
:10C6F0002244002305E04E49096D11700133DBB27D
:10C70000013299B28842F6D80444A4B24B4B1C8043
:10C7100040281BD0484B9C815B6913B19847002887
:10C7200032D0434A136B0293029B43F04F030293B0
:10C73000029B23F002030293029B13633C4B1B6B8F
:10C7400013F0020FFAD13E4B9847C0E73A4BDA8814
:10C750003C4B1B8823449A42DCDD374B9B899C422F
:10C7600027D0334A136B0593059B43F04F03059382
:10C77000059B23F002030593059B13632C4B1B6B56
:10C7800013F0020FFAD1A2E7274B9847284A136B00
:10C790000193019B43F04F030193019B23F002039C
:10C7A0000193019B1363224B1B6B13F0020FFAD111
:10C7B0008DE7214B5B6953B19847E8B121491F4A86
:10C7C0000B88108803440B8000231380C9E7164BA5
:10C7D0009847174A136B0393039B43F04F0303934C
:10C7E000039B23F002030393039B1363104B1B6B08
:10C7F00013F0020FFAD16AE70B4B98470C4A136B00
:10C800000493049B43F04F030493049B23F002031F
:10C810000493049B1363064B1B6B13F0020FFAD1B6
:10C8200055E700BF8E0E0020F5C34000A1C44000B4
:10C8300000400440DDC34000242300208A0E002075
:10C8400045C440008C0E00200023042B14D810B4E3
:10C850000A499A00D418A00004460844407C2144A8
:10C8600000F083026FF3C7124A740133DBB2042B6A
:10C87000EED95DF8044B7047704700BF900E002062
:10C8800038B5437C13F0100F16D00D46437C6FF380
:10C890000413437404687CB102F10C03074951F896
:10C8A000233013F4806F01D042F080028168012DA3
:10C8B00014BF00200120A04738BD00BF0040044045
:10C8C00010B500240BE023460134E4B203EB8303EC
:10C8D000980022460121034B1844034B9847042C2F
:10C8E000F1D910BD900E002081C8400010B500F0B5
:10C8F0000F02531E03EB83039C00012102482044D6
:10C90000024B984710BD00BF900E002081C8400028
:10C9100030B482B00246441E3B4900F10C0551F888
:10C92000253051F8251013F0020302D001F0400128
:10C9300051B9002B39D004EB84039900334B0B44DD
:10C94000597C6FF38301597404EB840399002F4BD6
:10C950000B445B7C13F00C0F32D12B4900F10C051A
:10C9600051F825300093009B43F04F030093009B48
:10C9700023F002030093009B41F8253002F10C03E1
:10C98000214951F8233013F0020FF7D1002838D095
:10C99000032836D004EB8404A2001C4B13445A7CB9
:10C9A000012161F383025A742BE004EB84039900A4
:10C9B000164B0B44597C012565F383015974C3E779
:10C9C00011490C3051F820300193019B43F04F0383
:10C9D0000193019B23F040030193019B41F8203018
:10C9E00002F10C03084951F8233013F0400FF7D13E
:10C9F00004EB8404A200054B13445A7C6FF38302BA
:10CA00005A7402B030BC704700400440900E0020C1
:10CA1000F0B4461EB300334499002A4A0A445368CE
:10CA2000D1680B449468641A128AC2F309029442D2
:10CA300009D31446002706EB86029500214A2A44B2
:10CA40002144D1601EE00127F5E71D781E4A00F160
:10CA5000140142F821505D7842F821509D7842F847
:10CA60002150DD7842F821501D7942F821505D793E
:10CA700042F821509D7942F82150DD7942F8215049
:10CA8000083C0833072CE0D807E01D7800F11402B9
:10CA90000D4941F82250013C0133002CF5D1094BDE
:10CAA000B1008819820010461A44527CC2F38102F8
:10CAB00003440132597C62F3830159743846F0BC57
:10CAC000704700BF900E00200040044070B582B057
:10CAD000441E04EB84039A00364B13445B7CC3F37F
:10CAE000810328B1032801D0022202E0012200E0E4
:10CAF00001229A4254DDA200224495002D4B2B4482
:10CB0000DA689B689A4205D32A4B2B445B7C13F06E
:10CB1000400F48D00E460546274B9847FEB1274A9E
:10CB20000C3552F825300193019B43F04F030193DC
:10CB3000019B43F010030193019B42F82530002331
:10CB40008DF8033006E000BF9DF803300133DBB2FF
:10CB50008DF803309DF80330DBB2132BF3D940B1CD
:10CB600004EB84039A00134B13445A7C6FF3861230
:10CB70005A74A200224491000E4B0B44DA689B6861
:10CB80009A4212D30B4B0B445B7C13F0400F0ED137
:10CB9000084B0B445A7C42F080025A74002000E09B
:10CBA000012002B070BD0020FBE70120F9E7012061
:10CBB000F7E700BF900E002011CA4000004004407B
:10CBC0002DE9F84305468446471EBB003B449A00C6
:10CBD0002A4C1444A268E368A2EB030EB4F8108058
:10CBE000C8F3090862681A440C30254951F82060DE
:10CBF000C6F30A4666B3B6450BD9B6464FF00009F0
:10CC000007EB870188001D4901447344CB60002174
:10CC10000AE04FF00109F3E70CF11403184850F84B
:10CC200023301370013101328E45F5D82846154B5B
:10CC30009847B9F1000F01D1B04507D905F10C03B0
:10CC40000F4A52F8233013F0200F04D0BDE8F883C8
:10CC50004FF00009EAE70123AB405361074ABB00EC
:10CC6000D819810008461144C968024491602A46D7
:10CC700000212046044B9847E8E700BF900E0020B3
:10CC80000040044011C9400081C840002DE9F04136
:10CC90008CB00124ADE12046B34B98470120FAE166
:10CCA000BB003B449900B14A0A44537CC3F3810161
:10CCB000033161F383035374537C13F0200F00F0AE
:10CCC000848013F00C0F3BD0A94A04F10C0152F8F8
:10CCD00021300193019B43F04F030193019B43F0EB
:10CCE00010030193019B42F8213000238DF801309D
:10CCF00006E000BF9DF801300133DBB28DF8013052
:10CD00009DF80130DBB2132BF3D9994A06F10C01DF
:10CD100052F821300293029B43F04F030293029B8F
:10CD200023F001030293029B42F8213006F10C0329
:10CD30008F4A52F8233013F0010FF7D10120AAE1F6
:10CD40008B4A04F10C0152F821300393039B43F00A
:10CD50004F030393039B23F001030393039B42F8C8
:10CD6000213006F10C03824A52F8233013F0010FF0
:10CD7000F7D1114606F10C0352F823200492049ACD
:10CD800042F04F020492049A42F020020492049A64
:10CD900041F8232000238DF8023006E000BF9DF803
:10CDA00002300133DBB28DF802309DF80230DBB285
:10CDB000132BF3D907EB8707BA006C4B13445A7C4B
:10CDC0006FF345125A74012065E113F0800F42D1D0
:10CDD000BB003B449A00654B1344DA689B689A4257
:10CDE0004CD307EB87039A00604B13445B7C13F032
:10CDF0004C0F43D1EFF31083B3FA83F35B090B932A
:10CE000072B6BFF35F8F00225A4B1A700B9B584AC1
:10CE100055612BB10122574B1A70BFF35F8F62B679
:10CE2000534A06F10C0152F821300593059B43F05B
:10CE30004F030593059B23F001030593059B42F8DF
:10CE4000213006F10C034A4A52F8233013F0010F47
:10CE5000F7D101201FE1BB003B449A00434B134430
:10CE6000597C6FF3C7115974DA689A60404B5D6161
:10CE7000224600214046404B9847A9E7002C4AD063
:10CE8000032C48D007EB87039A00384B13445B7C94
:10CE900013F00C0F3FD0364A06F10C0152F8213046
:10CEA0000693069B43F04F030693069B43F0100343
:10CEB0000693069B42F8213000238DF8033006E0EC
:10CEC00000BF9DF803300133DBB28DF803309DF8CD
:10CED0000330DBB2132BF3D9254A06F10C0152F8CB
:10CEE00021300793079B43F04F030793079B23F0E1
:10CEF00001030793079B42F8213006F10C031C4AFB
:10CF000052F8233013F0010FF7D1002120461B4BBC
:10CF100098470120BFE0002C4AD0032C48D00121C3
:10CF20002046164B984758B3114A06F10C0152F8A7
:10CF300021300893089B43F04F030893089B23F08C
:10CF400001030893089B42F8213006F10C03084ABC
:10CF500052F8233013F0010FF7D100212046074B80
:10CF60009847012097E000BFC1CB4000900E002001
:10CF7000004004402F03002081C84000CDCA40007B
:10CF80004749BB00D81982000A4492F811E06FF3B8
:10CF9000C71E82F811E0D2681F44BB0019448A60A2
:10CFA000404B5D612246002140463F4B9847BBE71E
:10CFB000012120463D4B98473A4A06F10C0152F8B0
:10CFC00021300993099B43F04F030993099B23F0F8
:10CFD00001030993099B42F8213006F10C03314A01
:10CFE00052F8233013F0010FF7D1012053E0013440
:10CFF000E4B2052C4ED82B4B9B6926460125A54053
:10D000002B42F4D0671E07EB87029300244A02EB01
:10D01000030804F10C03234A52F8233013F0420FA3
:10D020007FF439AE04F10C031E4A52F8233013F09A
:10D03000010F7FF435AE04F10C031A4A52F8233085
:10D0400013F0080FD3D004F10C0152F821300A93E9
:10D050000A9B43F04F030A930A9B23F008030A93A9
:10D060000A9B42F8213006F10C030E4A52F8233095
:10D0700013F0080FF7D106F10C0352F8233003F434
:10D08000E063B3F5807F09D006F10C0352F823303A
:10D09000012000E000200CB0BDE8F0810120FAE79B
:10D0A000900E00200040044081C84000CDCA4000DE
:10D0B00000B587B0534B1B78E3B9534B1B6BC3F3DD
:10D0C0000A43082B3BD0504A136B0193019B43F05A
:10D0D0004F030193019B23F004030193019B13630E
:10D0E000494B1B6B13F0040FFAD1484B984707B01C
:10D0F0005DF804FB464B9847464B9847DDE7424AAC
:10D10000116D454A99540133DBB2072BF7D9434BD4
:10D110009847B0B93C4A136B0293029B43F04F030C
:10D120000293029B23F004030293029B1363364B8A
:10D130001B6B13F0040FFAD1344B9847D7E7002349
:10D14000E3E7354B93F90030002B1EDB2E4A136BBF
:10D150000593059B43F04F030593059B23F00403C0
:10D160000593059B1363284B1B6B13F0040FFAD137
:10D17000294BDB88002B42D00023294A1380294AFF
:10D18000138001221F4B1A70B1E71F4A136B0393E0
:10D19000039B43F04F030393039B43F080030393EC
:10D1A000039B136300238DF8033006E000BF9DF856
:10D1B00003300133DBB28DF803309DF80330DBB26E
:10D1C000132BF3D9104A136B0493049B43F04F03C2
:10D1D0000493049B23F004030493049B13630A4BFE
:10D1E0001B6B13F0040FFAD100230D4A13800D4A74
:10D1F00013800222034B1A700B4B984777E70B4BB7
:10D20000984774E78E0E002000400440F5C34000AC
:10D21000A1C44000DDC340002423002035C04000ED
:10D220008C0E00208A0E0020B1C4400045C440008E
:10D23000204BDB6913F0010F37D000B583B01D4BD5
:10D240001B6B13F0040F24D11A4B1B6B13F0010F4F
:10D2500023D1184B1B6B13F0020F22D1154B1B6B04
:10D2600013F0080F23D0134A136B0193019B43F073
:10D270004F030193019B23F008030193019B136368
:10D280000C4B1B6B13F0080FFAD1012003B05DF8B3
:10D2900004FB094B98470120F8E7084B9847012009
:10D2A000F4E7074B98470120F0E700207047002083
:10D2B000ECE700BF00400440B1D04000B1C44000E2
:10D2C00089C6400010B54C4B984720B94B4BDB69E1
:10D2D00013F4807F10D03020494B9847474B9B690F
:10D2E00013F4006F04D0454BDB6913F4006F0AD1CF
:10D2F000444B984770B110BD72B6BFF35F8F0022E8
:10D30000414B1A7010BD4FF400623C4B1A623F4B08
:10D31000984710BD3E4B98470028ECD1374B9B698E
:10D3200013F4005F04D0354BDB6913F4005F3DD18B
:10D33000324B9B6913F4007F04D0304BDB6913F44C
:10D34000007F33D12D4B9B6913F4806F04D02B4B9E
:10D35000DB6913F4806F29D1284B9B6913F4807F1C
:10D3600004D0264BDB6913F4807F2FD1234BDB697C
:10D3700013F4805FBFD0214C4FF480532362254BC0
:10D380009847254B9847636823F0010363606368FF
:10D3900023F002036360214B9847214B98474FF4D9
:10D3A000807323614FF400632361A4E7134C4FF4AF
:10D3B00018532362636101201A4B98474FF480731E
:10D3C000236223614FF40063236110BD0B4B4FF4C4
:10D3D00080721A625A614FF400521A614FF400725F
:10D3E0001A614FF480621A6130200F4B9847002079
:10D3F0000C4B984710BD00BF65E44000004004405E
:10D400002DE3400031D240002F030020FDBF40003B
:10D410008DCC4000C1C8400011BE400029C340006F
:10D42000DDC3400085C2400081E3400010B582B0FA
:10D43000EFF31083B3FA83F35B09019372B6BFF382
:10D440005F8F0022144B1A70019C0120134B9847E8
:10D450003020134B9847134B5A6F22F480725A674F
:10D460005A6F42F400725A674FF480721A614FF497
:10D4700000521A614FF400721A614FF480621A610F
:10D480004FF400621A612CB10122034B1A70BFF3F2
:10D490005F8F62B602B010BD2F03002085C240002E
:10D4A0002DE340000040044030B583B0EFF310831B
:10D4B000B3FA83F35B09009372B6BFF35F8F002466
:10D4C000204B1C70009D204B984730201F4B9847E5
:10D4D0001F4B98471F4B502283F830234FF4803264
:10D4E0005A601D4B98474FF480201C4B98471C4BAB
:10D4F0001C701C4B1B78FF2B22D0EFF31083B3FA68
:10D5000083F35B09019372B6BFF35F8F00220D4B6B
:10D510001A700199134A13780133137029B101224B
:10D52000084B1A70BFF35F8F62B60F4B98472DB14F
:10D530000122044B1A70BFF35F8F62B603B030BD97
:10D54000FEE700BF2F03002031DD40002DE3400047
:10D5500019DF400000E100E049C8400051E440000C
:10D56000890E00203C2300202DD4400008B5064B36
:10D570005A6F42F480725A675A6F22F400725A67E7
:10D580000020024B984708BD0040044085C240007F
:10D5900010B582B0EFF31083B3FA83F35B09009305
:10D5A00072B6BFF35F8F0022144B1A70009C144BAD
:10D5B0009847144B1B7803B9FEE7EFF31083B3FAD7
:10D5C00083F35B09019372B6BFF35F8F00220B4BAD
:10D5D0001A7001990B4A1378013B137029B101228B
:10D5E000064B1A70BFF35F8F62B62CB10122034B5A
:10D5F0001A70BFF35F8F62B602B010BD2F03002018
:10D600006DD540003C2300200D4B5A6822F00102EA
:10D610005A609A6822F480729A60024670B19868E3
:10D6200020F07F0002F07F02104398609A6842F475
:10D6300080729A605A6842F001025A60704700BFD7
:10D6400000400440054B5B6813F0010F04D0034B0E
:10D65000986800F07F007047002070470040044049
:10D66000014B98609981704724230020F0B583B066
:10D6700045B200F00F00052873D801F003060446F8
:10D6800000F10C033B4F57F8233013F4004F6BD1DC
:10D69000012E53D0031FDBB2012B54D940239342F8
:10D6A00066DB461E06EB8607334B03EB870303F16D
:10D6B0001007B3F810E062F3090EA3F810E05B7CEA
:10D6C00003F07F036FF345137B70002D3EDB294E83
:10D6D000B36A012282401343B362264B9B6A1A420B
:10D6E000FBD0244B9E6A26EA02029A6200F10C02E9
:10D6F00053F822300193019B43F04F030193019BA8
:10D7000023F4074323F080030193002D23DB0A0257
:10D7100002F4407242F40042019B134301930199C9
:10D720000C30144B43F8201004F10C03114951F84C
:10D73000233032EA0303F7D1012013E0B0B103280C
:10D74000A8D100200EE04FF40073A8E77B786FF3B8
:10D7500083037B70BBE70A0202F4407242F4044286
:10D76000DAE7002003B0F0BD0020FBE70020F9E776
:10D770000020F7E700400440900E002000F00F0367
:10D78000052B1ED810B582B019460E4C0C3354F838
:10D7900023200192019A42F04F020192019A22F451
:10D7A00000420192019A44F8232001F10C03054A3A
:10D7B00052F8233013F4004FF7D1034B984702B0CF
:10D7C00010BD704700400440EDC8400000F00F005D
:10D7D000431E052815D803EB83039A000A4B134414
:10D7E0005B7C13F0200F08D10C30084B53F820302D
:10D7F00013F0280F03D0012070470120704700204C
:10D8000070470020704700BF900E00200040044089
:10D8100010B485B044B200F00F00052865D8421E50
:10D82000EFF31083B3FA83F35B09039372B6BFF38C
:10D830005F8F0021314B19700399002C14DB304AA3
:10D8400000F10C0452F824300293029B43F04F0382
:10D850000293029B43F020030293029B42F8243080
:10D8600000238DF807302EE000F10C03244C54F80F
:10D87000233013F0100F09D102EB82039C00214BDF
:10D8800023445B7CC3F38103012BD8DD02EB8202CE
:10D8900094001C4B23445A7C42F020025A7401230A
:10D8A00003FA00F0164B186121B30120134B1870D6
:10D8B000BFF35F8F62B619E000BF9DF807300133F8
:10D8C000DBB28DF807309DF80730DBB2132BF3D9AC
:10D8D000012303FA00F00A4B186169B10120074BDC
:10D8E0001870BFF35F8F62B600E0002005B05DF8EE
:10D8F000044B70470120F9E70120F7E72F030020D0
:10D9000000400440900E002000F00F0005286CD865
:10D9100030B583B00246441E04EB84039900354BB6
:10D920000B44597C6FF34511597400F10C033249D3
:10D9300051F8233013F0200F59D000F10C0551F8A5
:10D9400025300093009B43F04F030093009B23F08E
:10D9500020030093009B41F8253002F10C03264977
:10D9600051F8233013F0200FF7D10D468B6A0121B7
:10D9700081400B43AB62204B9B6A1942FBD01E4B8C
:10D980009D6A25EA010199620C3053F8201001913B
:10D99000019941F04F010191019921F00801019194
:10D9A000019943F8201002F10C03134951F8233078
:10D9B00013F0080FF7D104EB84039A000D4B1344C6
:10D9C0005B7C13F0100F01D1012011E00949A20086
:10D9D000101983000B44587C6FF3041058741444DE
:10D9E000A300CB589847012002E000207047012097
:10D9F00003B030BD900E002000400440F0B583B06D
:10DA000000F00F04052C00F2A28047B2651E04F15D
:10DA10000C00554E56F8200010F4004F00F09A808C
:10DA200005EB8500514E06EB8000407C10F0200F86
:10DA300040F0928004F10C004B4E56F8200010F09C
:10DA4000200F40F08B80EFF31080B0FA80F0400997
:10DA5000009072B6BFF35F8F002645480670DDF870
:10DA600000E005EB8500414E06EB8000407C10F0A5
:10DA7000100F0AD0BEF1000F72D001223C4B1A7079
:10DA8000BFF35F8F62B6002062E005EB8500374E82
:10DA900006EB8000467C46F010064674BEF1000F8F
:10DAA00005D0012632480670BFF35F8F62B6DFF8FB
:10DAB000BCE005EB850080000EEB00067260B360F1
:10DAC0000022F260089A4EF8002011B95BBB0120D9
:10DAD00000E00120254AA9004B1902EB83035B7C7F
:10DAE00060F386130D4402EB85026FF3C713537482
:10DAF000EFF31083B3FA83F35B09019372B6BFF3BC
:10DB00005F8F00221A4B1A70019D0123A340164A11
:10DB10001361002F09DB2DB30120154B1870BFF3E3
:10DB20005F8F62B614E00020D4E704F10C0352F8D2
:10DB3000233013F0110FEED1012120460D4B9847F1
:10DB40000028E8D0002120460A4B9847E3E7002050
:10DB500003B0F0BD0020FBE70020F9E70020F7E765
:10DB60000020F5E70120F3E700400440900E00207C
:10DB70002F030020CDCA400070B586B000F00F041E
:10DB8000052C00F2C98042B2EFF31083B3FA83F39D
:10DB90005B09059372B6BFF35F8F00215F4B19706D
:10DBA000059B26460125A5405D494D612BB101210C
:10DBB0005A4B1970BFF35F8F62B6002A80F29480CF
:10DBC00004F10C03564A52F8233013F0100F64D0BE
:10DBD000002C49D0032C47D004F10C0152F821301D
:10DBE0000193019B43F04F030193019B23F010032A
:10DBF0000193019B42F8213006F10C03484A52F888
:10DC0000233013F0100FF7D106F10C03444A52F8F9
:10DC1000233013F0100FF7D104F10C0152F821302A
:10DC20000293029B43F04F030293029B43F01003C5
:10DC30000293029B42F8213000238DF8033006E066
:10DC400000BF9DF803300133DBB28DF803309DF83F
:10DC50000330DBB2132BF3D906F10C03304A52F830
:10DC6000233013F0100FF7D02D4A04F10C0152F8B5
:10DC700021300393039B43F04F030393039B23F053
:10DC800010030393039B42F8213006F10C03244A4E
:10DC900052F8233013F0100FF7D1214A04F10C0190
:10DCA00052F821300493049B43F04F030493049BE8
:10DCB00023F001030493049B42F8213006F10C0386
:10DCC000174A52F8233013F0010FF7D1621E02EB0E
:10DCD00082029100134B0B445A7C6FF383025A74F7
:10DCE0000AE02046104B984706F10C030C4A52F804
:10DCF000233013F0420FF4D1094A936A2B43936205
:10DD0000074B9B6A1D42FBD0054A936A23EA05052F
:10DD100095622046054B984706B070BD2F03002042
:10DD200000400440900E002011C94000EDC84000A2
:10DD3000064BD3F8142122F44062C3F81421D3F81F
:10DD4000202142F00102C3F82021704700020E405A
:10DD50000B4619B1096801605B6843601AB113682A
:10DD6000036153684361704721F0FE01C905C90D85
:10DD70000162704710B51E4B53F820402268536A69
:10DD800013F0805F11D00223C2F8203123684FF0D6
:10DD9000FF32DA6100232375236913F0010F26D0C7
:10DDA000636823B32046984710BD13F0006F13D06B
:10DDB0000223C2F8203123684FF00062DA61236940
:10DDC00013F0020F03D0A3680BB1204698472368D5
:10DDD0000122C3F8202110BD13F0007F07D0236972
:10DDE00013F0040F03D0E3680BB12046984710BD31
:10DDF000F40E002008B50020014B984708BD00BF75
:10DE000075DD400008B50120014B984708BD00BFF3
:10DE100075DD400070B505460E46144601600123CD
:10DE20000B60214B99422BD00D20204B9847204B63
:10DE30001D6023781B0203F4FE43736063782BBBE1
:10DE40000022A3780BB142F00402E3780BB142F058
:10DE5000080223790BB142F0100263791B0203F42C
:10DE60007063A179090389B20B431343B365238916
:10DE7000C3F30E03628943EA0243F36500230CE017
:10DE800012200A4B98470A4B5D60D2E70222D8E77E
:10DE900005EB8302002151600133022BF8D90020E9
:10DEA0002861287570BD00BF000003402DE34000CD
:10DEB000F40E002012F0100F12D0C0F8B01012F0C3
:10DEC000200F07D0C0F8D41012F0400F05D0C0F8D2
:10DED000C0107047C0F8D010F6E7C0F8C410704703
:10DEE000C0F8B41070470164704741647047C06C5B
:10DEF0007047806C7047400900F5001000F2077011
:10DF00004002704740090B30704700F01F000123AA
:10DF100003FA00F07047000008B500200A4B98474C
:10DF20000A4B98470028FBD0094B9847094A0A4BEF
:10DF3000DA620A4B98470028FBD00020084B98472C
:10DF4000084B984708BD00BFA9E24000CDE2400061
:10DF500011E34000013FB80500040E401DE34000FE
:10DF600031E4400045E4400010B5A2B01848194B18
:10DF700098470020184B9847184B98470028FBD02B
:10DF8000174B9847174A184B9A62184B9847002826
:10DF9000FBD00020164B9847164B984716480D4B60
:10DFA0009847164B1A68164B1344164A934201D9E8
:10DFB00022B010BD2023009302AB0F220E21124885
:10DFC000124CA047BDF848101148124B9847EFE794
:10DFD000000E2707B5E74000A9E24000CDE240006F
:10DFE000F5E24000013FB70B00040E4001E34000A2
:10DFF00055E24000C1E640000000DC05300300208F
:10E00000C0D3BDF980C3C901000A0E401100002031
:10E0100010140E4075E4400070B50D4614460646D7
:10E0200058B14FF0FF360AE0064B1868064B1B68E4
:10E030002946984701350136013C002CF4DC304676
:10E0400070BD00BF4C2300204423002070B5013870
:10E0500002280FD8144600258CB10A4B18684E1CB4
:10E06000094B1B6809789847002806DB0135013CFD
:10E070003146F1E74FF0FF3501E04FF0FF3528461C
:10E0800070BD00BF4C23002048230020A1F10E03E7
:10E09000012B02D84FF0FF30704710B582B0EFF37C
:10E0A0001083B3FA83F35B09019372B6BFF35F8FFA
:10E0B00000240B4B1C70019C120222F07F4222F0C4
:10E0C000FF02C9B2114341F0B441064B98472CB14D
:10E0D0000122034B1A70BFF35F8F62B602B010BD0E
:10E0E0002F030020790000204C4B1B78FF2B31D0F0
:10E0F00000B583B0EFF31083B3FA83F35B090193A8
:10E1000072B6BFF35F8F0022454B1A700199434AE4
:10E1100013780133137029B10122414B1A70BFF3F8
:10E120005F8F62B63F4A904215D03F4A904220D05E
:10E130003E4A90422BD03E4A904236D03D4A9042D1
:10E1400041D03D4A90424CD03C4A904257D003B017
:10E150005DF804FBFEE71620394B98470720394B42
:10E16000984700210720384B98470720374B98479E
:10E17000EDE71520324B98470720324B9847002196
:10E180000720314B98470720304B9847DFE7142092
:10E190002B4B984707202B4B9847002107202A4BF1
:10E1A00098470720294B9847D1E71320244B9847DD
:10E1B0000620244B984700210620234B9847062031
:10E1C000224B9847C3E70E201D4B984706201D4B56
:10E1D0009847002106201C4B984706201B4B984768
:10E1E000B5E70920164B98470620164B98470021A3
:10E1F0000620154B98470620144B9847A7E70820A0
:10E200000F4B984706200F4B9847002106200E4BD6
:10E21000984706200D4B984799E700BF3C23002004
:10E220002F030020000004400080004000C0014097
:10E2300000800140004002400000024000C0004059
:10E240002DE340001DE44000D5E3400009E4400018
:10E2500001607047134A136B23F070031843106377
:10E260004FF400630F4A926E12F0080F02D1A3B16F
:10E27000013BF7E70B4A136B23F0030343F0020360
:10E2800013634FF40063074A926E12F0080F02D135
:10E290002BB1013BF7E700207047012070470120B8
:10E2A000704700BF00040E40012803D0054A064B0A
:10E2B0001A607047044A936843F0254343F480137F
:10E2C0009360F3E7080000A510140E40074B5B694C
:10E2D00013F0800F06D0064B9B6E13F0800F03D116
:10E2E00000207047002070470120704710140E4036
:10E2F00000040E400022014B9A62704700040E4059
:10E30000024B986E00F00200704700BF00040E4000
:10E310000022014BDA62704700040E40024B986EF7
:10E3200000F00400704700BF00040E4032281ED8E1
:10E330001F280CD8114B9A6901238340934318D0AE
:10E34000012303FA00F00D4B1861002070472038BC
:10E350000A4BD3F808210123834093430BD00123B8
:10E3600003FA00F0054BC3F80001002070470120BC
:10E370007047002070470020704700BF00040E4027
:10E38000322822D81F280ED8114B9A6901238340C6
:10E39000934301D000207047012303FA00F00C4B97
:10E3A0005861002070472038094BD3F80821012319
:10E3B0008340934301D000207047012303FA00F00B
:10E3C000034BC3F80401002070470120704700BFD1
:10E3D00000040E4041F0040100F11002094B43F823
:10E3E00022104FF40062074B996E4FF48073834004
:10E3F000194202D11AB1013AF5E700207047012015
:10E40000704700BF00040E404FF4807303FA00F021
:10E41000014B1860704700BF00040E404FF480733A
:10E4200003FA00F0014B5860704700BF00040E4033
:10E43000000200F4706040F00100014B98637047E7
:10E4400000040E408022014B1A60704700040E4009
:10E45000C0F31200024B1A6F10431867704700BFD9
:10E4600000040E40024B187880F00100704700BF96
:10E47000FC0E0020C36923F4F053490201F4F0516B
:10E48000194341F0B44141F48071C161704730B427
:10E49000B2EB011F17D3102401FB04F14B0803EB6F
:10E4A000C202B2FBF1F2D3085D1E4FF6FE718D423F
:10E4B00010D8082C09D0120402F4E0221A43026298
:10E4C000002030BC70470824E6E7416841F4002191
:10E4D0004160F0E70120F4E74023036070478823A0
:10E4E0000360704710230360704724230360704764
:10E4F0004FF48073036070474FF40023036070474C
:10E50000436913F0020F04D0C1F30801C161002078
:10E51000704701207047436913F0020FFBD0C1F32D
:10E520000801C16100207047436913F0010F05D055
:10E530008369C3F308030B60002070470120704714
:10E54000014BC0F8E43070470041535510B5044604
:10E55000094B9847002363606362A3622046074B20
:10E5600098472046064B98472046064B984720463A
:10E57000054B984710BD00BF41E54000DFE4400077
:10E58000EBE44000F1E44000F9E4400070B50546DA
:10E590000C461646104B98470022104B1A60B4B137
:10E5A0003246216828460E4B9847024688B9636870
:10E5B000A1680B4321690B43E1680B4307490868D5
:10E5C00003430B6069680B436B60104670BD01220A
:10E5D000FBE70122F9E700BF4DE54000000F0020F6
:10E5E0008FE4400000B583B0234B244A9A4209D0FF
:10E5F000214B224A03E01168196004330432204998
:10E600008B42F8D31F4B02E000221A6004331E4AEB
:10E610009342F9D31D4A22F07F011D4B9960EFF31D
:10E620001083B3FA83F35B09019372B6BFF35F8F74
:10E630000021184B1970019817490B6843F47003B7
:10E640000B60BFF34F8FBFF36F8F28B10121114BC8
:10E650001970BFF35F8F62B602F16042B2F5203FDE
:10E6600004D20B4A936843F0005393600B4B9847D6
:10E670000B4B9847FEE700BF10000020BC5941003B
:10E68000E80C0020E80C002030240020004040006E
:10E6900000ED00E02F03002088ED00E0D9194100D3
:10E6A0004D09410008B50120034B9847EFF3058061
:10E6B000024B9847FFDE00BF854D4000914D400062
:10E6C000344B1B6B03F00303012B20D083B1022BCF
:10E6D00039D0304B1B6B03F07003702B51D02D4B96
:10E6E0001A6BC2F302122C490B68D3400B607047BF
:10E6F0002A4B5B6913F0800F04D04FF40042264B85
:10E700001A60E6E74FF4FA42234B1A60E1E7214B27
:10E710001B6A13F0807F03D0214A1F4B1A60D8E791
:10E72000204A1D4B1A601B4B1B6A03F07003102B11
:10E7300005D0202BCDD11C4A174B1A60C9E71B4AC4
:10E74000154B1A60C5E7154B5B6913F0800F13D0AA
:10E750004FF40042104B1A600E4B1B6B03F0030387
:10E76000022BB6D10B4B9A6AC2F30C420A490B68D2
:10E7700002FB03330B60ACE74FF4FA42064B1A601E
:10E78000EAE7054A13680A49A1FB03135B08136013
:10E79000704700BF00040E403003002010140E40EC
:10E7A000001BB70000127A0000366E010024F4004E
:10E7B000ABAAAAAA144B98420FD9144B984211D96C
:10E7C000134B984212D9134B984213D9124B9842CB
:10E7D00014D9124A124B1A6070474FF08062104BE6
:10E7E0001A6070470F4A0E4B1A6070470E4A0C4B66
:10E7F0001A6070470D4A0A4B1A6070474FF00422A6
:10E80000074B1A60704700BFFF2C3101FF596202AD
:10E81000FF869303FFB3C404FFE0F5050005000481
:10E82000000A0E400001000400020004000300047E
:10E830000A4B1B6853B1094B1B681A1808499142CF
:10E8400008DB1046054A106018467047054A034B1E
:10E850001A60F0E74FF0FF30704700BF040F002050
:10E86000FC7F0220305400204FF0FF3070474FF4FF
:10E8700000534B6000207047012070470020704714
:10E8800000F1080343604FF0FF328260C360036110
:10E8900000230360704700230361704743684B60A7
:10E8A0009A688A609A6851609960086103680133C8
:10E8B0000360704730B40D68B5F1FF3F02D000F13E
:10E8C000080202E0026904E01A4653681C68A54287
:10E8D000FAD253684B6099608A605160086103689E
:10E8E0000133036030BC70470369426881689160FE
:10E8F0008268416851605A68904206D000220261E5
:10E900001A68013A1A601868704782685A60F5E719
:10E9100082B0002301934FF0500383F31188BFF3BB
:10E920006F8FBFF34F8F019B002BFCD002B070475D
:10E9300008480068006880F308884FF0000080F302
:10E94000148862B661B6BFF34F8FBFF36F8F00DFDD
:10E9500000BF000008ED00E0DFF80C00016841F4A2
:10E96000700101607047000088ED00E04FF0807397
:10E9700040F8043C21F0010140F8081C054B40F828
:10E980000C3C40F8202C6FF0020340F8243C443843
:10E99000704700BF11E940000000000000000000C7
:10E9A000074B19680868B0E8F04F80F30988BFF397
:10E9B0006F8F4FF0000080F311887047AFF3008035
:10E9C000080F00204FF0500383F31188BFF36F8FBF
:10E9D000BFF34F8F024A136801331360704700BFC3
:10E9E00034030020034A1368013B13600BB983F31F
:10E9F0001188704734030020000000000000000070
:10EA0000EFF30980BFF36F8F154B1A681EF0100FDC
:10EA100008BF20ED108A20E9F04F10602DE90900B1
:10EA20004FF0500080F31188BFF34F8FBFF36F8F0B
:10EA300000F07CFF4FF0000080F3118809BC1968DA
:10EA40000868B0E8F04F1EF0100F08BFB0EC108A55
:10EA500080F30988BFF36F8F704700BFAFF300806A
:10EA6000080F002008B54FF0500383F31188BFF35F
:10EA70006F8FBFF34F8F054B984718B14FF08052FF
:10EA8000034B1A60002383F3118808BDA9F64000E8
:10EA900004ED00E0054B00221A6005490A600549B3
:10EAA000054A116007221A60704700BF10E000E0BD
:10EAB00018E000E0FF7F010014E000E010B50E4B0D
:10EAC0001A6842F470021A601A6842F070421A60C2
:10EAD0000A4B984700240A4B1C600A4B98470A4A85
:10EAE000136843F040431360084B9847084B98471E
:10EAF000084B9847204610BD20ED00E095EA400005
:10EB00003403002059E9400034EF00E031E94000CF
:10EB10002DF9400011E9400010B50446044B984718
:10EB20002046044B98470446034B9847204610BDA7
:10EB30008DF64000511A41009DF7400048B110B5D4
:10EB40000446044B98472046034B9847034B98478D
:10EB500010BD70478DF64000611A41009DF74000DE
:10EB6000436A23B1036B1868C0F1050070470020A9
:10EB70007047000010B50446064B9847A26BE36B44
:10EB80009A4204D00024044B9847204610BD01242B
:10EB9000F9E700BFC5E94000E5E9400010B50446CB
:10EBA000054B9847A36B23B10024044B984720469C
:10EBB00010BD0124F9E700BFC5E94000E5E94000C8
:10EBC00070B504461646856B026C5AB903681BB1D2
:10EBD00000200135A56370BD4068174B984700239E
:10EBE0006360F6E76EB98068144B9847226CA3689F
:10EBF0001344A3606268934219D32368A360002082
:10EC0000E7E7C0680D4B9847226C5242E368134413
:10EC1000E36021688B4202D263681A44E260022EEC
:10EC200001D00020D5E725B1013D0020D1E700202B
:10EC3000CFE70020CDE700BF3DFC4000D1204100E0
:10EC4000026C72B110B5C3681344C3604468A34238
:10EC500001D30368C3600C46C1682046014B984746
:10EC600010BD7047D120410038B505461A4B984772
:10EC700095F8454064B201E0013C64B2002C0ADD25
:10EC80006B6A43B105F12400144B98470028F3D078
:10EC9000134B9847F0E7FF2385F84530114B984711
:10ECA0000D4B984795F8444064B201E0013C64B2D2
:10ECB000002C0ADD2B6943B105F11000074B984782
:10ECC0000028F3D0064B9847F0E7FF2385F844303F
:10ECD000044B984738BD00BFC5E9400031FA4000F9
:10ECE0002DFB4000E5E9400038B504460D46144BC5
:10ECF00098472168E26B236C03FB021060600020E0
:10ED0000A063A160013A02FB0313E360FF2384F8D0
:10ED1000443084F8453055B923691BB9094B9847ED
:10ED2000012038BD04F11000074B9847F6E704F1C5
:10ED30001000064DA84704F12400A847EEE700BFE5
:10ED4000C5E94000E5E9400031FA400081E84000B3
:10ED500038B51D46049C0B4649B12260E06323642C
:10ED600001212046034B984784F84C5038BD24605D
:10ED7000F4E700BFE9EC4000F0B583B00546174664
:10ED80000E4689B100FB01F05030084B984704460D
:10ED900038B100903B4600F1500231462846044D00
:10EDA000A847204603B0F0BD0020EDE719EB400076
:10EDB00051ED4000F0B585B004460F4601921E4665
:10EDC000002526E0324639462046354B9847636A8F
:10EDD00023B9344B9847012005B0F0BD04F124005D
:10EDE000314B9847F5E72F4B98470020F4E702A8EE
:10EDF0002E4B9847012519E0002384F8443021E088
:10EE0000002384F8453023E02046294B9847294BBE
:10EE10009847294B9847A26BE36B9A42D2D3022EB4
:10EE2000D0D0019B002BDED0002DE0D01D4B9847A9
:10EE3000224B9847204B984794F844305BB2B3F18B
:10EE4000FF3FD9D094F845305BB2B3F1FF3FD7D044
:10EE5000144B984701A902A8194B9847C8B92046F6
:10EE6000184B98470028CFD0019904F11000164B99
:10EE7000984720460E4B98470E4B98470028C8D11C
:10EE80004FF08052114B1A60BFF34F8FBFF36F8F5B
:10EE9000BFE72046064B9847064B984700209BE764
:10EEA000C1EB4000E5E9400031FA4000B1FA400012
:10EEB00069EC40009DF74000C5E940008DF6400038
:10EEC000C9FA400075EB4000E1F9400004ED00E0B4
:10EED00048B110B5002141600160C1600B460A468F
:10EEE000014CA04710BD7047B5ED400010B502467B
:10EEF00000210120034B98470446034B98472046C6
:10EF000010BD00BF79ED4000D1EE4000F8B5EFF341
:10EF100011864FF0500484F31188BFF36F8FBFF355
:10EF20004F8F856BC46BA54205D3022B03D0002005
:10EF300086F31188F8BD1746054690F8454064B23F
:10EF40001A460E4B9847B4F1FF3F05D0013464B226
:10EF500085F845400120EBE76B6A0BB90120E7E734
:10EF600005F12400064B984718B127B101203860FD
:10EF7000DEE70120DCE70120DAE700BFC1EB40005B
:10EF800031FA4000F0B585B004460F4601920026E4
:10EF900032E039462046384B9847013DA563236946
:10EFA00023B9364B9847012005B0F0BD04F110009D
:10EFB000334B9847F5E7314B98470020F4E702A818
:10EFC000304B9847012621E0002384F8443029E0A3
:10EFD000002384F845302BE020462B4B98472B4BE1
:10EFE000984709E02046284B9847284B98472046E9
:10EFF000274B984700283DD1264B9847A56B002DFD
:10F00000C7D1019B002BD6D0002ED8D01B4B9847E0
:10F01000214B98471F4B984794F844305BB2B3F1AB
:10F02000FF3FD1D094F845305BB2B3F1FF3FCFD072
:10F03000124B984701A902A8184B98470028D1D134
:10F040002046134B98470028C6D0019904F12400AC
:10F05000134B984720460C4B98470C4B9847002879
:10F06000CAD14FF080520F4B1A60BFF34F8FBFF3DE
:10F070006F8FC1E7002097E741EC4000E5E94000D1
:10F0800031FA4000B1FA400069EC40009DF74000C1
:10F090009DEB4000C5E940008DF64000C9FA4000F4
:10F0A000E1F9400004ED00E070B584B00446019140
:10F0B000002635463EE0013BA36323683BB123694C
:10F0C0004BB9444B98470126304604B070BD424BC3
:10F0D00098476060F3E704F11000404B9847F0E771
:10F0E0003C4B98470026EFE702A83D4B9847012587
:10F0F0002AE0002384F8443032E0002384F84530CD
:10F1000034E0384B98476068374B98470646314B98
:10F1100098473BE02046354B9847354B984709E0E8
:10F120002046324B9847324B98472046314B984700
:10F13000002840D12B4B9847A36B002BBBD1019BE0
:10F14000002BCDD0002DCFD0224B98472A4B98478B
:10F15000244B984794F844305BB2B3F1FF3FC8D0DA
:10F1600094F845305BB2B3F1FF3FC6D0194B9847D6
:10F1700001A902A8214B98470028D1D120461D4B58
:10F1800098470028C6D02368002BBAD0019904F113
:10F1900024001B4B98472046144B9847144B984724
:10F1A0000028C7D14FF08052164B1A60BFF34F8F23
:10F1B000BFF36F8FBEE7002E86D00A4B98472046DC
:10F1C000114B984701466068104B9847014B984790
:10F1D000002679E7E5E9400065FD400031FA40008E
:10F1E000B1FA4000C5E9400075FB400069EC400001
:10F1F0009DF740009DEB40008DF64000C9FA4000AD
:10F20000E1F9400004ED00E061EB4000C5FC400086
:10F210000023092B0CD8074A52F833200AB10133D6
:10F22000F7E7044A42F8331002EBC3035860704713
:10F23000704700BF5023002070B504460D461646A7
:10F24000124B984794F844305BB2B3F1FF3F0DD0B6
:10F2500094F845305BB2B3F1FF3F0BD00C4B9847AD
:10F26000A36B5BB120460B4B984770BD002384F81D
:10F270004430EDE7002384F84530EFE73246294675
:10F2800004F12400044B9847ECE700BFC5E94000B7
:10F29000E5E9400069EC400005FA4000F0B503687C
:10F2A0004BB343685B68436000F10807BB4204D07E
:10F2B0004368D3F80CE0002609E05B684360F7E799
:10F2C0005B68436008E02E46B6B9AE4514D043688B
:10F2D0005B6843609F42F3D04368DD6800230F2BD7
:10F2E000F2D8EA1892F83420CC5CA242ECD1002A81
:10F2F000E9D00133F3E700263046F0BD002301E0FA
:10F30000013001330278A52AFAD0C3F38F00704789
:10F310000A4B1B681B684BB901234BB9074B1B6891
:10F32000DB68DB685A68064B1A6070470023F4E715
:10F330004FF0FF32024B1A60704700BF0C0F0020E5
:10F34000B80F00202DE9F84F81460D4617469A4622
:10F350000A9EDDF82C800C9C9200A521206B1D4B91
:10F360009847236B07F18042013A03EB820727F0AD
:10F37000070700230F2B07D8E95CE21882F8341046
:10F38000EA5C0AB10133F5E7002384F84330042E28
:10F3900000D90426E662E66400252565201DDFF815
:10F3A0003CB0D84704F11800D8472461C6F10506DF
:10F3B000A6616462656584F85850524649463846ED
:10F3C000054B98472060B8F1000F01D0C8F8004005
:10F3D000BDE8F88FCD2241006DE9400097E840007C
:10F3E00070B5002407E004EB840293000B48184436
:10F3F0000B4B98470134042CF5D90A4E3046084C83
:10F40000A047094D2846A0470848A0470848A047FC
:10F41000084B1E60084B1D6070BD00BF140F00201C
:10F4200081E840008C0F0020A00F0020C00F0020BA
:10F43000D80F00200C0F0020100F002010B504463C
:10F440001C4B98471C4A1368013313601B4B1B6805
:10F45000002B26D01A4B1B683BB9184B1B68DA6A85
:10F46000E36A9A4201D8154B1C60164A13680133AF
:10F4700013606364E36A01229A40134908680243F7
:10F480000A6003EB83039A00211D10481044104BBF
:10F490009847104B98470A4B1B680BB1074B1B68EA
:10F4A00010BD064B1C601368012BDED10A4B984738
:10F4B000DBE700BFC5E94000780F0020080F0020FF
:10F4C000D40F0020840F0020880F0020140F00208C
:10F4D0009DE84000E5E94000E1F3400070B50446D6
:10F4E0000E461D4B1D681D4B186804301C4B984779
:10F4F00050B91A4B1B68DA6A012303FA02F2194960
:10F500000B6823EA02030B60B4F1FF3F13D02C44D5
:10F51000124B1B685C60A54216D8134B18680F4B42
:10F5200019680431114B9847114B1B689C4201D25A
:10F530000F4B1C6070BD002EE9D0084B19680431D8
:10F540000C480D4B984770BD0C4B1868034B19685D
:10F550000431064B984770BDEC0F0020080F0020C7
:10F56000E9E84000880F00200C0F0020B5E84000BB
:10F57000B80F0020D80F00209DE84000100F002099
:10F5800008B54FF08052044B1A60BFF34F8FBFF3A2
:10F590006F8F024B9847F4E704ED00E085084100C7
:10F5A0002DE9F04385B006460F4615469846900073
:10F5B000144B984700B381465C20124B9847044691
:10F5C000B0B1C0F83090CCB10023039302940D9BEE
:10F5D00001930C9B009343462A46394630460A4D18
:10F5E000A8472046094B9847012005B0BDE8F083A5
:10F5F0004846074B9847E6E70024E4E74FF0FF3022
:10F60000F3E700BF19EB400045F340003DF4400034
:10F610003DEB400010B582B0134B019300230093E3
:10F62000462212491248134CA047012803D0012852
:10F6300004D002B010BD104B9847F8E74FF05003CC
:10F6400083F31188BFF36F8FBFF34F8F4FF0FF32FB
:10F650000A4B1A6001220A4B1A600022094B1A60F9
:10F66000094B9847E5E700BFB40F00202C57410035
:10F6700081F54000A1F54000F9014100B80F0020DC
:10F68000D40F0020EC0F0020BDEA4000024A1368AE
:10F6900001331360704700BF800F0020014B1868D2
:10F6A000704700BFEC0F002070B52F4B1B68002B7C
:10F6B00052D12E4B1E6801361E604EB12C4B1B687A
:10F6C0009E422FD22B4B1B68002B42D0002070BDD6
:10F6D000294A1168294B186810601960284A136874
:10F6E00001331360274B9847E8E7012320E04FF0F0
:10F6F000FF321F4B1A60E5E71D4A1360E2E704F191
:10F700001800214B9847E36A01229A401F49086874
:10F7100002430A6003EB83039A0029461C48104405
:10F720001C4B9847144B1B681B68002BDDD0002333
:10F73000002BDCD1104B1B68DB68DC6863689E42E1
:10F74000DAD3251D2846104B9847A36A002BD6D143
:10F75000D9E7114B9847B9E7064A1368013313609C
:10F760000D4B9847B2E700BF800F0020EC0F002040
:10F77000B80F00207C0F00200C0F0020100F00207D
:10F78000BC0F002011F34000E9E84000880F002082
:10F79000140F00209DE840004909410070B5274B37
:10F7A0009847274B1A68013A1A601B68002B32D120
:10F7B000244B1B68002B2ED00024234B1B6813B353
:10F7C000214BDB68DC6804F11800204EB047251D92
:10F7D0002846B047E36A01229A401D49086802435F
:10F7E0000A6003EB83039A0029461A4810441A4B17
:10F7F0009847E26A194B1B68DB6A9A42DDD3012203
:10F80000174B1A60D9E70CB1164B9847164B1C687A
:10F810003CB9134B1B68154B9847002070BD013C49
:10F8200007D0134B98470028F9D001220C4B1A60DF
:10F83000F5E700220C4B1A60EBE700BFC5E940007A
:10F84000800F0020780F0020C00F0020E9E8400062
:10F85000880F0020140F00209DE84000080F0020B2
:10F86000F00F002011F340007C0F0020E5E940007C
:10F87000A9F6400010B550B9002038B94FF08052B9
:10F88000084B1A60BFF34F8FBFF36F8F10BD044654
:10F89000054B984700212046044B9847044B984756
:10F8A000EBE700BF04ED00E08DF64000DDF4400022
:10F8B0009DF7400070B50646154B98470524013C5E
:10F8C00004EB84029300314612481844124B9847C7
:10F8D000054608B9002CF2D12DB15DB18DB10F4BA9
:10F8E0009847284670BD0E4B186831460A4B98471A
:10F8F0000546F2E70B4B18683146074B984705461B
:10F90000ECE731460848044B98470546E7E700BF57
:10F910008DF64000140F00209DF240009DF740003E
:10F920000C0F0020100F0020D80F0020264B1B6862
:10F93000002B2FD110B50022244B1A60244B1B68DA
:10F940001B6B1A68B2F1A53F28D0214B18681968C3
:10F950003431204B9847204B1B68B3FA83F3DBB25A
:10F96000C3F11F031D489A00D418A10001444C683C
:10F9700064684C601A4491000831084484421AD0EB
:10F9800003EB83039A00154B13445B68DA68104B52
:10F990001A6010BD01220D4B1A6070475A68B2F10F
:10F9A000A53FD2D19A68B2F1A53FCED1DB68B3F1C1
:10F9B000A53FCAD1CFE7606803EB83029100074AF5
:10F9C0000A445060DCE700BF800F0020F00F0020E9
:10F9D000080F002049084100880F0020140F002064
:10F9E00010B50C46044B19681831044B9847012197
:10F9F0002046034B984710BD080F0020B5E8400093
:10FA0000DDF4400038B50D461446064B1968183130
:10FA1000054B98470CB14FF0FF3521462846034B64
:10FA2000984738BD080F00209DE84000DDF44000F5
:10FA300038B5C368DC6804F118052846144B9847AC
:10FA4000144B1B68E3B9251D2846114B9847E36A00
:10FA500001229A401049086802430A6003EB8303BD
:10FA60009A0029460D4810440D4B9847E26A0D4B09
:10FA70001B68DB6A9A4208D901200B4B186038BD1D
:10FA800029460A48064B9847F0E7002038BD00BFDA
:10FA9000E9E84000800F0020880F0020140F0020AC
:10FAA0009DE84000080F0020F00F0020C00F00204C
:10FAB000034B1B680360034B1B684360704700BF28
:10FAC000BC0F0020EC0F0020F8B504460D46124B89
:10FAD0009847124B19686268881A2B68B3F1FF3F88
:10FAE00016D027680E4E3668B74201D0914211D227
:10FAF000984206D300232B6001240A4B98472046E6
:10FB0000F8BD1B1A2B602046074B98470024F4E7EA
:10FB10000024F2E70124F0E7C5E94000EC0F0020E3
:10FB2000BC0F0020E5E94000B1FA40000122014B82
:10FB30001A607047F00F002008B5034618B1186B23
:10FB4000024B984708BD024B1B68F8E7FDF24000E6
:10FB5000080F0020054B1B6823B1054B1B681BB920
:10FB6000022070470120704700207047D40F00200A
:10FB7000800F0020002854D038B50446C26A2A49B4
:10FB80000968C96A8A4242D28169002905DB26498F
:10FB90000968C96AC1F105018161606902EB8202ED
:10FBA0009100224A0A44904207D000223AB91E4AE4
:10FBB0001268D26AE262012038BD0122F6E7251DF3
:10FBC00028461B4B984768B9E36A03EB83018A0018
:10FBD00016498A5832B901229A4016490B6823EA1D
:10FBE00002030B60104B1B68DB6AE362012404FA1A
:10FBF00003F21049086802430A6003EB83039A008A
:10FC000029460A4810440C4B9847204638BDC26C20
:10FC1000054B1B68DB6A9A4201D2012038BD0020E7
:10FC200038BD0020704700BF080F0020140F0020CF
:10FC3000E9E84000880F00209DE84000002834D00B
:10FC400038B50446026D013A0265C06AE16C88422B
:10FC50002DD00AB1002038BD251D2846154B9847E8
:10FC600068B9E36A03EB83018A0013498A5832B901
:10FC700001229A4011490B6823EA02030B60E36CEE
:10FC8000E362C3F10502A261012404FA03F20B4905
:10FC9000086802430A6003EB83039A00294606487A
:10FCA0001044074B9847204638BD0020704700207D
:10FCB00038BD00BFE9E84000140F0020880F002085
:10FCC0009DE84000002843D038B50446C26C8A4203
:10FCD00000D20A46E16A8A4202D0206D012800D093
:10FCE00038BDE262A069002802DBC2F10502A26110
:10FCF000636901EB81018800164A0244934225D0D2
:10FD00000022002AECD0251D2846134B984768B9DD
:10FD1000E36A03EB83018A000E498A5832B9012253
:10FD20009A400E490B6823EA02030B60E36A012242
:10FD30009A400A49086802430A6003EB83039A0069
:10FD4000294604481044064B9847C9E70122D8E7E2
:10FD5000704700BF140F0020E9E84000880F002022
:10FD60009DE84000054B1B6823B1044B1A68136DD6
:10FD700001331365014B1868704700BF080F00205E
:10FD800038B505460C461A4B98471A4B1B685B6DF5
:10FD90002BB9184B1B68012283F85820ACB9164BBD
:10FDA0009847134B9847134B1B685C6D24B1CDB932
:10FDB000104B1B68621E5A650E4B1B68002283F8AD
:10FDC00058200D4B9847204638BD114620460B4B16
:10FDD00098474FF080520A4B1A60BFF34F8FBFF322
:10FDE0006F8FDCE7034B1B6800225A65E4E700BF16
:10FDF000C5E94000080F0020E5E94000DDF44000BF
:10FE000004ED00E0F8B507460D4614461E46214BAA
:10FE10009847214B1B6893F85830DBB2022B0AD06D
:10FE20001D4B1A68506D20EA070050651B680122BF
:10FE300083F85820CEB9194B9847164B98471CB1F8
:10FE4000154B1B685B6D2360134B1B6893F8583090
:10FE5000DBB2022B16D000240F4B1B68002283F864
:10FE600058200E4B98472046F8BD114630460C4BA3
:10FE700098474FF080520B4B1A60BFF34F8FBFF380
:10FE80006F8FD8E7044B1A68536D23EA0505556553
:10FE90000124E1E7C5E94000080F0020E5E9400042
:10FEA000DDF4400004ED00E0F8B504460F461546C9
:10FEB0001E46214B98470EB1636D336094F858305D
:10FEC000DBB2022284F858206A1E032A1AD8DFE81F
:10FED00002F0020C1114626D174367650125012BB6
:10FEE00014D0164B98472846F8BD626D0132626502
:10FEF0000125F4E767650125F1E7022B04D067656A
:10FF00000125ECE70125EAE70025E8E7261D304654
:10FF10000B4B9847E36A01229A400A49086802435A
:10FF20000A6003EB83039A00314607481044074BED
:10FF30009847074B1B68D4E7C5E94000E5E9400056
:10FF4000E9E84000880F0020140F00209DE84000E1
:10FF5000080F0020F8B5EFF311854FF0500484F33B
:10FF60001188BFF36F8FBFF34F8F0BB1446D1C60CF
:10FF700090F85830DBB2022480F85840013A032A46
:10FF80001AD8DFE802F0020C1114426D11434165EA
:10FF90000126012B14D085F311883046F8BD426D3F
:10FFA000013242650126F4E741650126F1E7022BA3
:10FFB00004D041650126ECE70126EAE70026E8E7E0
:10FFC0000446164B1B68F3B9071D3846144B984777
:10FFD000E36A01229A401349086802430A6003EB6E
:10FFE00083039A00394610481044104B9847E26A40
:10FFF0000F4B1B68DB6A9A42CDD9069B4BB101239C
:020000040041B9
:10000000069A1360C7E700F118010A48074B9847A2
:10001000EDE70122084B1A60BDE700BF800F00200A
:10002000E9E84000880F0020140F00209DE8400000
:10003000080F0020C00F0020F00F0020F8B5EFF3EC
:1000400011854FF0500383F31188BFF36F8FBFF317
:100050004F8F90F85830DBB2022280F85820426D62
:1000600001324265012B02D085F31188F8BD0E469E
:100070000446154B1B68E3B9071D3846134B9847D8
:10008000E36A01229A401249086802430A6003EBBE
:1000900083039A0039460F4810440F4B9847E26A91
:1000A0000E4B1B68DB6A9A42DED946B101233360EE
:1000B000DAE700F118010A48074B9847EFE70122F9
:1000C000084B1A60D0E700BF800F0020E9E840002D
:1000D000880F0020140F00209DE84000080F00202A
:1000E000C00F0020F00F0020064B1A681368B3FA07
:1000F00083F35B09036013B9D36818687047002065
:10010000704700BFF40F002008B5416000619142C4
:100110000CD8D21A83699A4201D3012008BD011D6F
:10012000094B1868094B9847002008BD9A4201D234
:10013000994206D2011D064B1868044B98470020CF
:1001400008BD012008BD00BFF80F0020B5E8400041
:10015000F40F002070B5104B9847104B1B6813B17B
:100160000F4B984770BD0F4D28460F4EB0470F4CB0
:100170002046B0470E4B1D600E4B1C6000220C2128
:100180000A200D4B9847054B18600028E8D00B4912
:100190000B4B9847E4E700BFC5E94000281000205A
:1001A000E5E94000FC0F002081E84000101000202D
:1001B000F40F0020F80F002079ED40003457410083
:1001C00011F240002DE9F041079C7CB1984615469C
:1001D0000E460746064B98472760A661E561C4F8BE
:1001E0002080069B6362201D024B9847BDE8F0818A
:1001F0005501410097E8400010B582B0094B98477F
:10020000094B1B6863B1094B01930323009300233F
:100210004FF42F7206490748074CA04702B010BDA3
:100220000020FBE755014100281000202C10002081
:100230003C57410031054100A1F540002DE9F04156
:1002400082B005460E46174698462C20084B984724
:10025000044640B10190089B009343463A4631461C
:100260002846044DA847204602B0BDE8F08100BFF3
:1002700019EB4000C501410030B585B0134C25682D
:100280000DB31C46019102920390052913DC104B1B
:100290009847022807D000231A4601A90B48006896
:1002A0000C4CA0470DE00023089A01A907480068FC
:1002B000084CA04705E00023224601A92846064C29
:1002C000A04705B030BD0020FBE700BF281000208C
:1002D00055FB4000B5ED40000DEF400070B582B019
:1002E000154B1B681A6802B3DB681E68DC68251DA5
:1002F0002846124B9847636A20469847E369012BCA
:10030000EED1A36933449E4207D26360246129463B
:10031000094B18680A4B9847E2E7002100910B4609
:1003200032462046074CA047DAE7074A10680249E0
:100330000860136002B070BDF40F0020E9E84000CF
:10034000B5E8400079024100F80F002038B50546B5
:10035000084B98470446084B1B68984205D3002376
:100360002B60054B1C60204638BD044B9847012389
:100370002B60F6E79DF6400024100020DD024100CE
:1003800070B582B005460E460F4B1B68DB68DC6813
:10039000201D0E4B9847E369012B04D0636A204669
:1003A000984702B070BDA1692B46324629442046C9
:1003B000074EB0470028F1D0002100910B462A4695
:1003C0002046044DA847E9E7F40F0020E9E8400083
:1003D000090141007902410070B582B006460C4621
:1003E000174B984701A8174B9847019B23BB05461D
:1003F0000CB9B04219D22CB1134B1B681C68B4FA6B
:1004000084F464092246711B104B1868104B9847FE
:10041000104B984738B94FF080520F4B1A60BFF31A
:100420004F8FBFF36F8F02B070BD0A4B98472946BC
:1004300030460A4B9847F6E7064B9847F3E700BF6C
:100440008DF640004D034100F80F002028100020D9
:1004500039F240009DF7400004ED00E081034100C7
:1004600030B587B0002203A92A4B18682A4B984759
:1004700000284CD0039B002BF4DB059C636913B16F
:10048000201D264B984702A8254B9847039B092B14
:10049000E8D801A252F823F0C1044100C104410090
:1004A000C104410065044100F50441000705410015
:1004B000C1044100C104410065044100F50441004C
:1004C0000499A5690B46024629442046154DA847C4
:1004D0000028C7D0636A20469847E369012BC1D141
:1004E000A269002100910B460498024420460E4C5C
:1004F000A047B7E70499A16103460246014420469C
:10050000084CA047AEE72046084B9847AAE707B03B
:1005100030BD00BF2810002085EF4000E9E8400012
:100520004D03410009014100790241003DEB4000CB
:1005300000B583B001A8044B98470199034B984735
:10054000034B9847F6E700BFE9004100D90341009B
:1005500061044100064BDB6BC3F30023054A1370B3
:10056000054BDB6BC3F34033044A1370704700BF85
:1005700000100E4030100020000E0E403110002000
:1005800008B5054BDB6B13F4004F02D1034B9847C2
:1005900008BD034B984708BD000E0E40B9544000FB
:1005A000DD54400030B583B004460D46002301936E
:1005B0002E4B984213D02E4B9C421AD02D4B9C426E
:1005C00021D02D4B9C4228D02C4B9C422FD02C4B21
:1005D0009C4236D02B4B9C423DD003B030BD01A98C
:1005E0002046294B98470028F9D19DF804302B70FC
:1005F000E1E701A92046244B98470028F9D19DF84E
:1006000004302B70DAE701A920461F4B98470028D9
:10061000F9D19DF804302B70D3E701A920461A4B7D
:1006200098470028F9D19DF804302B70CCE701A938
:100630002046154B98470028F9D19DF804302B70BF
:10064000C5E701A92046104B98470028F9D19DF82D
:1006500004302B70BEE701A920460B4B98470028B9
:10066000F9D19DF804302B70B7E700BF00C20040FD
:1006700000020240004202400082014000C20140EC
:10068000008200400002044029E5400038B50446DD
:100690000D46274B984213D0264B984218D0264B34
:1006A00098421DD0254B984222D0254B984227D006
:1006B000244B98422CD0244B984231D0002038BD96
:1006C00029462046214B98470028F9D1012038BD02
:1006D000294620461D4B98470028F9D1012038BDF6
:1006E00029462046194B98470028F9D1012038BDEA
:1006F00029462046154B98470028F9D1012038BDDE
:1007000029462046114B98470028F9D1012038BDD1
:10071000294620460D4B98470028F9D1012038BDC5
:1007200029462046094B98470028F9D1012038BDB9
:1007300000C200400002024000420240008201402C
:1007400000C20140008200400002044001E5400078
:1007500000B583B002A9002341F8043D084B186896
:10076000084B9847019B3BB14FF08052064B1A60F3
:10077000BFF34F8FBFF36F8F03B05DF804FB00BF73
:10078000381000203D00410004ED00E070B58AB053
:100790001D4B0FCB0AAC04E90F001C4D1C4B1D6018
:1007A0001C4A1D4B1A601D4A1D4B1A60069B009384
:1007B000079B0193089B0293099B039300240494D5
:1007C000184E3046184B984701213046174B984732
:1007D000174A69462846174B98472846164B9847AC
:1007E0002846164B9847164E336821469868154D93
:1007F000A847336821465868A84733682146986857
:10080000A8470AB070BD00BF4457410000820140B4
:100810004C2300208D06410048230020A5054100FF
:100820004423002000800140E9E0400051E2400004
:100830000000DC058DE54000D9E44000E5E440001F
:100840003C030020B923410008B504460D460A4682
:1008500001460748074B98470220074B984729460F
:100860002046064B9847EFF30580054B9847FFDE7F
:1008700008584100291A4100854D4000714D400043
:10088000914D400070B51F4B98471F4B1B68C31A12
:10089000632B00D870BD1C4B18601C4B18681C4D96
:1008A000A8471C4C20601C481C4EB047A8476060FD
:1008B0001B48B047A847A0601A48B047A847E06067
:1008C0001948B047A84720611848B047A847606159
:1008D0001748B047A847A0611648B047A847E0614D
:1008E0001548B047A84720621448B047A84760623F
:1008F0001348B047A847A0621248B047A847E06233
:10090000C8E700BF9DF640003410002038100020DA
:1009100039FB4000C8230020FC574100B5F84000D7
:10092000C84E41006456410084564100B85641000B
:10093000D8564100F856410018564100604E41001B
:100940002C5741003C574100704700002DE9F0430F
:1009500083B04B4B98474B4A936843F0254343F48D
:1009600080139360484B9847484B9847484B9847AB
:10097000484B9847484B9847484B98470446484B44
:100980009847F02201462046464B9847464B9847E9
:100990004648474B03602223037123234371454D8F
:1009A0002946454CA0474548454B03602B2303711E
:1009B0002A2343712946A047424B9847424B984708
:1009C0004248434B98474348434CA0474349444817
:1009D000A04744494448A047444A45494548A047A0
:1009E00000230193042200924FF48072424943484D
:1009F000434CA047012802D04248374B98473E4815
:100A0000414B9847414B1860414B9847414B9847A1
:100A1000414B9847414B9847414A00210F20414E96
:100A2000B047414C03220B212046404DA847DFF838
:100A300010914A4600212820B0473D4F03220C2147
:100A40003846A8472820DFF8FC80C04701463846D2
:100A5000384FB8474A4600210D20B04703220B21EA
:100A60002046A8470D20C04701462046B847324BD4
:100A70009847324B9847002003B0BDE8F08300BF91
:100A80006945400010140E4069DF4000997D400028
:100A9000697140008D07410039794000F17A4000CA
:100AA000F97A4000B1794000CD794000B4230020AC
:100AB00000000240A0860100FD754000A023002038
:100AC00000C0014005BE40003170400051074100A8
:100AD0005D45400054574100291A41006C574100C0
:100AE00080574100104B41008C574100A0574100F6
:100AF000AC574100B8574100D0574100057B40003A
:100B0000A1F54000D8574100B5F84000381000204A
:100B1000019B4000E9B4400095A440000D934000C3
:100B20008105410069C14000000E0E40D9C140005E
:100B300000100E40E7DE40001F50400015F6400058
:100B4000550541000BDF400030B583B000248DF81F
:100B500004408DF805408DF806400F4B98470F4B29
:100B6000984720460E4B98470E4D01A928460E4B3C
:100B7000984772B60D480E4CA0472846A0470D4B2B
:100B800098470D4B98470D4B98470D4A136823F033
:100B90000103136003B030BD557D40008DF6400069
:100BA00001544000A0230020C1634000B423002072
:100BB00095764000A553400051BE40004D7A40005C
:100BC00010E000E000487047B42300200048704760
:100BD000A023002008B5014B984708BD017B4000C9
:100BE00008B5014B984708BD037B400070470120C2
:100BF0007047000008B50248024B984708BD00BF87
:100C0000B42300203577400008B50248024B9847CE
:100C100008BD00BFA023002035774000014B1878A5
:100C2000704700BF31100020014B1878704700BF9B
:100C30003010002008B50448044B984708B1022042
:100C400008BD012008BD00BFA02300207D65400035
:100C5000014B1878704700BF32100020014B18700C
:100C6000704700BF3210002070B58AB0044600F013
:100C70006FF8324B93F900506B1C064609D02146A1
:100C8000204600F08DFE20B90021204600F07EFEB7
:100C900010B130460AB070BD294B08902046019330
:100CA00000F006FBCDE90401CDE902012046CDB9F3
:100CB000244B4FF060420021CDE9062300F03EFEB8
:100CC000002833D002230093684600F085F9A8B1CC
:100CD000089BC3B9DDE9060100F03EFB064630463D
:100CE0000AB070BD184B00220021CDE9062300F0A8
:100CF00025FE68B102239D420093E5D100F066FE17
:100D000022230360E4E700F061FE089B0360E1E753
:100D10000123022D00930BD100F058FE2123036024
:100D20000A4800F05BF9CDE90601D1E70123009301
:100D3000684600F051F90028F2D1EDE738030020B1
:100D400020584100FFFFEFC70000F0FF2857410087
:100D50002DE9F84F30F000432DD00028014604461D
:100D60004ADBB0F1FF4F3BDAB0F5000F3CDB002669
:100D70008D4AC4F316052A4402F40002E41582F0F9
:100D80007E507F3C34444FF07E51284304EBD254D4
:100D900000F036FB05F10F03C3F316030F2B0646D5
:100DA00031DC002100F0CAFD002800F094804CB92D
:100DB0000020BDE8F88F00214FF04C4000F0DEFC31
:100DC000BDE8F88F204600F0D1FB7849054600F0D9
:100DD00021FC77490446284600F01CFC01462046C9
:100DE00000F010FBBDE8F88F4FF0984100F012FCC6
:100DF0006FF018060446BBE700F002FB002100F08C
:100E0000BDFCBDE8F88F4FF0804100F0FBFA0146D1
:100E1000304600F0B3FC8046204600F0A7FB414678
:100E20008146404600F0F6FB0146834600F0F2FBA7
:100E30006049DFF8A0A1074600F0ECFB5E4900F036
:100E4000E1FA394600F0E6FB5C4900F0DBFA39468E
:100E500000F0E0FB5A4900F0D5FA594600F0DAFB01
:100E600058498346384600F0D5FB574900F0CAFA86
:100E7000394600F0CFFB554900F0C4FA394600F07E
:100E8000C9FB0146584600F0BDFAC5F55713AA4400
:100E900003F5227343EA0A03002B074665DD4FF092
:100EA0007C51304600F0B6FB314600F0B3FB0546FE
:100EB000002C32D12946384600F0A4FA414600F011
:100EC000A9FB0146284600F09BFA0146304600F097
:100ED00097FABDE8F88F3E49304600F09BFB01468B
:100EE0004FF07C5000F08CFA31460546304600F059
:100EF00091FB0146284600F08DFB0546002C2ED0C4
:100F0000204600F033FB2949074600F083FB2849BF
:100F10000446384600F07EFB14E02449484600F0C1
:100F200079FB29460446384600F06CFA414600F049
:100F300071FB1F490746484600F06CFB01463846E6
:100F400000F060FA0146284600F05AFA314600F0F7
:100F500057FA0146204600F053FABDE8F88F0146E3
:100F6000304600F04DFABDE8F88F7CB10F49484695
:100F700000F050FB39460446304600F041FA414645
:100F800000F048FB0A4905464846C3E7014630469B
:100F900000F036FA414600F03DFB0146304600F0D5
:100FA0002FFABDE8F88F00BF20FB4A008071313F67
:100FB000D1F717379788173E25333A3E2549923E99
:100FC000ABAA2A3F4FD01C3E298E633ECDCCCC3EEF
:100FD000ABAAAA3E305CCFFF002070470020014939
:100FE000704700BF0000F87F81F0004102E000BFC1
:100FF00083F0004330B54FEA41044FEA430594EAD9
:10100000050F08BF90EA020F1FBF54EA000C55EA13
:10101000020C7FEA645C7FEA655C00F0E2804FEAE4
:101020005454D4EB5555B8BF6D420CDD2C4480EAC6
:10103000020281EA030382EA000083EA010180EAF6
:10104000020281EA0303362D88BF30BD11F0004F44
:101050004FEA01314FF4801C4CEA113102D040427A
:1010600061EB410113F0004F4FEA03334CEA1333B5
:1010700002D0524263EB430394EA050F00F0A780CD
:10108000A4F10104D5F1200E0DDB02FA0EFC22FAC8
:1010900005F2801841F1000103FA0EF2801843FABC
:1010A00005F359410EE0A5F120050EF1200E012AAD
:1010B00003FA0EFC28BF4CF0020C43FA05F3C018EB
:1010C00051EBE37101F0004507D54FF0000EDCF164
:1010D000000C7EEB00006EEB0101B1F5801F1BD30D
:1010E000B1F5001F0CD349085FEA30004FEA3C0C11
:1010F00004F101044FEA445212F5800F80F09A8007
:10110000BCF1004F08BF5FEA500C50F1000041EB0A
:10111000045141EA050130BD5FEA4C0C404141EB0E
:10112000010111F4801FA4F10104E9D191F0000F35
:1011300004BF01460020B1FA81F308BF2033A3F1B8
:101140000B03B3F120020CDA0C3208DD02F1140CAF
:10115000C2F10C0201FA0CF021FA02F10CE002F1EA
:101160001402D8BFC2F1200C01FA02F120FA0CFCE3
:10117000DCBF41EA0C019040E41AA2BF01EB04512C
:10118000294330BD6FEA04041F3C1CDA0C340EDC2A
:1011900004F11404C4F1200220FA04F001FA02F36D
:1011A00040EA030021FA04F345EA030130BDC4F12B
:1011B0000C04C4F1200220FA02F001FA04F340EA20
:1011C0000300294630BD21FA04F0294630BD94F0D1
:1011D000000F83F4801306BF81F480110134013DB8
:1011E0004EE77FEA645C18BF7FEA655C29D094EA29
:1011F000050F08BF90EA020F05D054EA000C04BFA7
:101200001946104630BD91EA030F1EBF0021002091
:1012100030BD5FEA545C05D14000494128BF41F030
:10122000004130BD14F580043CBF01F5801130BD94
:1012300001F0004545F0FE4141F470014FF000001F
:1012400030BD7FEA645C1ABF194610467FEA655CD0
:101250001CBF0B46024650EA013406BF52EA033572
:1012600091EA030F41F4002130BD00BF90F0000F60
:1012700004BF0021704730B54FF4806404F132049C
:101280004FF000054FF0000150E700BF90F0000F55
:1012900004BF0021704730B54FF4806404F132047C
:1012A00010F0004548BF40424FF000013EE700BF4C
:1012B00042004FEAE2014FEA31014FEA02701FBFDC
:1012C00012F07F4393F07F4F81F06051704792F0AE
:1012D000000F14BF93F07F4F704730B54FF4607428
:1012E00001F0004521F0004120E700BF50EA010273
:1012F00008BF704730B54FF000050AE050EA010220
:1013000008BF704730B511F0004502D5404261EB8F
:1013100041014FF4806404F132045FEA915C3FF4D0
:10132000DCAE4FF003025FEADC0C18BF03325FEA69
:10133000DC0C18BF033202EBDC02C2F1200300FA1E
:1013400003FC20FA02F001FA03FE40EA0E0021FA43
:1013500002F11444C1E600BF4FEA4102B2F1E0439A
:1013600024BFB3F5001CDCF1FE5C0DD901F0004C8C
:101370004FEAC0024CEA5070B2F1004F40EB8300DC
:1013800008BF20F00100704711F0804F21D113F108
:101390003872BCBF01F00040704741F480114FEA41
:1013A0005252C2F11802C2F1200C10FA0CF320FACA
:1013B00002F018BF40F001004FEAC1234FEAD323E7
:1013C00003FA0CFC40EA0C0023FA02F34FEA430351
:1013D000CCE77FEA625307D150EA01331EBF4FF0DA
:1013E000FE4040F44000704701F0004040F0FE40F5
:1013F00040F40000704700BF80F0004002E000BFF2
:1014000081F0004142001FBF5FEA410392EA030FEF
:101410007FEA226C7FEA236C6AD04FEA1262D2EB39
:101420001363C1BFD218414048404140B8BF5B423E
:10143000192B88BF704710F0004F40F4000020F0D7
:101440007F4018BF404211F0004F41F4000121F0ED
:101450007F4118BF494292EA030F3FD0A2F1010237
:1014600041FA03FC10EB0C00C3F1200301FA03F175
:1014700000F0004302D5494260EB4000B0F5000F98
:1014800013D3B0F1807F06D340084FEA310102F157
:101490000102FE2A51D2B1F1004F40EBC25008BF09
:1014A00020F0010040EA03007047490040EB0000D3
:1014B00010F4000FA2F10102EDD1B0FA80FCACF102
:1014C000080CB2EB0C0200FA0CF0AABF00EBC25001
:1014D00052421843BCBFD0401843704792F0000FEF
:1014E00081F4000106BF80F400000132013BB5E742
:1014F0004FEA41037FEA226C18BF7FEA236C21D0B8
:1015000092EA030F04D092F0000F08BF084670471C
:1015100090EA010F1CBF0020704712F07F4F04D1EA
:10152000400028BF40F00040704712F100723CBFFD
:1015300000F50000704700F0004343F0FE4040F427
:10154000000070477FEA226216BF08467FEA2363E5
:101550000146420206BF5FEA412390EA010F40F4D0
:10156000800070474FF0000304E000BF10F000431C
:1015700048BF40425FEA000C08BF704743F0964303
:1015800001464FF000001CE050EA010208BF70471E
:101590004FF000030AE000BF50EA010208BF7047A5
:1015A00011F0004302D5404261EB41015FEA010CBA
:1015B00002BF84460146002043F0B64308BFA3F1B2
:1015C0008053A3F50003BCFA8CF2083AA3EBC25394
:1015D00010DB01FA02FC634400FA02FCC2F12002B3
:1015E000BCF1004F20FA02F243EB020008BF20F0EA
:1015F0000100704702F1200201FA02FCC2F1200250
:1016000050EA4C0021FA02F243EB020008BF20EA44
:10161000DC7070474FF0FF0C1CEAD0521EBF1CEA72
:10162000D15392EA0C0F93EA0C0F6FD01A4480EA60
:10163000010C400218BF5FEA41211ED04FF0006349
:1016400043EA501043EA5111A0FB01310CF0004075
:10165000B1F5000F3EBF490041EAD3715B0040EA9B
:10166000010062F17F02FD2A1DD8B3F1004F40EB6B
:10167000C25008BF20F00100704790F0000F0CF03E
:10168000004C08BF49024CEA502040EA51207F3A02
:10169000C2BFD2F1FF0340EAC250704740F40000DD
:1016A0004FF00003013A5DDC12F1190FDCBF00F0CE
:1016B00000407047C2F10002410021FA02F1C2F17C
:1016C000200200FA02FC5FEA310040F1000053EA18
:1016D0004C0308BF20EADC70704792F0000F00F066
:1016E000004C02BF400010F4000F013AF9D040EA6C
:1016F0000C0093F0000F01F0004C02BF490011F400
:10170000000F013BF9D041EA0C018FE70CEAD153FD
:1017100092EA0C0F18BF93EA0C0F0AD030F0004C7D
:1017200018BF31F0004CD8D180EA010000F0004031
:10173000704790F0000F17BF90F0004F084691F0EF
:10174000000F91F0004F14D092EA0C0F01D1420229
:101750000FD193EA0C0F03D14B0218BF084608D1F2
:1017600080EA010000F0004040F0FE4040F400003C
:10177000704740F0FE4040F4400070474FF0FF0CCF
:101780001CEAD0521EBF1CEAD15392EA0C0F93EA16
:101790000C0F69D0A2EB030280EA010C49024FEA68
:1017A000402037D04FF0805343EA111143EA101321
:1017B0000CF000408B4238BF5B0042F17D024FF4D9
:1017C000000C8B4224BF5B1A40EA0C00B3EB510FB4
:1017D00024BFA3EB510340EA5C00B3EB910F24BF9D
:1017E000A3EB910340EA9C00B3EBD10F24BFA3EB22
:1017F000D10340EADC001B0118BF5FEA1C1CE0D1EA
:10180000FD2A3FF650AF8B4240EBC25008BF20F09C
:10181000010070470CF0004C4CEA50207F32C2BFF0
:10182000D2F1FF0340EAC250704740F400004FF08D
:101830000003013A37E792F0000F00F0004C02BFBE
:10184000400010F4000F013AF9D040EA0C0093F088
:10185000000F01F0004C02BF490011F4000F013BE2
:10186000F9D041EA0C0195E70CEAD15392EA0C0F4A
:1018700008D142027FF47DAF93EA0C0F7FF470AF82
:10188000084676E793EA0C0F04D14B023FF44CAFC5
:1018900008466EE730F0004C18BF31F0004CCAD15A
:1018A00030F000427FF45CAF31F000437FF43CAF96
:1018B0005FE700BF4FF0FF3C06E000BF4FF0010CB8
:1018C00002E000BF4FF0010C4DF804CD4FEA40029A
:1018D0004FEA41037FEA226C18BF7FEA236C11D0E4
:1018E00001B052EA530C18BF90EA010F58BFB2EB97
:1018F000030088BFC81738BF6FEAE17018BF40F017
:10190000010070477FEA226C02D15FEA402C05D1CA
:101910007FEA236CE4D15FEA412CE1D05DF8040B4F
:10192000704700BF844608466146FFE70FB5FFF7E2
:10193000C9FF002848BF10F1000F0FBD4DF808ED9A
:10194000FFF7F4FF0CBF012000205DF808FB00BF8B
:101950004DF808EDFFF7EAFF34BF012000205DF8E5
:1019600008FB00BF4DF808EDFFF7E0FF94BF012032
:1019700000205DF808FB00BF4DF808EDFFF7D2FF2F
:1019800094BF012000205DF808FB00BF4DF808ED72
:10199000FFF7C8FF34BF012000205DF808FB00BF3F
:1019A0004FEA40024FEA41037FEA226C02D15FEA2C
:1019B000402C08D17FEA236C02D15FEA412C02D18E
:1019C0004FF0000070474FF001007047014B18685E
:1019D000704700BF3C03002070B50F4E0F4D761BC3
:1019E000B61018BF002405D0013455F8043B9847C1
:1019F000A642F9D10A4E0B4D761B03F0C9FFB61073
:101A000018BF002406D0013455F8043B9847A6427D
:101A1000F9D170BD70BD00BF9C5941009C59410077
:101A2000A45941009C5941000FB400B5074983B047
:101A300004AB086853F8042B8168019300F06CFE36
:101A400003B05DF804EB04B0704700BF3C03002016
:101A5000024B0146186800F00BB800BF3C030020A1
:101A6000024B0146186801F073BF00BF3C03002021
:101A70002DE9F04F01F10B06162E83B0054640F21A
:101A80009E8036F0070600F1BD80B14200F2BA80B8
:101A900000F06AFCB6F5FC7FC0F09382730A00F098
:101AA000B880042B00F27981B30903F1390003F106
:101AB000380EC300BF4F3B44A3F108015C68A1424C
:101AC00006D10CE0002A80F2AA80E468A14206D088
:101AD000636823F003039A1B0F2AF3DD70463C6909
:101AE000DFF8E4E2744500F0AB81636823F00303A0
:101AF0009A1B0F2A00F39081002AC7F814E0C7F858
:101B000010E080F29D80B3F5007F80F06181DB08FA
:101B100003F1010C99107A6857F83C80C4F80880EA
:101B200001238B4007EBCC0113430839E1607B6054
:101B300047F83C40C8F80C408210012494409C4275
:101B400000F28B801C4206D120F0030064001C428E
:101B500000F10400FAD007EBC009CC468046DCF85F
:101B60000C309C4507D16DE1002A80F27B81DB6857
:101B70009C4500F06781596821F003018A1B0F2AF8
:101B8000F2DDD3F80CC0D3F8088000939C192846E6
:101B900046F0010642F001055E60C8F80CC0CCF8C2
:101BA00008807C613C61C4F80CE0C4F808E0656022
:101BB0005A5000F0DFFB009B03F108041EE01029DF
:101BC00020D800F0D1FB102618230220794F3B4487
:101BD000A3F108025C68944200F03D816368E1680B
:101BE000A66823F00303234428465A68F16042F0B4
:101BF00001028E605A6000F0BDFB0834204603B03D
:101C0000BDE8F08F00240C2320462B6003B0BDE814
:101C1000F08F40204FF400734FF03F0E4AE723440B
:101C2000E1685A68A66842F00102F16028468E60B9
:101C30005A6000F09FFB0834204603B0BDE8F08FE7
:101C4000234428465A6842F001025A6000F092FB91
:101C50000834204603B0BDE8F08FBC68636823F009
:101C60000308B04504D3A8EB06030F2B00F38580CF
:101C7000DFF85891504BD9F800201B6801323344EB
:101C800004EB080A00F0558103F580530F3323F469
:101C90007F6B2BF00F0B5946284600F07BFB411C55
:101CA000024600F0FC80824500F2F780434B196841
:101CB0005944196000F04D81D9F8000001301BBF74
:101CC000A2EB0A0A5144C9F80020196012F007017A
:101CD00000F01581C1F10800C1F5805102440831BE
:101CE00002EB0B09C9F30B09A1EB09094946284688
:101CF0000193009200F04EFB431C9DE80C0000F0A5
:101D00004381801A484440F001001968BA60494490
:101D1000BC425060196017D0B8F10F0F40F2FB8041
:101D20006068A8F10C0222F0070204EB020E00F03A
:101D300001004FF0050C10430F2A6060CEF804C07C
:101D4000CEF808C000F217811D4BBC681A6891429A
:101D500088BF19601B4B1A689142626888BF19607E
:101D600022F003029642A2EB060301D80F2B04DCFB
:101D7000284600F0FFFA002440E7A21943F00103CF
:101D800046F0010666602846BA60536000F0F2FA39
:101D90000834204603B0BDE8F08F142B71D9542BC2
:101DA00000F2A380330B03F16F0003F16E0EC3004A
:101DB00080E600BF680700206C1000203C10002067
:101DC000641000206810002070070020700B0020B5
:101DD0005A0A042A5BD9142A00F2AE8002F15C018F
:101DE000C9005B3207EB010C7958ACF1080C8C454B
:101DF00000F088804A6822F00302934273D2896817
:101E00008C45F7D1DCF80C207B68E260C4F808C090
:101E10009460CCF80C408FE6A11946F0010C42F01A
:101E20000106C4F804C0284679613961C1F80CE0A4
:101E3000C1F808E04E60E25000F09CFA0834DDE69C
:101E40007B6879E608F1010818F0030F0CF1080C23
:101E50007FF485AE2DE0DC68A34208BF02303FF47A
:101E60003EAEBBE619441C464A68DB6854F8086F6E
:101E700042F001024A602846F3609E6000F07AFA60
:101E8000BCE603F15C0003F15B0EC30012E69A09A5
:101E900002F13901C9003832A4E7BC4254D0BC6811
:101EA000626822F003025DE759F80839994540F06D
:101EB000868010F0030F00F1FF30F5D17B6823EA34
:101EC00004037B6064009C423FF6C7AE002C3FF4E5
:101ED000C4AE1C4240467FF43EAE64001C4200F19A
:101EE0000400FAD037E68C468CE7B3F5AA7F15D804
:101EF000F30B03F1780003F1770EC300DAE54FF43A
:101F00008051EDE67B689210012101FA02F2134341
:101F10007B60624679E70123536029E740F254521F
:101F2000934222D8B30C03F17D0003F17C0EC30071
:101F3000C0E503F1100BAEE6542A29D81A0B02F1C2
:101F40006F01C9006E324DE7204B19685944196082
:101F5000B2E6CAF30B0000287FF4AEAE08EB0B0329
:101F6000BA6843F001035360EEE67F204FF47E73BE
:101F70004FF07E0E9EE504F108012846009301F023
:101F8000E7FC009B1968DFE601204FF00009BCE682
:101F9000B2F5AA7F05D8DA0B02F17801C9007732D1
:101FA00020E740F254518A4205D89A0C02F17D0193
:101FB000C9007C3216E74FF47E717E2212E77B68FF
:101FC00080E7F00806F1080300E600BF3C1000209F
:101FD00001F0FF01102A2BDB10F0070F08D010F8DA
:101FE000013B013A8B422DD010F0070F42B3F6D1DE
:101FF000F0B441EA012141EA014122F007047FF0F7
:1020000000070023F0E80256083C85EA010586EA4D
:10201000010685FA47F5A3FA87F586FA47F6A5FA89
:1020200087F68EB9EED1F0BC01F0FF0102F0070295
:1020300032B110F8013B013A83EA010313B1F8D140
:102040000020704701387047002D06BF3546033821
:10205000073815F0010F07D1013015F4807F02BF5A
:10206000013015F4C03F0130F0BC0138704700BFAB
:10207000032A70B422D940EA01039B0711D00378E8
:102080000C78A3421DD10A44013105E010F8013F4C
:1020900011F8014BA34214D19142F7D1002070BC3A
:1020A00070470D680668AE420C46034601F1040114
:1020B00000F1040008D1043A032AF2D8002ADED144
:1020C000ECE7181B70BC704721461846D7E700BFE5
:1020D000844641EA000313F003036DD1403A41D333
:1020E00051F8043B40F8043B51F8043B40F8043BF2
:1020F00051F8043B40F8043B51F8043B40F8043BE2
:1021000051F8043B40F8043B51F8043B40F8043BD1
:1021100051F8043B40F8043B51F8043B40F8043BC1
:1021200051F8043B40F8043B51F8043B40F8043BB1
:1021300051F8043B40F8043B51F8043B40F8043BA1
:1021400051F8043B40F8043B51F8043B40F8043B91
:1021500051F8043B40F8043B51F8043B40F8043B81
:10216000403ABDD2303211D351F8043B40F8043B21
:1021700051F8043B40F8043B51F8043B40F8043B61
:1021800051F8043B40F8043B103AEDD20C3205D331
:1021900051F8043B40F8043B043AF9D2043208D029
:1021A000D2071CBF11F8013B00F8013B01D30B889B
:1021B00003806046704700BF082A13D38B078DD079
:1021C00010F003038AD0C3F10403D21ADB071CBF4B
:1021D00011F8013B00F8013B80D331F8023B20F8B5
:1021E000023B7BE7043AD9D3013A11F8013B00F8EE
:1021F000013BF9D20B7803704B7843708B78837076
:10220000604670478842F0B50DD98B1898420AD2C3
:102210008418002A51D0224613F8014D02F8014DCE
:102220009942F9D1F0BD0F2A48D941EA00039B0732
:1022300046D100F1100401F11003154653F8106C5B
:1022400044F8106C53F80C6C44F80C6C53F8086CA0
:1022500044F8086C103D53F8046C44F8046C0F2DDE
:1022600003F1100304F11004E8D8A2F1100323F0E5
:102270000F0302F00F0E1033BEF1030F1944034495
:1022800021D91E1F0D467446043C55F8047B46F8C0
:10229000047F032CF8D8AEF1040424F003040434C2
:1022A0002144234402F0030262B1013B0A4411F8C5
:1022B000014B03F8014F8A42F9D1F0BD0346F3E721
:1022C0000346F2E7F0BD7246EEE700BF70B4860742
:1022D00046D0541E002A41D0CAB2034602E014F18F
:1022E000FF343BD303F8012B9D07F8D1032C2ED9E3
:1022F000CDB245EA05250F2C45EA054519D903F16C
:1023000010022646103E0F2E42F8105C42F80C5C7C
:1023100042F8085C42F8045C02F11002F2D8A4F121
:10232000100222F00F0204F00F041032032C1344A9
:102330000DD91E462246043A032A46F8045BFAD811
:10234000221F22F003020432134404F003042CB1D0
:10235000C9B21C4403F8011B9C42FBD170BC7047FE
:1023600014460346C2E700BF014801F08BBD00BF21
:1023700018240020014801F087BD00BF1824002068
:1023800010B5034B0446196801F022FE204610BD2B
:102390003C03002038B5074C00230546084623605F
:1023A000FCF746FA431C00D038BD2368002BFBD055
:1023B0002B6038BD2C24002000290CBF02220022F3
:1023C0004FF4806300F000B82DE9F043614C2568BC
:1023D00083B004460F4690461E4615B1AB6B002BEA
:1023E00064D0B8F1020F06D0B8F1010F00F29F805F
:1023F000002EC0F29C80636ED80734D52146284653
:1024000001F028F9216B41B104F14003994202D057
:10241000284601F09DFA00232363B4F90C30002212
:10242000A26162601A063AD423F44A6323F00303DC
:10243000B8F1020FA3811DD001AB6A4621462846A0
:1024400001F024FDA3891843A081002E32D1009E03
:102450003046FFF7FDFA074600286BD0A38943F00A
:102460008003A38128E0A3899905C7D4A06D01F05A
:1024700009FDC3E70025616E002604F1430243F025
:1024800002030120A660CE07A38122602261606161
:1024900001D498053ED5284603B0BDE8F0832169F4
:1024A000284601F055FAB4F90C30BDE7284601F092
:1024B00029F996E7002FCBD0AB6B002B33D0009BD4
:1024C000B4F90C2027609E421CBF42F40062A28136
:1024D000B8F1010F04BF42F00102A28192B212F0E2
:1024E0000803276166610ED0D1071AD5656E764262
:1024F000002315F00105A661A36009D00025284638
:1025000003B0BDE8F083A360656E15F00105F5D159
:102510009305C0D4A06D01F0B7FC284603B0BDE818
:10252000F083A660F0E7284601F0ECF8C7E74FF02B
:10253000FF35B0E7DDF80090B14504D04846FFF71D
:1025400087FA074620B9B4F90C304FF0FF3592E70F
:102550004E4683E73C03002000000000000000001E
:10256000000000000000000000000000000000006B
:10257000000000000000000000000000000000005B
:1025800090F800F06DE9024520F007016FF0000CB3
:1025900010F0070491F820F040F049804FF000045B
:1025A0006FF00700D1E9002391F840F000F1080036
:1025B00082FA4CF2A4FA8CF283FA4CF3A2FA8CF36E
:1025C0004BBBD1E9022382FA4CF200F10800A4FAD5
:1025D0008CF283FA4CF3A2FA8CF3E3B9D1E9042329
:1025E00082FA4CF200F10800A4FA8CF283FA4CF360
:1025F000A2FA8CF37BB9D1E9062301F1200182FA1A
:102600004CF200F10800A4FA8CF283FA4CF3A2FA1F
:102610008CF3002BC6D0002A04BF04301A4612BA2D
:10262000B2FA82F2FDE8024500EBD2007047D1E930
:10263000002304F00305C4F100004FEAC50514F0BF
:10264000040F91F840F00CFA05F562EA05021CBF90
:1026500063EA050362464FF00004A9E7B1B10378CD
:10266000B3B10144431C994214D010B41A785C1CD5
:1026700032B1A142234606D01A785C1C002AF8D158
:10268000181A10BC7047081A10BC704708467047EB
:1026900018467047081A70472DE9F84F4B6E9C0496
:1026A00093462FD59368126853B30E46074602F13E
:1026B000080919E920045FEA9A0817D0043D0024AC
:1026C00001E0A04510D0324655F8041F384601F00D
:1026D000BBF8431C04F10104F3D10023CBF808300C
:1026E000CBF80430BDE8F88FDBF808302AF0030A95
:1026F000A3EB0A03CBF8083009F10809002BD8D165
:102700000020EAE701F00AFA0023CBF80830CBF802
:102710000430BDE8F88F00BF2DE9F04FADB01D4685
:102720008B4690460793069018B1836B002B00F000
:10273000F380DBF86430BBF90C00DF0781B202D410
:102740008E0540F1FC808C040AD4DBF8643040F440
:10275000005123F40053ABF80C10CBF8643089B26D
:10276000080740F1B380DBF81030002B00F0AE809A
:1027700001F01A030A2B00F0B58000230DF1700957
:102780000B93119310930393CDF83C90CA46CDF868
:1027900010B098F800304446FBB1252B02D11CE064
:1027A000252B03D014F8013F002BF9D1A4EB080529
:1027B0009DB1109B119ACAF8008001332A44072B5F
:1027C000CAF80450119210937ADD002A40F0B084C8
:1027D000039B10922B44CA4603932378002B00F0EE
:1027E000E08300204FF000038DF8373004F101083A
:1027F00062780546064603464FF0FF3408F10108AB
:10280000A2F12001582900F2DE82DFE811F0210256
:10281000DC02DC022902DC02DC02DC02DC02DC027B
:10282000DC0289029502DC02A200BD02DC029F01EB
:10283000A401A401A401A401A401A401A401A40170
:10284000A401DC02DC02DC02DC02DC02DC02DC02D1
:10285000DC02DC02DC02B201DC02DC02DC02DC02B3
:10286000DC02DC02DC02DC02DC02DC029701DC02BE
:10287000DC02DC02DC02DC029B01DC02DC02530233
:10288000DC02DC02DC02DC02DC02DC02DC02DC0258
:10289000DC02DC025A021B02DC02DC02DC026E02F9
:1028A0001B02DC02DC027302DC02F5018201090278
:1028B000D702DC029A02DC02A700DC02DC022E0254
:1028C0000AF1080A039B2B44039386E759460698AE
:1028D00000F0ACFD18BBBBF80C1001F01A030A2B7A
:1028E0007FF44BAFBBF90E30002BFFF646AFDBF8A1
:1028F0006430DB0705D48F0503D4DBF8580001F002
:10290000C3FA2B4642465946069800F04DFD039007
:1029100003982DB0BDE8F08F00F0F4FE09E7DBF876
:102920006430D90704D4BBF80C309A0540F1AA846E
:102930004FF0FF33039303982DB0BDE8F08FDBF821
:10294000580001F09FFABBF90C0081B2FBE6764219
:10295000079243F0040398F800204FE708969E067C
:1029600000F150840799DD060A4600F1EF8358060E
:1029700040F1EC830E8804310027012207914FF0CB
:1029800000018DF837100025611C00F0168123F03E
:102990008001029156EA070140F01481002C40F0BA
:1029A0005C83002A40F0B78313F00103059300F025
:1029B00057840DF1B00B30230BF8413D059BA3422A
:1029C000B8BF234601930DB101330193029B13F06D
:1029D0000203099302D0019B02330193029B13F07F
:1029E00084030A9340F01782089B019A9D1A002DD8
:1029F00040F31182102D40F39084109B119AC44E25
:102A0000D6461027A2461946069C07E001F1020CA3
:102A10000EF1080E0146103D102D11DD481C10323C
:102A2000072811928EE8C0001090EFDD002A40F0D8
:102A3000E481103D102D11464FF0010CCE46EDDC27
:102A400054466146F2462A4407291192CAF80060AA
:102A5000CAF80450109100F3EC829DF837500AF147
:102A6000080A481C002D40F0DE81099B002B00F075
:102A7000F88102320EA902230728119210908AE8E9
:102A80000A0040F3EA81002A40F08C830A9B802BE5
:102A90004FF001001146CA4640F0E781089B019DB6
:102AA0005E1B002E40F3E181102E9A4D40F35084BE
:102AB000D4461027A246069C07E001F1020E0CF155
:102AC000080C0146103E102E11DD481C103207285C
:102AD00011928CE8A0001090EFDD002A40F09D825A
:102AE000103E102E4FF0010E1146CC46EDDC544640
:102AF000E2463244BEF1070F11928AE86000CDF839
:102B000040E000F369830AF1080A0EF10100714602
:102B1000ABE1089613F0200240F08C8313F0100113
:102B200040F01A8313F0400200F0168307980A461B
:102B30000146043106880791002720E7089643F0F4
:102B40001003E7E7089643F0100308E743F080031B
:102B500098F8002052E6A2F13001002618F8012B67
:102B600006EB860601EB4606A2F130010929F5D9EC
:102B700046E60896002840F0088443F010039E06BD
:102B800000F14C83DD0600F1F382580640F1F0823B
:102B9000079DB5F900602A46F717043230463946DA
:102BA0000792002871F10002C0F25D83611C9DF85C
:102BB00037504FF001027FF4EAAE56EA070100F009
:102BC0004D820293012A00F08C82022A40F05C823E
:102BD0000B98CB46330906F00F0143EA07733A0915
:102BE0001E461746435C0BF8013D56EA0703F1D138
:102BF000A9EB0B030593E1E6002840F0C08399069A
:102C000000F16783DA0600F1F1805B0640F1EE80A7
:102C1000079A136804320792BDF80C201A80B8E5B1
:102C200007983D4A08960B920668782230210430B6
:102C30008DF8392043F00203079000278DF83810F3
:102C400002229CE60896002899D08DF8375096E726
:102C500098F80020002D7FF4D1AD01202025CDE58E
:102C600043F0010398F80020C8E50896002840F0DA
:102C7000938329490B919F0600F1E8820798DE06AD
:102C8000014600F170825D0640F16D8204310688D4
:102C900007910027D80740F1228256EA070100F089
:102CA0001E8230218DF8392043F002038DF8381050
:102CB000022264E60896002840F06B8317490B91C6
:102CC000D9E7079908960A688DF848204FF0000068
:102CD0000A468DF8370004320120019007920590D2
:102CE0000DF1480B0293002470E643F0400398F87E
:102CF000002083E598F800206C2A03BF98F8012093
:102D000043F0200308F1010843F0100376E500BF0B
:102D10005C5841006C584100405841002C5841001B
:102D200007990E680A46002E02F10402FFF60FAE64
:102D3000079298F8002061E598F8002001202B25E3
:102D40005CE507990896D1F800B04FF000028DF8C5
:102D500037200E1DBBF1000F00F0E582671C00F06C
:102D6000C4822246002158460193FFF731F9019BA6
:102D7000002800F0E582A0EB0B0205920796029373
:102D80009DF83750002419E698F800202A2A08F107
:102D9000010700F0E982A2F130010929B8464FF09D
:102DA00000043FF62DAD18F8012B04EB840401EB71
:102DB0004404A2F130010929F5D921E543F02003AB
:102DC00098F800201AE50896002840F0DB82002AD7
:102DD00000F0E78001218DF848204FF000020191BA
:102DE0008DF8372005910DF1480B7BE7079A1368A2
:102DF00004320792039A1A60CBE40FAA0499204682
:102E0000FFF74AFC002840F039811099119A01F12E
:102E1000010CCE46FFE51099119A481C9DF83750D9
:102E2000002D3FF422AE01320DF1370501210728B4
:102E300011921090CAF80050CAF8041040F30881AB
:102E4000002A40F0BC81099B002B3FF41FAE0EAB63
:102E5000022208461C931D92CA4601460AF1080A3E
:102E600001300A9B802B3FF419AE059BE41A002C1D
:102E70002EDD102CB34D1EDDD6461026069FDDF844
:102E800010A006E0881C0EF1080E1946103C102C0C
:102E900010DD4B1C1032072B11928EE8600010934E
:102EA000F0DD002A65D1103C102C4FF001001146D6
:102EB000CE46EEDCF246224407281192CAF80050B2
:102EC000CAF80440109000F385800AF1080A013026
:102ED0000599CAF800B00A4407281192CAF80410EC
:102EE000109040F38280002A40F01881029B1092DB
:102EF000580735D5089B01995C1A002C40F3E780F0
:102F0000CA46102C40F3188210998F4E069FDDF8A8
:102F100010B0102506E0881C0AF1080A1946103C7A
:102F2000102C11DD4B1C1032072B1192CAF80060D7
:102F3000CAF804501093EEDD42BB103C102C4FF049
:102F400001001146CA46EDDC224407281192CAF856
:102F50000060CAF80440109051DD002A40F09B81C7
:102F6000039B089A01998A42ACBF9B185B18039394
:102F70004EE00FAA51463846FFF78EFB002840F07E
:102F80003F811099119A481CCE467FE70FAA5946F7
:102F90003846FFF781FB60B91099119A481CCA4660
:102FA000BDE7119BDDF810B0002B40F0D481002369
:102FB0001093DBF8643013F0010FBBF80C3002D132
:102FC0009A0540F1DE805B063FF5B2AC03982DB068
:102FD000BDE8F08F002A40F00681059A1D9201237A
:102FE0001192CDF870B01093CA460AF1080A029BFC
:102FF000590704D5089B01995C1A002C81DC039BBE
:10300000089901988142ACBF5B181B18039372BBEF
:1030100000231093CA46FFF7BCBB0FAA04992046B1
:10302000FFF73AFB50BB1099119A01F1010ECC4603
:1030300048E5002A40F040819DF83710002900F053
:103040001B8101220DF1370110461D921C91CA46C9
:1030500001460AF1080A013007E5029B012A00F047
:103060009880022A0DD1029300260027B0E50FAA0E
:1030700004990698FFF710FB0028C9D0DDF810B0BE
:1030800097E7029300260027494600E05946F208D8
:1030900042EA4772F80806F007030746164630333F
:1030A00056EA070201F8013C01F1FF3BEED1029A1A
:1030B000D6077FF59DAD302B3FF49AAD0239302312
:1030C0000BF8013CA9EB010305938B4676E4039BC7
:1030D000089A8A42ACBF9B185B18039398E70222B8
:1030E0004DE4002F08BF0A2E52D3CB463046394656
:1030F0000A22002301F054FB30320BF8012D304638
:10310000394600230A2201F04BFB06460F4656EAD9
:103110000703EBD16CE50594CB464FE40FAA049965
:103120000698FFF7B9FA0028A8D1119ACA465EE7B7
:103130000FAA04990698FFF7AFFA00289ED1CA4655
:10314000FFF7C0BB6C5841005C5841000431166861
:1031500007910122002712E407980146043106680E
:10316000079100270BE40E6804310791002791E5D1
:1031700007990E680A46F717043207923046394617
:103180000FE5DBF8580000F07FFEBBF80C301AE7C3
:10319000029B02930DF1B00B303601230BF8416D09
:1031A00005930BE40FAA04990698FFF775FA002817
:1031B0007FF464AF1099119A481CCA4651E60FAAD1
:1031C00004990698FFF768FA00287FF457AF109922
:1031D000119A481CCA4648E4002A40F09180012018
:1031E0001146CA4641E60FAA04990698FFF754FA19
:1031F00000287FF443AF1098119A0130CA4667E661
:10320000D346D6E6079E073626F0070202F10801EC
:10321000D2E9006707910122FFF7B1BB079E07368D
:1032200026F00706D6E9000106F1080207920646D5
:103230000F46B6E4079E073626F0070202F10801A2
:10324000D2E9006707910022FFF799BB079E073676
:1032500026F0070101F108000790D1E9006719E5A0
:10326000CB46FFF7ABBB2D25764267EB47078DF8C2
:1032700037500122FFF788BB099BB3B911460120E3
:10328000CA46F2E5DBF8580000F0FEFD4FF0FF33D0
:103290000393FFF750BB0FAA04990698FFF7FCF9B8
:1032A00000287FF4EBAE119AA9E60EAB02221C9324
:1032B0001D920120CA46D0E50FAA04990698FFF78F
:1032C000EBF900287FF4DAAE1099119A481CCA462F
:1032D000A4E5079A03991368CD17084604322946D6
:1032E0000792C3E90001FFF754BA584607960293C4
:1032F000FFF746F9002405909DF83750FFF75EBBB5
:103300000FAA04990698FFF7C7F900287FF4B6AE14
:103310001099119A481CCA46A7E51099119A204E97
:103320000131FFF790BB062C28BF062405940796B1
:103330000194DFF870B0D5E41098194E013003E61F
:1033400005949DF83750079602930446FFF736BB65
:103350008646FFF7CEBB06980FAA5946FFF79CF9A1
:1033600000283FF424AE24E6079998F801200C6861
:10337000043144EAE474B8460791FFF73FBA8DF888
:1033800037503CE48DF8375021E58DF83750FFF782
:10339000F4BB8DF8375091E48DF8375069E400BFE5
:1033A0005C584100545841002DE9F0410C46ADF500
:1033B0008D6D8989666EE589199621F002010646B0
:1033C000E069ADF80C1017464FF48061626AADF801
:1033D0000E5098461AAD0023079016A8099206933E
:1033E000009504950291059100F048FD43463A4648
:1033F00069463046FFF790F9051E07DB30466946FF
:1034000000F028F9002818BF4FF0FF35BDF80C3048
:103410005B0603D5A38943F04003A381169800F00F
:103420002FFD28460DF58D6DBDE8F08138B5304B88
:103430001B6805460C4613B19A6B002A38D0B4F9C4
:103440000C2093B218070CD52069A8B113F0010223
:103450001ED0636900225B42A361A260F0B100202C
:1034600038BDD9063CD5580726D4206942F0080358
:10347000A3819BB20028E9D103F42072B2F5007F4A
:10348000E4D02846214600F02FFDA3892069DDE71E
:10349000990758BF6269A2600028E0D1B4F90C30E6
:1034A0001A06DDD543F04003A3814FF0FF3038BD4D
:1034B000184600F027F9C2E7216B51B104F140032F
:1034C000994204D0284600F043FAB4F90C200023B6
:1034D000236300232069636022F024022060C5E793
:1034E00042F0400209232B604FF0FF30A28138BD2B
:1034F0003C030020024B13B1024800F005B87047AE
:103500000000000075374100002301461A461846A6
:1035100001F01EB8B1F90C309AB22DE9F0410D4618
:10352000110780463AD46A6843F40063002AAB81ED
:103530006FDDAC6A002C49D000229BB2D8F8006045
:10354000C8F8002013F4805267D02A6D5F0705D5B4
:1035500069682B6B521A0BB1EB6BD21A0023E96925
:103560004046A047441C3CD0B5F90C302A692A607B
:1035700023F400630022AB81DB046A6047D4296B2B
:10358000C8F8006011B305F14003994202D04046EB
:1035900000F0DEF900202863BDE8F0812E69AEB1AD
:1035A0002C682E6091070CBF6B690023A41BAB60D5
:1035B0000AE0234632466F6AE9694046B847002868
:1035C000A4EB0004064404DD002CF2DC0020BDE87E
:1035D000F081AB8943F04003AB814FF0FF30BDE891
:1035E000F081D8F800401D2CF3D8194BE340DB43A1
:1035F00013F00103EDD1B5F90C206B6022F40063E8
:103600002969AB81DA042960B9D5002CB7D12865C6
:10361000B5E7EA6B002A8CDCD8E70123E96940466C
:10362000A047431C024602D0AB89AC6A8EE7D8F8AB
:103630000030002BF8D01D2B01D0162B02D1C8F87A
:103640000060C3E7AB8943F04003AB81BDE8F08184
:103650000100402038B50D46044608B1836BBBB16C
:10366000B5F90C0088B16B6EDB0701D4810517D565
:1036700020462946FFF74EFF6B6EDA07044602D458
:10368000AB899B0507D5204638BD0446204638BD8A
:1036900000F038F8E4E7A86D00F0F6FB204638BDEE
:1036A000A86D00F0EFFBE3E7014900F0AFBB00BFFE
:1036B0003946410010B5002304468181C281036070
:1036C0004360836043660361436183611946082256
:1036D0005C30FEF7FBFD07480749084A084B2062AB
:1036E000E4616162A262E36204F15800BDE8104047
:1036F00000F0C4BB7D434100A1434100DD434100D4
:10370000FD43410010B50446124800F0BBFBA26B1C
:10371000D2B904F53B731048C4F8E8320321C4F869
:10372000E022E063C4F8E41260680421FFF7C2FFFE
:1037300001220921A068FFF7BDFF02221221E068E3
:10374000FFF7B8FF0123A3630248BDE8104000F073
:103750009BBB00BF14240020A9364100014800F0A3
:1037600091BB00BF28240020014800F08DBB00BFA2
:103770002824002038B50A4C0A4D641BA4100AD036
:1037800004F18043013B05EB8305013C55F8043906
:103790009847002CF9D1BDE8384002F003B900BFCA
:1037A000B4594100B05941002DE9F04782B080463C
:1037B0008946144600F054FB012836D04A4604F1ED
:1037C0005C0301A9404600F075FE421C064625D068
:1037D000A8B39DF804E000250DF1040A09E0236870
:1037E0005A1C226083F800E00135B54227D215F853
:1037F0000AE0A368013B002BA360F0DAA769BB4293
:1038000071462246404602DBBEF10A0FE7D100F0C6
:10381000F9FD431CE8D102B0BDE8F087A38943F06D
:103820004003A38102B0BDE8F08709F1FF33FE2B0E
:10383000C4D85FFA89FE06468DF804E0CBE7484617
:1038400002B0BDE8F08700BF30B5536E13F0010F32
:10385000B2F90C30144683B005469AB201D19005F6
:103860001CD5900406D4626E43F4005342F4005217
:10387000A381626628462246FFF796FF636EDA0749
:10388000054602D4A3899B0502D5284603B030BD66
:10389000A06D00F0F9FA284603B030BDA06D01918B
:1038A00000F0F0FAB4F90C3001999AB2D9E700BFF0
:1038B000F8B5244F0C460646FEF756FDBB685D681A
:1038C000C4F57E610F3125F00305294421F47F61A1
:1038D00021F00F01A1F58054B4F5805F07DB0021D2
:1038E0003046FEF757FDBB682B44984204D0304663
:1038F000FEF740FD0020F8BD61423046FEF74AFD6C
:1039000001300DD0104BBA6819682D1B45F0010528
:103910003046091B55601960FEF72CFD0120F8BDEB
:1039200000213046FEF736FDBA68831A0F2BDEDD24
:10393000064C0549246843F00103001B53600860EE
:10394000D5E700BF680700203C100020700B002066
:10395000002944D02DE9F0410D468046FEF704FDD4
:1039600055F8047C694927F00103A5F10804E21821
:103970008E685068B24220F003005ED0FE075060AF
:103980000BD455F8087CE41B01F1080EA5687545B9
:103990003B446DD0E768EF60BD6015186D68ED07BA
:1039A0003ED543F001026260E350B3F5007F17D2C9
:1039B000DB08581C9A104D6851F83070A76001233D
:1039C000934001EBC0022B43083AE2604B6041F8A0
:1039D0003040FC604046BDE8F041FEF7CBBC70478C
:1039E0005A0A042A52D89A0902F13907FF0002F153
:1039F0003805C819CA59083890424FD0516821F08B
:103A000003018B4232D292689042F7D1C368A06022
:103A1000E3609C60C4604046BDE8F041FEF7AABC8C
:103A200095683B4FBD42034440D0D068E86043F006
:103A3000010285606260E350B7E7FF07034407D4E3
:103A400055F8082CA41A1344A068E268C26090607C
:103A5000304A126843F00100934260608C60B9D331
:103A60002D4B40461968FFF723FFB3E71046CDE71B
:103A700011184968C90744D49168D268CA600344E0
:103A800043F0010091606060E350A3E7142A16D868
:103A900002F15C07FF0002F15B05AAE7AA1001230F
:103AA0004D6893402B434B600346B0E743F001025F
:103AB0004C610C61E560A5606260E3508AE7542ABE
:103AC00006D81A0B02F16F07FF0002F16E0590E7AE
:103AD000B2F5AA7F06D8DA0B02F17807FF0002F1EF
:103AE000770586E740F25450824206D89A0C02F1DC
:103AF0007D07FF0002F17C057BE74FF47E777E2592
:103B000077E743F001016160136063E76807002015
:103B100070070020740B00206C1000209368002BAD
:103B200073D02DE9F04F8B8983B00C4619070090B4
:103B3000164626D5226922B313F0020035682CD030
:103B40004FF00009B04FC846B246B84543464A4612
:103B500028BF3B460098B8F1000F50D0E169666A73
:103B6000B047002858DDDAF808301B1A8144A8EB6A
:103B70000008CAF80830002BE7D1002003B0BDE8E8
:103B8000F08F21460098FFF751FC002840F0338168
:103B9000A389356813F00200D2D113F0010945D191
:103BA0004F46019637B39A05D4F8088040F18380D8
:103BB0004745C346C0F0AB8013F4906F40F0AC8033
:103BC0002068BA465A464946FEF71CFBA26823689D
:103BD000A2EB08025B44A2602360019A9368A3EB06
:103BE0000A03D144A7EB0A079360002BC5D0A38931
:103BF000002FD8D1D5F800906F680835D2E7D5F8F6
:103C00000090D5F8048008359FE7002070472146D2
:103C10000098FFF71FFD70B3B4F90C3043F0400378
:103C20004FF0FF30A38103B0BDE8F08F81463346EB
:103C30004E46A8469A464D464EB380B32068236947
:103C40006269B145CB4628BFB34698425F4604D966
:103C5000A36813449B4500F3A68093454BDB1346B2
:103C6000676AE16900982A46B847071ED4DDB9EBB8
:103C70000709CCD00120DAF80830DB1B3D44F61BE5
:103C8000CAF80830002B3FF478AF002ED5D108F1E8
:103C9000080313E9600098460833002EF9D0324635
:103CA0000A212846FEF794F9002800F0A18001308F
:103CB000A0EB0509C2E720682369984202D863692E
:103CC0009F425DD2B84528BFB84642464946FEF7F6
:103CD00099FAA3682268A3EB08034244A360226018
:103CE0000BB1C24679E721460098FFF7B3FC0028E4
:103CF00092D1C24671E75A462946FEF783FAA26876
:103D00002368A2EB0B025B44A2602360AFE720684C
:103D1000B846BA46BB4655E762692068216902EB9E
:103D20004208A0EB010A08EBD8780AF101004FEA3B
:103D3000680838444045424684BF804642465B0599
:103D400044D511460098FDF793FE8346002855D0D0
:103D500052462169FEF7BCF9A38923F4906343F02E
:103D60008003A3810BEB0A00A8EB0A03C4F810B090
:103D7000C4F814802060A360B846BA46BB4621E769
:103D80006FF00041B94228BF39464A4691FBF3F132
:103D90000098666A03FB01F3E169B047B0F1000ADD
:103DA0003FF71BAF38E71A4629460193FEF72AFA78
:103DB0002268019B00981A4422602146FFF74AFCC2
:103DC000019B00287FF428AF1F4650E7009800F0C1
:103DD0002FF983460028C5D1009D21692846FFF7A9
:103DE000B7FDB4F90C300C2223F080032A6015E7EC
:103DF00006F1010922E74FF0FF30BFE6009A0C23DD
:103E00001360B4F90C3009E700FCFF7F2DE9F8439B
:103E100010F538771FD0884606464FF000097D68B8
:103E2000BC68013D11D4A389012B05F1FF3508D9E8
:103E3000B4F90E3001332146304602D0C04749EA7A
:103E400000096B1C04F16804EDD13F68002FE6D136
:103E50004846BDE8F883B9464846BDE8F88300BF48
:103E6000044B054A1B685B6B002B08BF134693F895
:103E7000280170473C0300207C0B0020704700BFE6
:103E8000704700BF704700BF704700BF70B50C4659
:103E9000B1F90E10002990B015461E4614DB01AA98
:103EA00000F02CFC00280FDB029A02F47042A2F50D
:103EB0000052B2FA82F252094FF480634FF400606C
:103EC00032602B6010B070BDA289002312F0800018
:103ED000336004D0402218462A6010B070BD4FF401
:103EE00080632B6010B070BD8A8992070B4606D59F
:103EF00001F1430201211A601A6159617047F0B55E
:103F000083B001AB6A460C460646FFF7BFFF009937
:103F100005463046FDF7ACFDB4F90C30D8B1019A36
:103F2000154F0099F76343F08003A381206020615F
:103F300061611AB92B43A38103B0F0BD3046B4F9D7
:103F40000E1000F0EFFBA0B1A38923F0030343F0B0
:103F500001031BB2EEE79A05EED423F0030304F14C
:103F6000430243F002030121A381226022616161C7
:103F7000E2E7B4F90C30DDE7A936410070B4124C29
:103F800004F5806554F8083F5E6826F003060F2E9E
:103F90003146D4BF00200120E3689C4208D05A6813
:103FA000DB6822F003029C4200F101001144F6D1CB
:103FB0000834A542F0D1054B1A685E62521A586067
:103FC0001962DA6170BC7047680700203C1000205D
:103FD000F8B50B4D064608460F46FEF7C5F9FFF744
:103FE000CDFF0FCD34460FC40FCD0FC495E80300AD
:103FF00084E803003846FEF7BDF93046F8BD00BF3F
:104000003C10002082B049B15AB16BB113780B60FB
:104010001278101C18BF012002B0704701A9002AB5
:10402000F3D1104602B070476FF00100F4E700BF13
:10403000002900F095802DE9F04F0D46164683B01B
:10404000804606F10B07FEF78FF955F804EC162FA2
:104050002EF00304A5F108093CD810221746BE42F1
:104060003DD8944243DAC44B996809EB0400884276
:1040700000F0B480436823F0010101444968C90796
:104080004CD51EF0010F00F09B8031464046FDF7F5
:10409000EFFC064600283AD055F8043C23F0010313
:1040A0004B44A0F108029A4200F02181221F242AE9
:1040B00000F20781132A00F2DB8003462A461168CA
:1040C00019605168596092689A6029464046FFF726
:1040D0003FFC1CE027F00707002F3A46BFDA002616
:1040E0000C233046C8F8003003B0BDE8F08F2E46F0
:1040F000E31B0F2B1ED8D9F8043003F00103234330
:104100004C44C9F80430636843F0010363604046DF
:10411000FEF730F9304603B0BDE8F08F23F003031B
:10412000E11891421FDBC36882682E46D3600C46BB
:104130009A60DDE7D9F8042009EB070102F00102DB
:104140004C4443F001031743C9F804704B606368A3
:1041500043F00103083163604046FFF7F9FBD6E7FF
:104160001146FDF785BC1EF0010F8ED155F8081CD5
:10417000A9EB010ADAF8041021F003010B442344EF
:10418000934225DBC26881685646CA609160DAF8BE
:104190000C1056F8080F221F242AC160886000F214
:1041A0009480132A6FD92968CAF808106968CAF878
:1041B0000C101B2A00F2A28008350AF1100263E0FD
:1041C00055F8083CA9EB030ADAF8041021F00301C2
:1041D00063189342FFF659AF5646D8E7416821F07D
:1041E000030BA34407F11000834556DA1EF0010FBC
:1041F0007FF44BAF55F8081CA9EB010ADAF804105C
:1042000021F003018B445845E2DC5646DAF80C10E5
:1042100056F8080F221F242AC160886000F28F80A0
:10422000132A40F28A802968CAF808106968CAF817
:104230000C101B2A00F28A8008350AF11002296846
:10424000116069685160A96891600AEB0701ABEBE6
:10425000070242F0010299604A60DAF8043003F084
:1042600001031F434046CAF80470FEF783F851E784
:104270002B6803606B6843601B2A2DD800F108038C
:1042800005F108021BE73246296811606968516030
:10429000A96891601C46D1462AE709EB0701ABEB00
:1042A000070B4BF0010299604A6055F8043C03F09B
:1042B00001031F43404645F8047CFEF75BF82E4699
:1042C00028E72946FDF79EFFFFE6294630461C46B3
:1042D000D146FDF797FF0BE7AB688360EB68C360DF
:1042E000242A17D000F1100305F11002E7E650F878
:1042F000043C23F003031C442E46F9E6A968CAF8DF
:104300001010E968CAF81410242A0CD010350AF1EC
:104310001802B9E72B6903616B69436105F1180263
:1043200000F11803CBE62A69CAF818206A69CAF8AE
:104330001C2018350AF12002A6E732467FE72946FD
:1043400030460193FDF75EFF019B7EE7A968CAF83E
:104350001010E968CAF81410242A03D010350AF1A5
:1043600018026CE72A69CAF818206A69CAF81C2082
:1043700018350AF1200262E76807002010B50C46E4
:10438000B1F90E1000F0F6F9002803DB236D0344A9
:10439000236510BDA38923F48053A38110BD00BF02
:1043A0002DE9F0411646B1F90C201F46D3050C4605
:1043B000054607D500220223B1F90E1000F0C4F91A
:1043C000B4F90C20B4F90E1022F48052A2813B46BD
:1043D00032462846BDE8F04100F0A4B810B50C46BE
:1043E000B1F90E1000F0B0F9A389421C0EBF23F4FE
:1043F000805343F480532065A38110BDB1F90E10A2
:1044000000F008B9F8B50D461446064610B1836BA6
:10441000002B4BD0B4F90C20A369A36091B208071C
:1044200039D52369002B36D0EDB289042F4615D536
:1044300022686169D31A8B421CDA0133A168501CCF
:104440000139A1602060157062699A421AD0A3896F
:10445000DB0701D50A2D15D03846F8BD616E42F450
:10446000005221F40051A281226861666169D31A69
:104470008B42E2DB21463046FFF7ECF840B9226878
:104480000123DBE721463046FFF7E4F80028E3D0BC
:104490004FF0FF37E0E721463046FEF7C7FF002820
:1044A000F6D1B4F90C20236991B2BDE7FFF72AF9E0
:1044B000B0E700BFF0B5064685B01F4689B1104C85
:1044C000104D2468646B002C08BF2C46D4F8E040E3
:1044D000A047431C03D100228A233A60336005B011
:1044E000F0BD0C460649074A0968496B002908BF18
:1044F00011462246D1F8E04001A9A047E9E700BFF4
:104500003C0300207C0B002021B1FF2A04D80A7054
:1045100001207047084670478A2303604FF0FF3040
:10452000704700BF70B50D46084C114606461A4646
:10453000284600232360F9F789FD431C00D070BD95
:104540002368002BFBD0336070BD00BF2C240020FB
:104550002DE9F8432C4D0646286898460F469146AB
:10456000FFF790FC294B1C68D4F84831002B3ED053
:104570005A681F2A1CDC02F1010E76B103EB82019E
:104580000124C1F88890D3F8880194402043022E7A
:10459000C3F88801C1F8088123D00232C3F804E0CF
:1045A000286843F82270FFF76FFC0020BDE8F8830D
:1045B000174B0BB34FF4C870FDF74AFA0346D8B156
:1045C000D4F848210260002141600A46C4F848013D
:1045D0004FF0010EC0F88811C0F88C11002EDCD00D
:1045E000CCE7D3F88C110C43C3F88C41D5E704F524
:1045F000A673C4F84831BBE72868FFF745FC4FF0C5
:10460000FF30BDE8F88300BF780B00202858410038
:10461000511A410038B5074C00230546084623606F
:10462000FAF722F9431C00D038BD2368002BFBD0D9
:104630002B6038BD2C24002070B559B105460C46BE
:1046400010B1836B002B3CD0636ED80705D5B4F94D
:104650000C302BB90026304670BDA38999053CD596
:1046600021462846FEF756FFE36A064633B1E16964
:10467000284698470028B8BF4FF0FF36A3891A068E
:1046800022D4216B41B104F14003994202D0284663
:10469000FFF75EF900232363616C21B12846FFF721
:1046A00057F900236364FFF759F8636E0022DB07B4
:1046B000A2810ED5A06DFFF7E3FBFFF755F830465A
:1046C00070BDFFF71FF8BFE721692846FFF740F9E3
:1046D000D7E7A06DFFF7D8FBECE7A06DFFF7D2FBA3
:1046E000B4F90C30002BBBD1666E16F00106B1D1C7
:1046F000A06DFFF7C9FB304670BD00BF38B50B4653
:10470000074C05461146184600232360FAF7AFF818
:10471000431C00D038BD2368002BFBD02B6038BD74
:104720002C24002038B5074C00230546084623609A
:10473000FAF7A2F8431C00D038BD2368002BFBD049
:104740002B6038BD2C24002070B50D46084C114656
:1047500006461A46284600232360FAF78FF8431CC2
:1047600000D070BD2368002BFBD0336070BD00BF4C
:104770002C24002070B50D46084C114606461A46FA
:10478000284600232360F9F747FC431C00D070BD86
:104790002368002BFBD0336070BD00BF2C240020A9
:1047A00053B94AB9002908BF00281CBF4FF0FF3198
:1047B0004FF0FF3000F07AB9ADF1080C6DE904CE8E
:1047C00000F006F8DDF804E0DDE9022304B07047EC
:1047D0002DE9F0478C460D460446089E002B51D12A
:1047E0008A4217466DD9B2FA82FEBEF1000F0BD095
:1047F000CEF1200C01FA0EF520FA0CFC02FA0EF7AD
:104800004CEA050C00FA0EF44FEA174A250CBCFBE3
:10481000FAF81FFA87F90AFB18CC45EA0C4508FBA1
:1048200009F3AB420AD9ED1908F1FF3280F0238178
:10483000AB4240F22081A8F102083D44ED1AA4B237
:10484000B5FBFAF00AFB105544EA054400FB09F9F0
:10485000A14509D9E41900F1FF3380F00A81A1458F
:1048600040F2078102383C44A4EB090440EA0840C6
:104870000021002E61D024FA0EF40023346073600E
:10488000BDE8F0878B4207D9002E54D0002186E87E
:1048900021000846BDE8F087B3FA83F1002940F013
:1048A0008E80AB4202D3824200F2FA80841A65EB1A
:1048B00003050120AC46002E3FD086E81010BDE86D
:1048C000F08712B90127B7FBF2F7B7FA87FEBEF1FE
:1048D000000F34D1EB1B3A0C1FFA87FC0121B3FB0C
:1048E000F2F8250C02FB183345EA03450CFB08F3EC
:1048F000AB4207D9ED1908F1FF3002D2AB4200F20A
:10490000D1808046ED1AA3B2B5FBF2F002FB105540
:1049100043EA05440CFB00FCA44507D9E41900F167
:10492000FF3302D2A44500F2B8801846A4EB0C0471
:1049300040EA08409DE731463046BDE8F087CEF1B9
:10494000200405FA0EF307FA0EF720FA04F83A0CE1
:1049500025FA04F448EA0308B4FBF2F14FEA1845DB
:1049600002FB11441FFA87FC45EA044501FB0CF3E6
:10497000AB4200FA0EF409D9ED1901F1FF3080F0D5
:104980008A80AB4240F2878002393D44EB1A1FFA1D
:1049900088F5B3FBF2F002FB103345EA034500FB58
:1049A0000CF3AB4207D9ED1900F1FF386FD2AB42DF
:1049B0006DD902383D44EB1A40EA01418FE7C1F15D
:1049C000200722FA07F88B4005FA01F448EA0303AE
:1049D00020FA07FE4FEA134CFD404EEA040EB5FBE9
:1049E000FCF94FEA1E440CFB19551FFA83F844EA00
:1049F000054509FB08F4AC4202FA01F200FA01FA9B
:104A000008D9ED1809F1FF3043D2AC4241D9A9F1E0
:104A100002091D442D1B1FFA8EFEB5FBFCF00CFB9A
:104A200010554EEA054400FB08F8A04507D9E418E4
:104A300000F1FF3529D2A04527D902381C4440EAAD
:104A40000940A4EB0804A0FB02894C45C6464D462C
:104A500015D312D056B1BAEB0E0364EB050404FA79
:104A600007F7CB401F43CC40376074600021BDE89E
:104A7000F0871846F8E69046E0E6C245EAD2B8EB81
:104A8000020E69EB03050138E4E72846D7E7404604
:104A900091E78146BEE7014678E702383C4445E7A6
:104AA000084608E7A8F102083D442BE7704700BF1D
:104AB00001000000020000000400000008000000E7
:104AC00010000000200000004000000080000000F6
:104AD000000080000000000100000002000000044F
:104AE00000000008000000100000000000000000AE
:104AF00000000000000000000000000000000000B6
:104B000000000000000000000000000000000000A5
:104B1000302E332E3200000064617461000000000A
:104B2000737461636B0000006865617000000000D1
:104B30005A81000001280110020380025329035109
:104B4000FF01026902026B100580004040110881DC
:104B500002560009000F00088202560009000F00EB
:104B600002250103F0AA1104C00040000AC2010A94
:104B7000010A010A00900203F0AA1202D32003BF27
:104B800037BE00000128011002038102532903519E
:104B9000FF01026902026B102D7011000089108064
:104BA000078003C0078003C003C002000358002031
:104BB000C637000D000F00110008180010F0030C9C
:104BC0002000060B0B33058001404011088102567E
:104BD0000009000F00088202560009000F0002259C
:104BE0000103F0AA1002D10203F0AA1104C0004090
:104BF000000AC2010A010A010A00900203F0AA1287
:104C000002D32003BF37BE00012801100203800237
:104C100053290351FF01026900026B100580004017
:104C20004011088104AC0010001000088204AC00A0
:104C30001000100002250103F0AA1104C00040007A
:104C40000AC2010A010A010A00908203F0AA1202B4
:104C5000D32003BF37BE00000101020380025329A5
:104C60000351FF01026900026B10058000404011F2
:104C700008810256000A00100008820256000A004D
:104C8000100002350002250103F0AA110AC2010A30
:104C9000010A010A00900203F0AA1202D32003BF06
:104CA00037BE03F0AA1105C4AA55018004C5001F30
:104CB000FF00000001280110020381025329035163
:104CC000FF01026900026B102D7011000089108035
:104CD00009F004F804F804F804F80200041B0020AA
:104CE00091BF0011000F00190009180010F0030C0B
:104CF0002000060B0B330580013E3E11088101E1C7
:104D00000006001000088201E100060010000225E4
:104D10000103F0AA1002D10203F0AA110AC2010A8B
:104D2000010A010A00908203F0AA1202D32003BFF5
:104D300037BE0000012801100203810253290351EC
:104D4000FF01026900026B102D70110000891080B4
:104D500009F004F804F804F804F80200041B002029
:104D600091BF0011000F00190009180010F0030C8A
:104D70002000060B0B330580013E3E11088101E146
:104D80000006001000088201E10006001000022564
:104D90000103F0AA1002D10203F0AA110AC2010A0B
:104DA000010A010A00900203F0AA1202D32003BFF5
:104DB00037BE00000128011002038102532903516C
:104DC000FF01026900026B102D7011000089108034
:104DD00009F004F804F804F804F80200041B0020A9
:104DE00091BF0011000F00190009180010F0030C0A
:104DF0002000060B0B330580013E3E11088101E1C6
:104E00000010001000088201E100100010000225CF
:104E10000103F0AA1002D10203F0AA1104C000405D
:104E2000000AC2010A010A010A00900203F0AA1254
:104E300002D32003BF37BE00585F666D747B828942
:104E400090979EA5AC000000BD351725000100001D
:104E50005658523030000000302E332E3200000001
:104E600055534152540000004661696C65642074DA
:104E70006F2063726561746520757361727420744C
:104E800061736B0D0A00000048494420436F6D6D4B
:104E9000616E6473000000004661696C6564207493
:104EA0006F206372656174652048494420636F6DAB
:104EB0006D616E642070726F636573736F722074BE
:104EC00061736B0D0A000000484944205265706F01
:104ED000727400004661696C656420746F206372AF
:104EE000656174652048494420706572696F646922
:104EF00063207265706F7274207461736B0D0A00A9
:104F000056585244454C45544500000043524153C5
:104F1000484E4F570000000000FFFFFFFFFFFF005B
:104F200009279550D2040000021E0104A500007854
:104F3000E700000000000000000000000000010188
:104F40000101010101010101010101010101CAB4D5
:104F50000080F080187040209200FFFF0000001ECB
:104F6000A5510080A00020A040200204FFFF000007
:104F7000001E000000000000000000000000000013
:104F80000000000000000010000000000000000011
:104F900000000000000001757012790000000000A0
:104FA0000000000000000000000000000000000001
:104FB00000000000000000000000000000000000F1
:104FC00000000000000000000000000000000000E1
:104FD00000000000000000000000000000000000D1
:104FE00000000000000000000000000000000000C1
:104FF00000000000000000000000000000000000B1
:1050000000000000000000000000000000000000A0
:10501000000000000000759000FFFFFFFFFFFF0091
:1050200009273412D2040000FF200104A5000078F3
:10503000007875AA553BB2291050540000000101B8
:105040000101010101010101010101010101000052
:105050000010000000000000000000000000000040
:105060000000001000000000000000000000000030
:105070000000000000100000000000000000000020
:1050800000000000000000FC004265796F6E640AB9
:10509000202020202020015B7020790700220914A5
:1050A00061430C88DF137F003F801F00EF0917006A
:1050B0000E8001007E00073A029281000800000085
:1050C00000000000000000000000000000000000E0
:1050D00000000000000000000000000000000000D0
:1050E00000000000000000000000000000000000C0
:1050F00000000000000000000000000000000000B0
:10510000000000000000000000000000000000009F
:10511000000000000000209000FFFFFFFFFFFF00E5
:1051200009279550D2040000021E0104A500007852
:10513000E700000000000000000000000000010186
:105140000101010101010101010101010101CAB4D3
:105150000080F080187040209200FFFF0000001EC9
:10516000A5510080A00020A040200204FFFF000005
:10517000001E000000000000000000000000000011
:10518000000000000000001000000000000000000F
:105190000000000000000175701279000003001487
:1051A000689F0080FF137F003F801F00FF091F00E2
:1051B0000F8001000000000000000000000000005F
:1051C00000000000000000000000000000000000DF
:1051D00000000000000000000000000000000000CF
:1051E00000000000000000000000000000000000BF
:1051F00000000000000000000000000000000000AF
:10520000000000000000000000000000000000009E
:10521000000000000000B19000FFFFFFFFFFFF0053
:1052200009273412D2040000FF200104A5000078F1
:10523000007875AA553BB2291050540000000101B6
:105240000101010101010101010101010101000050
:10525000001000000000000000000000000000003E
:10526000000000100000000000000000000000002E
:10527000000000000010000000000000000000001E
:1052800000000000000000FC004265796F6E640AB7
:10529000202020202020015B7020790700220914A3
:1052A00041B70E88DF137F003F801F00EF09170012
:1052B0000E8001007E00073A029281000800000083
:1052C00000000000000000000000000000000000DE
:1052D00000000000000000000000000000000000CE
:1052E00000000000000000000000000000000000BE
:1052F00000000000000000000000000000000000AE
:10530000000000000000000000000000000000009D
:10531000000000000000CA9000FFFFFFFFFFFF0039
:1053200009273412D2040000FF200104A5000078F0
:10533000007875AA553BB2291050540000000101B5
:10534000010101010101010101010101010100004F
:10535000001000000000000000000000000000003D
:10536000000000100000000000000000000000002D
:10537000000000000010000000000000000000001D
:1053800000000000000000FC004265796F6E640AB6
:10539000202020202020015B7020790700220914A2
:1053A00039540F88DF137F003F801F00EF0917007B
:1053B0000E8001007E00073A029281000800000082
:1053C00000000000000000000000000000000000DD
:1053D00000000000000000000000000000000000CD
:1053E00000000000000000000000000000000000BD
:1053F00000000000000000000000000000000000AD
:10540000000000000000000000000000000000009C
:10541000000000000000349000FFFFFFFFFFFF00CE
:1054200009273412D2040000FF200104A5000078EF
:10543000007875AA553BB2291050540000000101B4
:10544000010101010101010101010101010100004E
:10545000001000000000000000000000000000003C
:10546000000000100000000000000000000000002C
:10547000000000000010000000000000000000001C
:1054800000000000000000FC004265796F6E640AB5
:10549000202020202020015B7020790700220914A1
:1054A0001EF50A88FF0EFF003F801F007F071B00CC
:1054B0000E8001007E00073A029281000800000081
:1054C00000000000000000000000000000000000DC
:1054D00000000000000000000000000000000000CC
:1054E00000000000000000000000000000000000BC
:1054F00000000000000000000000000000000000AC
:10550000000000000000000000000000000000009B
:10551000000000000000869000FFFFFFFFFFFF007B
:1055200009273412D2040000FF200104A5000078EE
:10553000007875AA553BB2291050540000000101B3
:10554000010101010101010101010101010100004D
:10555000001000000000000000000000000000003B
:10556000000000100000000000000000000000002B
:10557000000000000010000000000000000000001B
:1055800000000000000000FC004265796F6E640AB4
:10559000202020202020015B70207907002209288C
:1055A00039540F88DF137F003F801F00EF09170079
:1055B0000E8001001EF50A08FF0EFF003F801F004D
:1055C0007F071B000E8001007E00073A02928100D7
:1055D00008000000000000000000000000000000C3
:1055E00000000000000000000000000000000000BB
:1055F00000000000000000000000000000000000AB
:10560000000000000000000000000000000000009A
:10561000000000000000E190766964656F5F7072C1
:105620006F6300004661696C656420746F2063726B
:105630006561746520766964656F2070726F63655B
:1056400073736F72207461736B0D0A0070726F78E0
:105650005F74696D656F75745F74696D6572000064
:10566000FF00FF00493243004661696C65642074A5
:105670006F206372656174652049324320746173E1
:105680006B0D0A0054494D45445F53544152540038
:105690004661696C656420746F206372656174652E
:1056A0002074696D65642073746172747570207400
:1056B00061736B0D0A000000414443004661696C50
:1056C000656420746F206372656174652041444392
:1056D000207461736B0D0A004C4544004661696C8F
:1056E000656420746F20637265617465204C454465
:1056F000207461736B0D0A0046414E004661696C6F
:10570000656420746F206372656174652046616E04
:10571000207461736B0D0A00313233342020202055
:1057200020202020202020200000000049444C455B
:1057300000000000546D725100000000546D722092
:105740005376630000C20100C000000000080000A2
:10575000000000002D2D2042696773637265656E3D
:10576000204265796F6E64202D2D0A004449535004
:105770004C4159424F4152442056302E342E320073
:105780002D2D202573202D2D0A0000002D2D2056B3
:10579000657273696F6E202573202D2D0A0000003D
:1057A00031313A33353A3330000000004F63742012
:1057B00033312032303234002D2D20436F6D70692B
:1057C0006C65643A202573202573202D2D0A000076
:1057D0005553424C6F6164004661696C6564207486
:1057E0006F2063726561746520555342204C6F6170
:1057F000646572207461736B0D0A0000484944208F
:10580000436F6D6D616E6400737461636B206F76BE
:105810006572666C6F772025782025730D0A00006D
:105820006C6F6766000000004003002030313233A7
:10583000343536373839414243444546000000008C
:1058400030313233343536373839616263646566F6
:1058500000000000286E756C6C29000020202020BC
:1058600020202020202020202020202030303030F8
:1058700030303030303030303030303043000000A5
:10588000504F5349580000002E00000000202020F7
:1058900020202020202028282828282020202020E0
:1058A00020202020202020202020202020881010B0
:1058B000101010101010101010101010100404040C
:1058C00004040404040404101010101010104141CA
:1058D00041414141010101010101010101010101B8
:1058E00001010101010101011010101010104242CC
:1058F0004242424202020202020202020202020288
:105900000202020202020202101010102000000027
:105910000000000000000000000000000000000087
:105920000000000000000000000000000000000077
:105930000000000000000000000000000000000067
:105940000000000000000000000000000000000057
:105950000000000000000000000000000000000047
:105960000000000000000000000000000000000037
:105970000000000000000000000000000000000027
:105980000000000000000000000000000000000017
:10599000F8B500BFF8BC08BC9E467047F53441001E
:1059A00029444000F8B500BFF8BC08BC9E467047CB
:1059B000054440001CEEFF7F0100000030B482B0BF
:1059C000049C5BB31D46036843F480330360C9B293
:1059D00041F0B441416083680193019B13F0010FD2
:1059E000F9D1002306E0990001F58001096845F826
:1059F00023100133A342F6D3D2B242F0B442426044
:105A000083680193019B13F0010FF9D0036823F41D
:105A100080330360002002B030BC70470220FAE7F8
:105A20000160704782B0416083680193019B13F06D
:105A3000010FF9D0019800F00E0002B0704700008D
:105A40007144400075444000774440007B4440006E
:105A50007F444000B9444000094540008144400073
:105A6000854440009144400009022200010100C029
:105A700032090400000103000000092111010001A6
:105A800022260007058103400004000012010002E5
:105A900000000040BD3501100001010203010000BB
:105AA000B8020020BC000020F40000200180FFFFAD
:105AB000FFFF00000110FFFF0210FFFF0310FFFFB8
:105AC0000410FFFF0120FFFF0220FFFF0500000080
:105AD00001000000185541000A010100807C797620
:105AE00073706D6A6764615F5C595754524F4D4BD8
:105AF00048464442403E3B3A38363432302F2D2B14
:105B00002A282725242221201E1D1C1B1A1817169F
:105B1000151413121111100F0E0D0D0C0B0B0A0999
:105B20000908080707060605050404040303030320
:105B30000202020201010101010100000000000057
:105B40000000000101020202020203030303030337
:105B500003040404040405050505050606060707F5
:105B6000070808080909090A0A0B0B0C0C0D0D0E91
:105B70000F0F1011111213141515161718191B1CDD
:105B80001D1E202122242527292A2C2E303234378D
:105B9000393C3E4144474A4D5054575B5F63676C04
:105BA00070757A80474700009802002008020020A4
:105BB0000000000010020020AC0200200902850055
:105BC000030100C032080B000201010002090400B9
:105BD00000000101000209240100011E0001010C66
:105BE0002402010102000203000000092403020153
:105BF0000100010009040100000102000209040182
:105C0000010101020002072401020101000B24022C
:105C1000010202100180BB0009058405000101009A
:105C20000007250100000000090402000103000034
:105C3000000921110100012226000705810340000F
:105C4000040000001201000200000040BD35010107
:105C5000000101020301000094000020A8000020C0
:105C6000B802002041B6400061B64000B9B640001D
:105C700063B640000000000006FFFF0901A1010912
:105C8000020903150026FF007508954081020906E8
:105C90000907150026FF0075089540B102C00000F5
:105CA00000030000000000000000000000000000F1
:105CB00000000000000000000000000000000000E4
:105CC000000000000403090442696773637265659C
:105CD0006E0000004265796F6E64000100127A0068
:105CE000AAAAAAAA010000004003002000000000A8
:105CF0002C06002094060020FC0600200000000076
:105D00000000000000000000000000000000000093
:105D10000000000000000000000000000000000083
:105D20000000000000000000000000000000000073
:105D30000000000000000000000000000000000063
:105D40000000000000000000000000000000000053
:105D50000000000000000000000000000000000043
:105D60000000000000000000000000000000000033
:105D70000000000000000000000000000000000023
:105D80000000000000000000000000000000000013
:105D90000000000001000000000000000E33CDAB49
:105DA00034126DE6ECDE05000B0000000000000080
:105DB00000000000000000000000000000000000E3
:105DC00000000000000000000000000000000000D3
:105DD00000000000000000000000000000000000C3
:105DE00000000000000000000000000000000000B3
:1061100000000000000000000000000068070020F0
:106120006807002070070020700700207807002013
:1061300078070020800700208007002088070020C3
:106140008807002090070020900700209807002073
:1061500098070020A0070020A0070020A807002023
:10616000A8070020B0070020B0070020B8070020D3
:10617000B8070020C0070020C0070020C807002083
:10618000C8070020D0070020D0070020D807002033
:10619000D8070020E0070020E0070020E8070020E3
:1061A000E8070020F0070020F0070020F807002093
:1061B000F807002000080020000800200808002040
:1061C00008080020100800201008002018080020EF
